:020000040002F8
:1070000018900020C5730200CD730200CF730200F8
:10701000D1730200D3730200D57302000000000098
:10702000000000000000000000000000D773020014
:10703000D973020000000000DB730200DD73020060
:1070400075810200DF730200058B020031870200A8
:1070500045870200DF730200B5800200D984020078
:10706000D58A0200ED8A0200DF730200DF7302009E
:10707000DF730200DF730200DF730200DF730200C0
:10708000158B0200D1810200DF730200DF73020062
:10709000DF730200DF7302006D870200DF730200FE
:1070A000DF730200DF730200DF730200DF73020090
:1070B000BD810200DF73020000000000000000003C
:1070C000DF730200DF730200DF73020059870200E2
:1070D000E9810200DF730200DF730200DF73020048
:1070E000DF7302000000000000000000000000004C
:1070F00000000000DF73020000000000DF730200E8
:10710000000000000000000000000000000000007F
:10711000000000000000000000000000000000006F
:10712000000000000000000000000000000000005F
:10713000000000000000000000000000000000004F
:10714000000000000000000000000000000000003F
:10715000000000000000000000000000000000002F
:10716000000000000000000000000000000000001F
:10717000000000000000000000000000000000000F
:1071800000000000000000000000000000000000FF
:1071900000000000000000000000000000000000EF
:1071A00000000000000000000000000000000000DF
:1071B00000000000000000000000000000000000CF
:1071C00000000000000000000000000000000000BF
:1071D00000000000000000000000000000000000AF
:1071E000000000000000000000000000000000009F
:1071F000000000000000000000000000000000008F
:10720000DFF810D000F042FA00480047C1D2020077
:10721000AFF300801890002030B450E8012F93B2F3
:10722000C48923448489A34228BF1B1B0489A34229
:1072300002BFBFF32F8F002007E0C3EA020340E83C
:107240000134002CE9D14FF001000A6030BC7047D6
:1072500050E8012FC2EA024240E801210029F7D19B
:10726000704730B450E8022F1FFAA2F3C488A3423B
:1072700002BFBFF32F8F00200DE0C489234484890F
:10728000A34228BF1B1BC2EA034340E80234002C80
:10729000E8D14FF001000A6030BC704750E8022F7F
:1072A000C2EA224240E802210029F7D17047034692
:1072B00053E8022FD988B2EB324F4FF0000017BFCE
:1072C00092B241EA014142EA014104E05A68B2EB5C
:1072D000324F08BF012043E80212002AE8D170476C
:1072E00030B4044654E8000F0D4644E80053002B28
:1072F000F8D1156030BC704730B4044654E8000F34
:1073000040EA010544E80053002BF7D1156030BC7A
:10731000704730B4044654E8000F00EA010544E821
:107320000053002BF7D1156030BC704730B40446D1
:1073300054E8000F80EA010544E80053002BF7D120
:10734000156030BC704730B4044654E8000F00EBC1
:10735000010544E80053002BF7D1156030BC70479D
:1073600030B4044654E8000FA0EB010544E8005394
:10737000002BF7D1156030BC704770B404464FF055
:10738000000054E8006F0D68AE4207BF44E80023D8
:10739000012044E800630E60002B1CBF0020F0E7D2
:1073A00070BC704730B4044654E8000F88422CBFCC
:1073B000451A054644E80053002BF5D1156030BC52
:1073C000704700000648804706480047FEE7FEE792
:1073D000FEE7FEE7FEE7FEE7FEE7FEE7FEE7FEE785
:1073E0001989020001720200004870471448030026
:1073F00010B50446FFF7F8FF0068005D00F00100DB
:1074000010BD40EA01039B0703D009E008C9121F21
:1074100008C0042AFAD203E011F8013B00F8013B4E
:10742000521EF9D27047D2B201E000F8012B491E7A
:10743000FBD270470022F6E710B513460A46044611
:107440001946FFF7F0FF204610BD421C10F8011B43
:107450000029FBD1801A704730B50446002003464E
:1074600000E05B1C934203D2E05CCD5C401BF8D093
:1074700030BD034611F8012B00F8012B002AF9D189
:10748000184670470FB400B58DB010A909900B9045
:1074900000914FF0FF300A9000200C9005480690B4
:1074A000054807906A4609A80F9900F0C1F80DB089
:1074B0005DF814FB4D7602006B7602002DE9FF5F4C
:1074C0001D464FF0FF3BD5E9014691465F464FF020
:1074D0000008A9697F1C01988847296A8246884765
:1074E0000028F6D1BAF1FF3F0CD024F4C064002E7E
:1074F00019DD600614D5BAF12B0F09D0BAF12D0FA2
:107500000ED103E0584604B0BDE8F09F44F4806417
:10751000A9697F1C01988847761E8246002E02DDED
:10752000BAF1300F03D0B9F1000F26D032E0A969CB
:10753000761E44F400747F1C019888478246002E12
:1075400005DDBAF1780F06D0BAF1580F03D0B9F1C2
:10755000000F10D01EE0B9F1000F02D0B9F1100FEA
:1075600018D1A969761E24F400747F1C01988847FD
:107570008246102002E0082000E00A20814609E04F
:1075800008FB0908A969761E44F400747F1C019861
:1075900088478246002E05DD4946504600F034F803
:1075A0000028EDDAE96901988847A00502D46FF058
:1075B0000100A8E7E00725D1600613D5600502D5D4
:1075C000C8F1000000E0404629680A1D2A600968E9
:1075D000220501D5087015E0220701D5088011E0C9
:1075E00008600FE02868011D29600068210502D5A8
:1075F00080F8008006E0210702D5A0F8008001E0B5
:10760000C0F8008038467EE73A2800D2303820F0B3
:107610002002412A01D3A2F13700884201D34FF062
:10762000FF307047026811441378016018467047B4
:10763000D160044951610449116200211161114670
:1076400000F036B825760200F1730200426842B1BC
:10765000016811F8013B23B1521EC0E9001218461F
:1076600070470121C160881E704742685AB1C368E3
:10767000016843B983688B4205D0491E521CC0E99A
:107680000012002070474FF0FF307047064C074D46
:1076900006E0E06840F0010394E8070098471034E2
:1076A000AC42F6D3FFF7B0FD305303005053030054
:1076B0002DE9F34F8BB04FF0000801F10C000C46A0
:1076C0004FF0010B46460DF1080A01906269012155
:1076D00001989047051E2DD0252D2CD0216A884772
:1076E000C0B16269012101989047216A884700284A
:1076F000F7D1411E62690198904700E0761CA169AC
:107700000B988847216A88470028F7D1E1690B98D0
:107710008847DBE7A1690B9888470746A84201D153
:10772000761CD3E7E1690B9888477F1C02D1B8F13A
:10773000000F6FD047E1002762693D463946019846
:1077400090472A2804D162690121019890470125B8
:10775000DFF888926269012101989047A0F1300119
:107760000A290AD24F45E5DC07EB870100EB410708
:10777000303FDFD445F01005ECE7E90601D46FF0A7
:1077800000476C280AD04C2814D0682815D06A28E5
:107790000DD074281CD07A281AD01DE0626901210E
:1077A000019890476C2802D045F0040514E045F09C
:1077B00002050DE045F020050AE06269012101980B
:1077C0009047682802D045F0080505E045F40065BB
:1077D0006269012101989047C4E9015765283DD0AD
:1077E00019DC58287AD00CDC452837D004DC252851
:1077F00026D0412831D131E046282FD047282CD13E
:107800002CE05B2877D0612828D063287CD06428BE
:1078100023D15AE0D1E06F2848D008DC66281DD07B
:1078200067281BD0692821D06E2816D127E0702840
:1078300045D0732868D0752847D078280DD14DE001
:10784000A1690B988847054625283FF469AFE1698F
:107850000B9888476D1C3FF46AAFB4E023466A4634
:107860006FF001000B99AFF300809FE045F04000FE
:107870006060A80723464FF0000236D43EE0E807D8
:107880007FF447AF2068011D21600068290501D5FC
:1078900006701BE7290701D5068017E7A90703D55E
:1078A000F117C0E9006111E706600FE745F04000FD
:1078B0006060A80723464FF0080216D41EE040F689
:1078C0000E0125EA0100606016E045F040006060AE
:1078D000A80723464FF00A0207D40FE045F0400006
:1078E0006060A80708D5234610226FF001000B99AD
:1078F000AFF300805AE007E0234610226FF001004A
:107900000B99FFF7DBFD51E04FF000094F464B4666
:10791000632802D05B2807D041E02079C00601D45B
:107920000120A06001273AE0626901210198904797
:107930005E2805D14FF001096269494601989047D8
:10794000216939B900210A46534643F82120491CD0
:107950000829FADBB0B3216969B9C11700EBD1621C
:1079600053110AEB830122F01F02821A01200B68D7
:10797000904003430B6062690121019890475D28A4
:10798000E8D1B9F1000F09D00020514651F820206C
:10799000D24341F82020401C0828F7DB02AB2246E6
:1079A00000976FF001000B99AFF3008000280CDA0C
:1079B000401C08D1BBF1000F05D04FF0FF300DB0D7
:1079C000BDE8F08FFFE74046F9E7E90701D108F18C
:1079D000010806444FF0000B78E60000CCCCCC0C3C
:1079E00070B58C1810F8015B15F0070301D110F881
:1079F000013B2A1106D110F8012B03E010F8016BAE
:107A000001F8016B5B1EF9D12B0705D40023521E30
:107A10000DD401F8013BFAE710F8013BCB1A921C98
:107A200003E013F8015B01F8015B521EF9D5A14296
:107A3000D8D3002070BD00002CB5294800F080F894
:107A400028480078002847D100BF274A012127484D
:107A500002F01EF80546D5B125482649264A891A5E
:107A6000C9080322CDE9000542EA014040F215238E
:107A700022A228A106F0E6FF06F01EFE00BF00BF0E
:107A800024B100BF204601F035FD00BF00BF00BF9C
:107A900000BF284A0021284801F0FAFF0546D5B169
:107AA00026481449144A891AC9080322CDE9000559
:107AB00042EA014040F2162310A216A106F0C2FFCE
:107AC00006F0FAFD00BF00BF24B100BF204601F060
:107AD00011FD00BF00BF00BF0120024908702CBD8E
:107AE00011950200652D0020558202009C43030081
:107AF00064480300F8530300605303007372635C2F
:107B00006170705F626C655F736572766963652E24
:107B10006300000025733A2564205A4552524F52A3
:107B20005F434845434B28257329206661696C3AB9
:107B30002564000019820200A0430300BC48030032
:107B400004490A680968491C024B1960024941F856
:107B500022007047D02D0020DC5500207047704770
:107B6000704700002CB5002109200CF0E7FB00BF96
:107B7000114A0121114801F08BFF0546CDB1104893
:107B80001049114A891AC9080322CDE9000542EAC1
:107B900001402B230DA215A106F054FF06F08CFD29
:107BA00000BF00BF24B100BF204601F0A3FC00BF0E
:107BB00000BF00BF2CBD00000D7C0200A4430300E9
:107BC000B4490300F8530300605303007372635C0D
:107BD000626F6172645C626F6172645F6C69676836
:107BE000745F6374726C2E630000000025733A2585
:107BF00064205A4552524F525F434845434B282513
:107C00007329206661696C3A2564000010B504464A
:107C10002348007830B92348007808B3002000F0EA
:107C200075F836E01E480078012806D11D48007816
:107C3000B0B9012000F06AF82BE01948007802285A
:107C400027D119480068022818DA1749086800EB9C
:107C5000D0714910A0EB410119B9012000F056F88C
:107C600017E01149086800EBD0714910A0EB410101
:107C700001290ED1002000F049F80AE00A48006806
:107C800064214843B0F57A7F03DB00200649086091
:107C900010BD05480068401C0349086000BFF7E7B5
:107CA000D82D0020D92D0020DC2D0020014800789F
:107CB00070470000D82D002010B50446114804700C
:107CC00024B1012C0AD0022C18D10FE00E48006814
:107CD00001F057FF002000F019F810E00A48006892
:107CE00001F04FFF012000F011F808E0002240F2FF
:107CF00066610548006801F015FF00E000BF00BFA5
:107D000010BD0000D82D0020A443030038B5044660
:107D10008CB109200090684606F002FB054601215F
:107D2000009A01FA02F0C5F8080500BF00BF012063
:107D30000A49087010E009200090684606F0F0FA41
:107D400005460121009A01FA02F0C5F80C0500BFB2
:107D500000BF00200149087038BD0000D92D002067
:107D600010B520480078022800D110BD01221EA1C4
:107D7000002004F037FA002003F01EFF0022114615
:107D8000052006F04FFA002211460B2006F04AFAB1
:107D900000221146112006F045FA00221146042067
:107DA00006F040FA01211E2006F056FB642005F083
:107DB0000DFF00211E2006F04FFB0021012006F0E0
:107DC0004BFB00211C2006F047FB1E2005F0FEFEA9
:107DD00001211C2006F040FB02200249087000BF70
:107DE000C3E70000002E0020000000002DE9F8434A
:107DF00057480078012801D1BDE8F88301211E20F1
:107E000006F02AFB0121084606F026FB1E2005F09D
:107E1000DDFE00211E2006F01FFB01244FF00A08A2
:107E200005E0002003F064FD0446A8F10108B8F164
:107E3000000F01D0002CF4D1002C25D04549464A32
:107E4000891AC908032242EA0140224643A106F0EA
:107E5000C9FD00BF49A03F493F4A891AC90803220A
:107E6000009042EA01409A2345A24DA106F0D6FDBA
:107E700006F022FC00BF4FF0000800BF002001F018
:107E800039FB00BF00BF00BF3249334A891AC90815
:107E9000032242EA014048A106F09AFD01224EA1C8
:107EA0004E4804F09FF90546002D24D029492A4A5E
:107EB000891AC908032242EA014049A106F088FD57
:107EC00000BF2EA02349244A891AC9080322009022
:107ED00042EA0140A1232AA231A106F09FFD06F04B
:107EE000EBFB00BF4FF0000800BF002001F002FBD9
:107EF00000BF00BF00BF3E48006841693C4888475A
:107F000040684FF48011B1FBF0F6394800684169D0
:107F1000374888470068B0FBF6F70E490E4A891AC1
:107F2000C908032242EA014032A106F051FD094985
:107F3000094A891AC908032242EA01403A4631A196
:107F400006F050FD01200249087000BF54E7000010
:107F5000002E0020F8530300605303004469736B44
:107F600020696E697469616C697A6174696F6E20E9
:107F70006661696C65642E20256400003000000095
:107F80007372635C626F6172645C626F6172645F82
:107F90007364636172645F6472697665722E6300F4
:107FA00025733A2564205A4153534552542825736A
:107FB00029206661696C00004469736B20696E69F1
:107FC0007469616C697A6174696F6E20737563633B
:107FD00065656465642E0000000000000456002002
:107FE0004D6F756E74206661696C65642E000000CB
:107FF000B04303004D6F756E7420737563636573D2
:108000007300000043617061636974793A202564EC
:10801000204D42000148007870470000002E0020EB
:1080200010B51E48007800B110BD00221146052091
:1080300006F0F8F8002211460B2006F0F3F80022B3
:108040001146112006F0EEF800221146042006F039
:10805000E9F803211C200CF071F901211C2006F025
:10806000FBF9032101200CF069F90021012006F041
:10807000F3F903211E200CF061F900211E2006F007
:10808000EBF90020064908700121064803F07EFE46
:1080900001200249087000BFC6E70000012E002041
:1080A000002E0020042E00200148007870470000B8
:1080B000B82D00202DE9FC470026002000900190FB
:1080C0004FF480770125002410E0384606F0FAF9D5
:1080D00040B100BF25480068284018B1384606F076
:1080E000E3F92E436D00381D87B2641C082CECD3D5
:1080F0004FF4BE7006F0E6F950B14FF4BE7006F0D2
:10810000D3F946F000466A460221002006F0C4F882
:10811000F0B210B3012500241DE005EA0600C0B14D
:1081200000BF134850F82400C0F30520814600BF6B
:108130000F4850F82400C0F301408246204602F068
:1081400037FE8046B8F1000F02D051464846C0477E
:1081500000BF6D00641C082CDFD306F0004010B196
:10816000684608F04DFCBDE8FC8700000463004051
:108170001065004010B54FF4807005F00BFD50B154
:108180004FF4807005F00FFD012005F015FD0A4841
:108190000168002088474FF4827005F0FBFC50B165
:1081A0004FF4827005F0FFFC022005F005FD024847
:1081B00001680120884710BD202E002010B502491B
:1081C000024804F0ABFE10BD302E002000C001407C
:1081D00010B5034A1068034A1168884710BD0000B3
:1081E000802E00207C2E002010B5042200210248A1
:1081F00004F0E6FE10BD00000040024010B5002073
:10820000034908700348006801F0BBFC002010BD62
:10821000642D00209C43030010B50446024800680A
:1082200000F004F810BD0000602D002070B5054678
:10823000074C07266A20A070002060700320207081
:10824000C4F80350314620460BF0A7FE70BD000075
:10825000D44F00202DE9FC4E81466548007808B9CE
:10826000BDE8FC8E6348006800284AD14FF4807155
:108270006148FFF7DFF84FF480725F495F4800689C
:1082800000F0C2FA8246BAF1000F36DC5C495D4A62
:10829000891AC908032242EA01405BA106F098FB53
:1082A00000BF60484FF4F67102685F48006801F053
:1082B00039FC8346BBF1000F1BD05C485049514A42
:1082C000891AC9080322CDE9000B42EA0140C42300
:1082D00057A25DA106F0B6FB06F0EEF900BF00BFA5
:1082E000B8F1000F04D000BF404601F003F900BF11
:1082F00000BF00BFFFF782FFB2E73E48C0F800A012
:1083000000BF3C48006800B9AAE70BF023FC054613
:10831000802D01DA284600E08020054635480068B7
:10832000C0F580703449461832480068A84201DD23
:10833000284601E02F48006807463149314A891A2A
:10834000C908032242EA01402A4900953A460B68CF
:1083500045A106F063FB0BF0EBFE60B92849294A02
:10836000891AC908032242EA014043A106F030FB02
:10837000FFF744FF74E7B8B2019001A930460BF053
:10838000B3FD044600BF0CB3082C0CD11C491D4A98
:10839000891AC908032242EA01403FA106F018FBEE
:1083A000FFF72CFF5CE7112C01D0132C00D157E70D
:1083B0001349144A891AC908032242EA0140224695
:1083C0003DA106F00FFBFFF719FF49E7002006E08B
:1083D000315C144A12681144124A1160401CB842C0
:1083E000F6D304480068C01B0249086000BF37E7A5
:1083F000642D00205C2D0020F8510020582D002015
:10840000F853030060530300726561642066696C71
:108410006520656E642C73746F702075706C6F616D
:1084200064000000602D0020A043030040490300C9
:108430007372635C6170705F626C655F73657276A6
:108440006963652E6300000025733A2564205A4550
:1084500052524F525F434845434B282573292066AB
:1084600061696C3A2564000075706C6F6164202549
:108470006420256420256400626C65206973206493
:108480006973636F6E6E65637465642C73746F706B
:108490002075706C6F616400626C6520756E656E2E
:1084A00061626C65206E6F746966792C73746F708D
:1084B0002075706C6F616400626C652073656E641A
:1084C000206572726F722C73746F702075706C6F90
:1084D0006164202578000000FEB54FF4827006F03C
:1084E00047FD002837D04FF4827006F04BFD6C48F2
:1084F00090F82E0018B16A4890F82F0058B3002069
:108500008DF8000066484068019065480189ADF823
:108510000810C06818B900206149087412E060486A
:10852000008B5F4948830846C06848600846008B56
:1085300008810020C860084690F82E0010B900207D
:1085400006F02CFD564801686846884700205449CB
:1085500081F82F0000BF524890F82E00002852D01A
:108560004FF4807006F004FD00284CD04FF480706A
:1085700006F008FD4A48408B494991F82D10884281
:1085800016DD4748408B464991F82D10401A444962
:1085900048830A4612890B465B8BD21A0B465B68EE
:1085A00003EB42000A4692F82D1006F0D9FC23E0B6
:1085B0003B48408B3A4991F82D1088420FD13848FA
:1085C000C06860B10120364981F82F00002048833F
:1085D0000A4692F82D10D06806F0C2FC0CE0304834
:1085E000408B2F4991F82D10884205D101202C494C
:1085F00081F82F00002048834FF4827006F0C2FCFF
:10860000042006F0CBFC4FF4887006F0B1FC70B18A
:108610004FF4887006F0B6FC00202149087402204F
:108620008DF80000084601686846884700BF4FF48F
:108630008A7006F09DFC38B14FF48A7006F0A2FCF7
:108640000020174908742AE01548456924E0B5FA66
:1086500085F64FF00040F0408543B00000F58C7483
:10866000204606F085FCB8B1204606F08BFC0120C0
:108670008DF80000A4F58C70C0F3C7008DF80400DD
:10868000A4F58C70012121EA90018DF805100448B1
:1086900001686846884700BF002DD8D100BFFEBDE5
:1086A000A859002010B500F055FA10BD2DE9F0478B
:1086B000074688461646C24607EB47011B4800EBB3
:1086C000C109D9F8140020B1012811D0022826D1FF
:1086D0001EE0484600F076FA0546B54201D2002475
:1086E00005E0344632465146484600F0B2FA18E0FA
:1086F000484600F067FA0546B54201D2284600E038
:108700003046044622465146484600F0A2FA08E0A8
:1087100032465146484600F063FA044601E0002420
:1087200000BF00BF2046BDE8F08700001879002098
:1087300010B50249024804F0DFFB10BDD8590020F3
:108740000030004010B503494FF040200AF018FEF9
:1087500010BD0000405A002010B50249024804F044
:10876000CBFB10BDFC5900200030024010B506F0D4
:1087700019FE10BD10B50949094A891AC908032212
:1087800042EA014007A106F023F9FFF743FC012864
:1087900001D108F075FBFFF7E3FA10BDF8530300B1
:1087A000605303006368616E676520746F206578AD
:1087B00074206D6F6465000010B50749074A891A77
:1087C000C908032242EA014005A106F001F9FFF7BA
:1087D0000DFB08F055FB10BDF85303006053030078
:1087E0006368616E676520746F206C6F63616C20D5
:1087F0006D6F64650000000010B5FFF711FCFFF716
:10880000DBFFFFF7B7FF10BD2DE9FC4180460D46A9
:10881000164600BF21480078002817D120A0234920
:10882000234A891AC9080322009042EA01408F2393
:1088300020A229A106F0F2F805F03EFF00BF0027B4
:1088400000BF002000F056FE00BF00BF00BF01AB1C
:1088500032462946264803F0EAFD044600BF002CB4
:1088600017D024A01149124A891AC908032200907E
:1088700042EA014092230FA217A106F0CFF805F0BB
:108880001BFF00BF002700BF002000F033FE00BF29
:1088900000BF00BF0198BDE8FC810000882D0020CA
:1088A0006D5F69735F6F70656E000000F8530300C1
:1088B000605303007372635C73616D706C655F6419
:1088C0006174615F6D616E616765725F7365727619
:1088D0006963652E6300000025733A2564205A41C0
:1088E000535345525428257329206661696C000052
:1088F000A453002066665F726573756C74203D3DFD
:108900002046525F4F4B0000014802490860704703
:108910000090D003282F002010B504F0F5FE40B1E0
:108920000020644908604FF08041C1F8100162499D
:10893000086004F003FF002855D0604800686049D3
:1089400008605E48001D0068091D08605B4808302B
:108950000068091D086059480C300068091D08604E
:10896000564810300068091D0860544814300068EB
:10897000091D0860514818300068514920310860CD
:108980004E481C300068091D08604C4820300068C3
:10899000091D0860494824300068091D08604748DF
:1089A00028300068091D086044482C300068091D03
:1089B00008604248303000684149403108603F4813
:1089C00034300068091D08603C4838300068091DD3
:1089D00008603A483C300068091D0860374840305C
:1089E0000068091D086004F05BFE40B1354800686E
:1089F00000F0010018B16FF0010032490860324800
:108A0000006840F470003049086000BF00BF00BF3C
:108A1000BFF34F8F00BF00BF00BF00BF00BF00BF4C
:108A2000BFF36F8F00BF00BF00BF00BF04F052FE56
:108A300020B12648006820492031086000BF234843
:108A4000001D006800F0010080B3012007F014FA57
:108A50001E48001D006820F001004FF01021C1F8F1
:108A60000C0207F013FA002007F006FA00BF00BF5F
:108A700000BF00BF00BFBFF34F8F00BF00BF00BFEC
:108A800011487C38006800F4E06011490843001D7B
:108A90000D497C39086000BF00BF00BFBFF34F8F96
:108AA00000BF00BF00BF00BF00BFFDE7FFE7FFF74B
:108AB0002BFF10BD0C0100403805004004040010DD
:108AC00020C500400004004088ED00E008120010BE
:108AD0000000FA0510B504220249034804F0CCFA5C
:108AE00010BD00007C5A00200080004010B5042218
:108AF0000249034804F0C0FA10BD0000885A002063
:108B00000090004010B502490868804710BD000081
:108B1000282E002008B500BF4FF480700B49405844
:108B200008B1012000E0002078B1094800688047C2
:108B300000BF00204FF48071044A88500846114657
:108B40004058009000BF00BF00BF08BD00000140BA
:108B50003C2E002010B5124C02202061606111A053
:108B6000A0611349E1614FF4007121620021A1620B
:108B70006162E1620BA0A0640E49E16410212165ED
:108B80000021A1656165E1650BA1E01DFEF771FCA7
:108B90000AA12046FEF76DFC2020A07110BD000048
:108BA000007900205465726D696E616C00000000F0
:108BB00078790020787B0020525454005345474771
:108BC0004552000010B501460A69CB689A4204D8A4
:108BD0008C68641EE41AA01801E0D41A601E10BD4F
:108BE0002DE9F0470446894617464FF0000AE5682C
:108BF00000BFD4F81080A84503D9A8EB0500461E95
:108C000004E0A5EB0800401CA1680E1AA068401BF8
:108C1000B04201D9304601E0A068401B0646BE4282
:108C200001D2304600E038460646616848193246AF
:108C30004946FEF7E6FBB244B144BF1B3544A06889
:108C4000A84200D10025E560002FD2D15046BDE8F2
:108C5000F0872DE9F047044689461546E668A06886
:108C6000871BAF4208D9616888192A464946FEF732
:108C7000C8FB7019E06010E0B84661688819424688
:108C80004946FEF7BEFBA5EB070809EB0701424684
:108C90006068FEF7B6FBC4F80C80BDE8F08702E020
:108CA00008C8121F08C1002AFAD170477047002077
:108CB00001E001C1121F002AFBD1704701462029A3
:108CC00008DA012088400A4A104008B101207047A4
:108CD0000020FCE7402909DAA1F12000012202FA74
:108CE00000F008B10120F2E70020F0E70120EEE7F4
:108CF000FC06FFBD00BFEFF31081084672B6704757
:108D00000246002104E0505C08B101207047491C74
:108D10000629F8D30020F9E7FEB5FF208D49C87079
:108D2000142088700F20487029200870C0078860C0
:108D30000320087300BF00231A46874805F06AF82D
:108D40000546002D19D085A09049914A891AC90875
:108D50000322CDE9000542EA014086238DA294A1B9
:108D600005F070FE05F0A8FC00BF00BF24B100BFF5
:108D7000204600F0BFFB00BF00BF00BF0021032062
:108D80000BF0DCFA00211D200BF0D8FA032005F0CF
:108D90003CFB1D2005F039FB8D488E490860002002
:108DA00048608D488D49086001204860884989489D
:108DB00000F010FA8849894800F00CFA40218548F3
:108DC00000F00AFA06467149714A891AC908032255
:108DD00042EA0140324682A105F004FE40217F486C
:108DE00000F0FAF906466949694A891AC908032256
:108DF00042EA0140324680A105F0F4FD002211460E
:108E0000744800F023FA0020029002AB412280490E
:108E100080A00AF043FABDF80800002837DD5B495E
:108E20005B4A891AC908032242EA01407BA105F086
:108E3000CFFD82227F497648FEF70EFB50B15349A1
:108E4000534A891AC908032242EA01407AA105F06F
:108E5000BFFD09E04D494E4A891AC908032242EA7A
:108E600001407EA105F0B4FD00240BE0684800EB52
:108E700044004278664810F81410564800F0F6F99D
:108E8000601C84B2BDF808008442EFDB0FE00024D0
:108E90000BE0684800EB44004278664810F8141074
:108EA0004C4800F0E3F9601C84B2412CF1D302ABD2
:108EB0004122714971A00AF0F1F9BDF808000028BB
:108EC00037DD3249324A891AC908032242EA014091
:108ED0006CA105F07DFD822270496748FEF7BCFA5F
:108EE00050B12A492A4A891AC908032242EA014094
:108EF0006BA105F06DFD09E02449254A891AC908CE
:108F0000032242EA01406FA105F062FD00240BE05C
:108F1000594800EB44004278574810F814102F4885
:108F200000F0A4F9601C84B2BDF808008442EFDBB5
:108F30000FE000240BE0594800EB4400427857480A
:108F400010F81410254800F091F9601C84B2412CEF
:108F5000F1D3FEBDE82C0020884303006E72665FEB
:108F60006472765F7370695F696E697428267370C6
:108F7000692C20267370695F636F6E6669672C20A9
:108F80004E554C4C2C204E554C4C2900F8530300A8
:108F9000605303007372635C616473313239335F11
:108FA00073696D706C655F7465737465722E6300B0
:108FB00025733A2564205A4552524F525F43484523
:108FC000434B28257329206661696C3A25640000AB
:108FD000FD910200B82B002025920200C02B00203A
:108FE000616473313239335F302072657669643A77
:108FF0002025640A00000000616473313239335F58
:10900000312072657669643A2025640A0000000008
:1090100050310020302E6366670000006C6F616481
:1090200020302E6366672066726F6D2066617466FD
:10903000730A0000C82B0020302E63666720697316
:1090400020646966666572656E742066726F6D2055
:1090500064656661756C740A00000000302E6366FA
:10906000672069732073616D652061732064656694
:1090700061756C740A000000D2310020312E6366E5
:10908000670000006C6F616420312E6366672066A4
:10909000726F6D2066617466730A00004A2C0020AE
:1090A000312E636667206973206469666665726540
:1090B0006E742066726F6D2064656661756C740AEB
:1090C00000000000312E6366672069732073616DB4
:1090D000652061732064656661756C740A00000028
:1090E000FEB505460C46002637260020009001906C
:1090F000029009236A463146284600F043F89DF85D
:10910000000000049DF8011000EB01209DF8021002
:10911000084420609DF8030000049DF8041000EB53
:1091200001209DF80510084460609DF806000004C9
:109130009DF8071000EB01209DF808100844A0607E
:10914000FEBD70B505460C46002020706070A07012
:10915000E07020716071A071072322461821284613
:1091600000F010F870BD000070B504460D460448CC
:109170000068401C024908600AF022F870BD000037
:10918000E02C00202DE9F04105460E4617461C460E
:10919000FF2C01DDFF2000E02046044646F0800859
:1091A0000A4880F800802146401CFEF743F9601C05
:1091B000C2B2074905482B68984722460449491C12
:1091C0003846FEF71EF9BDE8F08100002C2F002084
:1091D0002C300020016070477CB504460D4645F0F8
:1091E00080008DF8040000208DF8050002226946F9
:1091F00001A8236898479DF801007CBDF8B5044696
:109200000D461646032005F061F82B4632462146EE
:109210000348009604F042FE032005F0F6F8F8BD7E
:1092200088430300F8B504460D4616461D2005F098
:109230004DF82B46324621460348009604F02EFE98
:109240001D2005F0E2F8F8BD88430300F8B5044698
:109250000D46164605F07F008DF800008DF8016080
:1092600002220021684623689847F8BDFEB50646ED
:109270000C461546002002900295182C02DB1E2C8D
:1092800000DCFEBD302C02DB3F2C00DCF9E7402C7B
:1092900000D1F6E7502C00D1F3E702AB2A46214675
:1092A000304600F02FF89DF80800A8420FD09DF836
:1092B0000800CDE900500749074BC91AC908012326
:1092C00043EA0140234605A1726805F0BBFB00BFDD
:1092D000D7E70000F8530300605303006164735F35
:1092E0002564207772697465202578206661696C31
:1092F00065642C773A2578207265616462616B3A07
:1093000025780A002DE9F04105460E4617461C4611
:109310003A4631462846FFF799FF31462846FFF77F
:109320005BFF2070BDE8F0811CB5032004F0CEFF88
:109330001D2004F0CBFF00208DF8040001208DF8E3
:10934000050000200346022201A90090044804F011
:10935000A5FD032005F059F81D2005F056F81CBDA9
:109360008843030070B504460D4604F22740FFF71A
:10937000C7FC0646012D06D0022D0DD0032D11D0BD
:10938000042D19D113E0A07928B194F8240010B964
:109390000EB1012070BD00BFE07910B10EB1022006
:1093A000F8E700BF207A08B10320F3E700BF607A36
:1093B00008B10420EEE700BF0020EBE70146481C9F
:1093C000052290FBF2F302FB1300C0B27047014686
:1093D00091F82420012A01D1EE2000E01F207047DF
:1093E00010B501220221002001F0E8FB044600BF75
:1093F0001CB1072C01D0204610BD00BF072202215E
:10940000012001F0DBFB044600BF1CB1072C01D09A
:109410002046F1E700BF0A220021084601F0CEFBFA
:10942000044600BF1CB1072C01D02046E4E700BF72
:109430000020E1E710B572B600BF05F0B7FB00BF32
:1094400000BF05F039F90028FBD100BF00BF1E495D
:109450001E4A891AC908012242EA01401CA105F0EE
:10946000B7FA00BF1D48006800F0010000B100BE5F
:1094700000BF1549154A891AC908022242EA01406B
:1094800017A105F0A5FA00BF00BF00BF00BF00BFD5
:10949000BFF34F8F00BF00BF00BF1048E438006823
:1094A00000F4E06012490843001D0C49E4390860EB
:1094B00000BF00BF00BFBFF34F8F00BF00BF00BFA2
:1094C00000BF00BFFDE70000F85303006053030036
:1094D000466174616C206572726F7200F0ED00E09D
:1094E00053797374656D20726573657400000000B4
:1094F0000000FA053EB5044600200090019002905D
:1095000002946A46002144F20100FFF793FF3EBD3A
:1095100070B505460E462C46207820B96179207931
:1095200007F0F4FB1CE02078012807D10D48006803
:10953000401C0C490860FEF7B7FD11E020780928AF
:1095400002D107F0D3FB0BE02078032808D10648AE
:10955000007828B1042204F10801606807F044FB98
:1095600070BD00007C2D0020112D00202DE9F84356
:1095700007460C46904626480088844244DC4FF655
:10958000FF7500200090684600F01EFB00BF2148D8
:1095900090F800902048007804F05AF8484501D12E
:1095A000012000E0002030B91B480578007804F065
:1095B0004FF8194908709DF8000000F00BFB4FF6BA
:1095C000FF7085421ED01548006840F835808FB185
:1095D000002C0FDD124909680D4A128805FB0210A4
:1095E00022463946FDF70DFF0C48006800EBC50028
:1095F000848005E000200949096801EBC5018880E5
:10960000002600E0042600E009263046BDE8F88385
:10961000522E0020502E0020512E0020482E0020D7
:109620004C2E00202DE9F0411AE016480478164827
:1096300000681649098804FB01051548006800EB1D
:10964000C40086881248006850F8347031462846B5
:10965000B8470C48007803F0FBFF0A49087000BFC8
:1096600000BF002058B900BF0649087809490978A9
:10967000814201D1012100E000210029D5D0BDE8BF
:10968000F0810000502E00204C2E0020522E002091
:10969000482E0020512E002030B50346481C4FF6BE
:1096A000FF7505EAC004104600F003050DB9012559
:1096B00000E000250DB9072030BD084802601019F0
:1096C000074D28600020074D2870074D2870074877
:1096D0000380074801800020EEE70000482E0020AC
:1096E0004C2E0020512E0020502E0020522E002003
:1096F000542E00202DE9F04707460E4614461F4819
:1097000090F8220010B90820BDE8F0871B4890F8B7
:109710002200032801D01120F6E70CB90720F3E757
:109720000421164880F82210807AC0F3C00018B9CE
:1097300071021248016101E0104806610F48C760DC
:109740008482C48200218183012C01DD522000E04B
:1097500051208146094801220169484607F08AFEE6
:10976000054600BFA846B8F1000F04D000BF404630
:10977000FFF7C0FE00BF00BF0020C5E7645B00200C
:109780002DE9F04107460E4615462D4890F8220077
:1097900010B90820BDE8F081294890F8220003287C
:1097A00001D01120F6E70DB90720F3E70521244881
:1097B00080F82210807AC0F3C00018B971022048E6
:1097C000016101E01E4806611D48C7608582C582AF
:1097D00000218183012D12D101220169582007F057
:1097E00049FE044600BFA046B8F1000F04D000BFF8
:1097F0004046FFF77FFE00BF00BF0020CAE71048C9
:10980000807A00F00700012807D10D480122016984
:10981000592007F02FFE044605E001222946D720F3
:1098200007F028FE044600BFA046B8F1000F04D0A0
:1098300000BF4046FFF75EFE00BF00BF0020A9E763
:10984000645B0020064890F82200032805D00448F5
:1098500090F8220008B1012070470020FCE70000CA
:10986000645B0020044890F82200032802DB0248D1
:10987000001D70470020FCE7645B0020F0B587B056
:1098800004460E463A4890F8220010B1082007B06E
:10989000F0BD5EB1E078FF2808D06078FF2805D0E1
:1098A0002078FF2802D0A078FF2801D10720EEE71A
:1098B000E0782F4981F85800084690F85870002049
:1098C00000900346012211460190384604F067FCDF
:1098D00000BF00BF264991F8580004F0B0FD00BF5A
:1098E000244B0FCB03AD0FC5A0788DF80C0020786A
:1098F0008DF80D0060788DF80E0000231E4A03A934
:109900001E4804F087FA054600BF2F4627B100BF66
:109910003846FFF7EFFD00BF00BF15480660012184
:1099200080F82210807A20F0070111488172807A35
:1099300020F008010E488172002180F82310FF20DA
:109940000B4981F828000A2001F13803012228314F
:1099500000900A4804F0BBFA054600BF2F4627B125
:1099600000BF3846FFF7C6FD00BF00BF00208EE7EE
:10997000645B002078460300AD29030068460300BD
:109980007CB5144890F8220008B908207CBD114825
:1099900090F82200032801D01120F7E70E4C201D7B
:1099A00006F0CCF900BF0B4890F858400025002085
:1099B00000902B46024601460190204604F0EFFB42
:1099C00000BF0021034880F8231080F822100020F7
:1099D000DCE70000645B00206846030010B5044625
:1099E000022C0AD10C490D4A891AC908032242EAFD
:1099F00001400BA104F0ECFF01E0012010BD00BF0D
:109A00000549064A891AC908032242EA014010A101
:109A100004F0DEFF0120F1E7F85303006053030078
:109A2000506F776572206D616E6167656D656E74EC
:109A30002077616E747320746F2072657365742073
:109A4000746F20444655206D6F64652E0000000041
:109A5000506F776572206D616E6167656D656E74BC
:109A600020616C6C6F77656420746F20726573651C
:109A70007420746F20444655206D6F64652E00007D
:109A800010B5024802F0DEF910BD0000582E00208B
:109A900030B503460C460AB9072030BD19684FF0AF
:109AA000FF358D60CD604A61012C01D1012000E0BD
:109AB000002008610020F0E738B5134800680090E6
:109AC0000823A82211491248006803F051FE0446F9
:109AD0000CB1204638BD0F4A69460F4802F0B8F96C
:109AE00004460CB12046F5E701210B4802F056FA76
:109AF00001230A4A1946084802F076F9012008496C
:109B000008702046E6E7000088440300945A0020CD
:109B100078440300DD100300582E0020FFFF7F0073
:109B2000642E00202DE9F84306460D469046344643
:109B300000200090684600F047F84FF0FF33D4E96A
:109B4000021059405840014308D103F00FF9401961
:109B500041F10001C4E90201012700E000279DF85E
:109B6000000000F037F817B90020BDE8F883C4F80A
:109B70001880206900B125612146002009F0FEFA15
:109B8000F3E7F8B50446254600200090684600F04B
:109B90001BF84FF0FF33D5E90210594058400143FC
:109BA00001D1002604E04FF0FF31A960E9600126F1
:109BB0009DF8000000F00EF80EB90020F8BD29460F
:109BC000012009F0DBFAF9E710B50446204607F05A
:109BD000A1FB10BD70B5044625460E488068B0B1A3
:109BE000ADB9FFF787F806460A4800680A490860D9
:109BF000084840684FF0E021C1F804010020054901
:109C000088601EB900BF62B600BF00BF00BF00BFC2
:109C100070BD00004C5B002000E100E0F8B5054697
:109C20000C4617462088001DB84201D90C20F8BD0B
:109C3000684679DF064600BF304600B1F7E700BF4F
:109C40000320218868542088401C20801920218806
:109C500068542088401C208020884119BDF80000ED
:109C600009F005FE2188084420800020DFE700007D
:109C7000002113E00C480269012308E000BFD0680E
:109C80000079884201D1002303E0D0680268002AED
:109C9000F4D100BF0BB108467047491C0A29E9DB23
:109CA0004FF0FF30F8E70000E07800202DE9FC419C
:109CB000054688461646002437880020308095F8EF
:109CC0002D0058B13A463146404600F095FA044618
:109CD00000BF204608B1BDE8FC8100BFA87850B1A4
:109CE0003A4631464046FFF799FF044600BF2046FA
:109CF00000B1F0E700BFE87860B1E97848B23B46D0
:109D00003246414602F072FE044600BF204600B1D2
:109D1000E1E700BF686868B1696891F900003B46F7
:109D20003246414609F082FD044600BF204600B19C
:109D3000D1E700BF288900280EDD43460622022114
:109D400005F10800CDE9006709F03DFE044600BFBB
:109D5000204600B1BFE700BF288A00280EDD434639
:109D60000722032105F11000CDE9006709F02BFE61
:109D7000044600BF204600B1ADE700BF288B002895
:109D80000EDD43461522142105F11800CDE90067C8
:109D900009F019FE044600BF204600B19BE700BF52
:109DA000286A58B13B4632464146286A01F01DFAFE
:109DB000044600BF204600B18DE700BF686A58B175
:109DC0003B4632464146686A03F0E0FA044600BF6B
:109DD000204600B17FE700BF95F82C0000280BDD7E
:109DE0003B4632464146284608F002FB044600BF87
:109DF000204600B16FE700BF287858B13B46324695
:109E00004146284603F0C0FB044600BF204600B18F
:109E100061E700BF20465EE7F8B504460E461546EA
:109E2000002000902B466A463146204600F008F894
:109E300007460FB90020F8BDBDF800002044FAE73E
:109E4000F0B504460D461E4604B10AB90020F0BD27
:109E5000002103E0605C401C084481B2481CA84219
:109E600006DA10888842F5DC481C205CB042F1D14B
:109E7000A94201DB0020EAE7881C87B2605C10B1D0
:109E8000605C401E00E0002083B213B1F818A842C5
:109E900001DD0020DBE717801846D8E780F8301096
:109EA000704770B504460D4605B10CB90E2070BD63
:109EB00005F1780001F042F908B90720F7E7002022
:109EC000A0702C2205F17801201DFDF79AFA0020E0
:109ED00084F83000D5F8A4006063D5F8A800A0632A
:109EE0004FF6FF70A4F8240404F58260C4F820043F
:109EF000002140F22C40C4F82614A4F82A1401557D
:109F0000207810B9FF2084F8540004F15500C4F8FB
:109F100010042046FFF75BFA40F21441085304F2A4
:109F2000144204F155012846FFF7C0FE064600BF63
:109F3000304600B1BBE700BF04F231204FF483612B
:109F400008512046FFF743FAA4F81C044FF483603D
:109F5000015904F21C4205F13C00FFF7A7FE06463A
:109F600000BF304600B1A2E700BF012151200155DA
:109F7000208B81B248200153012084F83C0000214D
:109F80002164502001556169616404F13C020021A3
:109F900004F1540072DF064600BF304600B186E788
:109FA00000BF01202070304681E770B504460D46A1
:109FB0002E462088102804D0112807D026280FD13B
:109FC00009E02146304606F0B9F80AE0214630465D
:109FD00006F0B0FA05E02146304606F033FC00E01A
:109FE00000BF00BF70BD70B504460E46207808B9AA
:109FF000082070BDA670002140F22C40C4F8261441
:10A00000A4F82A140155A07910B1A078012809D02C
:10A01000E07910B1A078012804D0E07970B1A0787F
:10A0200002280BD1606B30B1012084F82D04082088
:10A03000616B884702E0002084F82D0431462046F9
:10A04000FFF790F9A070606BA0B1A078032802D050
:10A05000A07804280ED1607960B194F82E0448B934
:10A06000002084F83004012084F82F040720616B5D
:10A07000884702E0002084F82F04182104F13C00F6
:10A08000FDF7D8F9012084F83C0004F12C0006F01B
:10A0900068FC20B194F82C105120015502E00121F8
:10A0A0005120015594F8240060B104F1280006F015
:10A0B00058FC20B194F828105220015502E00121EB
:10A0C00052200155002150200155A078052824D2A6
:10A0D000DFE800F01F030A11180004F13C012046DC
:10A0E00008F0E9F9054619E004F13C01204608F0C2
:10A0F000CAF9054612E004F13C01204608F0EDF9EA
:10A1000005460BE004F13C01204608F014FA054630
:10A1100004E0002084F8310000E000BF00BFA07818
:10A1200098B104F13C0204F15400D4F8201472DF19
:10A1300005460DB128465CE794F8301094F85400B9
:10A1400073DF05460DB1284653E7606B18B194F8EC
:10A150003100616B884700204BE700002DE9F0419A
:10A16000044600BF14B90E20BDE8F08100BF1C22D8
:10A1700021461C48FDF745F91B481A49086020682C
:10A1800060B120687ADF05460DB12846ECE7164835
:10A1900021680A6802604968416005E012487BDF77
:10A1A00005460DB12846DFE7002617E006EB8600DE
:10A1B0000E4901EB800700BF4FF6FF70388000BFEB
:10A1C0000B4800EB461078600A4A0021381DFFF763
:10A1D0005FFC05460DB10320C6E7761C002EE5D0D6
:10A1E0000020C1E794580020182E0020805800203D
:10A1F00060580020353903002DE9FC4105460C4626
:10A20000174620880930B84202D90C20BDE8FC81ED
:10A2100068466DDF064600BF304600B1F6E700BF76
:10A220000820218868542088401C20801B20218819
:10A2300068542088401C208020882844DDF80110C4
:10A240000160BDF8051081802088801D20809DF868
:10A250000000400818B900202188685402E001205D
:10A26000218868542088401C20800020CEE7000010
:10A2700070B503F0C3FC044600BF204600B170BDBA
:10A2800000BF00BF084D28464FF0030C00DF00BFA1
:10A29000044600BF204600B1F1E700BF03F028FDEF
:10A2A00004462046EBE70000EC7F002010B5134980
:10A2B000134A891AC908042242EA014011A104F094
:10A2C00087FB4FF0FF3100203DDF044600BF2046F2
:10A2D00000B110BD00BFB12100203CDF044600BF2B
:10A2E000204600B1F5E700BF1348416901208847C7
:10A2F000022004F0B1FD0020EBE70000F85303005A
:10A3000060530300496E20626C655F6466755F622E
:10A310007574746F6E6C6573735F626F6F746C6F5E
:10A32000616465725F73746172745F66696E616C9B
:10A33000697A650D0A000000D07F002010B505483D
:10A340000068416900208847FFF7B0FF04462046B7
:10A3500010BD0000242F002070B504460D4600BF3C
:10A3600004B970BD00BF2088102806D0112808D07D
:10A3700051280AD0532810D10BE0204605F0D8FE12
:10A380000CE0204606F0C8F808E0204606F038FA4F
:10A3900004E0204606F010FA00E000BF00BF00BF56
:10A3A000DFE7000070B504460426207B012802D0B8
:10A3B000022822D109E001F08FFE05460DB90126E1
:10A3C00002E0112D00D1062619E0607B142801DC83
:10A3D000607B08B905260FE0627B04F10E0112488C
:10A3E000FDF70FF8607B1049091F8861084608F0E7
:10A3F000D1F8054605B9012601E0022600BF00BFDD
:10A40000012E0FD0207B314600F058F8054625B1CB
:10A41000064800684169032088470448006841698C
:10A420000220884770BD0000FC7F0020242F002000
:10A4300070B505460E4600BF1E48006820B11D4895
:10A44000406808B1012000E0002000B970BD00BFE5
:10A45000184800F10801426828469047044600BFAA
:10A46000082C24D07CB900201349096848760121C2
:10A47000022000F023F80446CCB10F48006841697F
:10A480000320884713E000200B490968487606211D
:10A49000022000F013F8044624B10748006841691F
:10A4A000032088470448006841690220884700BFAC
:10A4B000CCE70000EC7F0020242F0020F0B587B00F
:10A4C00004460D460327002001900290039004905B
:10A4D0000320069020208DF814008DF815408DF88B
:10A4E00016500E48C088ADF8040002208DF8060012
:10A4F0000020ADF8080006A8039005A804900749BD
:10A50000888801A9AEDF064626B9BDF818000328E1
:10A5100000D00C26304607B0F0BD0000D07F0020F0
:10A5200070B505460E462888102802D011282CD177
:10A5300015E01748006860B900F0BEFE044600BF91
:10A5400034B11448006818B1204612490968884798
:10A5500000BF0F480068401C0D49086016E00C4819
:10A560000068401E0A4908600846006860B9FEF7A6
:10A5700037FF044600BF34B10648006818B12046D2
:10A5800004490968884700BF00E000BF00BF70BDF4
:10A59000142E0020102E002070B504460D46208891
:10A5A000102806D0112808D012280ED0502810D11B
:10A5B00007E0204605F084FD0CE0204605F092FF00
:10A5C00008E0204606F05EF904E0204605F060FD54
:10A5D00000E000BF00BF70BD2DE9F04104460F460A
:10A5E000A6882088102806D0112817D019283DD019
:10A5F0001A2848D116E006F0EBFC304606F0C4FC01
:10A6000020B900BF0420FEF775FF06E0E07B0228BA
:10A6100003D131461D4803F015F934E0304606F009
:10A62000FBFC30E0207A0509042D01DB012000E06D
:10A6300000200246314615480C3002F0C8F9032DBF
:10A6400001DB012000E00020024631460F480830BF
:10A6500002F0BDF9022D01DB012000E000200246DE
:10A6600031460A48001D02F0B2F90CE0207A48B9E0
:10A67000607AC0F3C0052A46314604480C3002F027
:10A68000A6F900BF00BF00BFBDE8F081BC580020A4
:10A690002DE9BE4105460F46288821282BD006DC2F
:10A6A00010280BD0112817D013287DD154E03B2857
:10A6B0007BD052287BD05628F7D1C5E0A8887749AF
:10A6C00008800120764908707648006818B108466D
:10A6D000744909688847DDE04FF6FF706F490880CC
:10A6E00002206F4908706F48006818B108466D492C
:10A6F00009688847CEE06C496C4A891AC908042267
:10A7000042EA01406AA104F063F900200290A8889F
:10A7100002A98FDF044600BFA046B8F1000F19D090
:10A7200068A06149614A891AC9080322CDE9000875
:10A7300042EA0140462366A26DA104F083F903F0CA
:10A74000BBFF00BF00BF26B100BF3046FEF7D2FE00
:10A7500000BF00BF00BF9DE000231A4685214F487F
:10A7600000887FDF044600BFA046B8F1000F19D073
:10A7700054A04D494D4A891AC9080322CDE9000861
:10A7800042EA01404C2352A259A104F05BF903F0C4
:10A7900093FF00BF00BF26B100BF3046FEF7AAFE00
:10A7A00000BF00BF00BF75E073E028E0FFE70023B3
:10A7B0001A46194639480088B1DF044600BFA04652
:10A7C000B8F1000F19D03FA03749384A891AC90893
:10A7D0000322CDE9000842EA014052233CA244A1F1
:10A7E00004F030F903F068FF00BF00BF26B100BFDE
:10A7F0003046FEF77FFE00BF00BF00BF4AE0A888DA
:10A80000132176DF044600BFA046B8F1000F19D02F
:10A810002CA02549254A891AC9080322CDE9000838
:10A8200042EA014058232AA231A104F00BF903F0B7
:10A8300043FF00BF00BF26B100BF3046FEF75AFEFF
:10A8400000BF00BF00BF25E0A888132176DF0446C3
:10A8500000BFA046B8F1000F19D01AA01249134A40
:10A86000891AC9080322CDE9000842EA01405E23A3
:10A8700017A21FA104F0E6F803F01EFF00BF00BFFF
:10A8800026B100BF3046FEF735FE00BF00BF00BF57
:10A8900000E000BF00BFBDE8BE810000042F002023
:10A8A0000C2F0020082F0020F853030060530300F2
:10A8B00050485920757064617465207265717565C2
:10A8C00073742E006572725F636F64650000000030
:10A8D0002E2E5C6C69627A6E6F726469635C73724F
:10A8E000635C7A626C655F6D6F64756C652E630086
:10A8F00025733A2564205A4552524F525F434845CA
:10A90000434B28257329206661696C3A2564000051
:10A9100070B50446204608F0A4FF0546C5F3400084
:10A9200070BD70B50446204608F09BFF054605F053
:10A93000010070BD30B50246087A0B7833B1012BA7
:10A9400005D0022B05D0032B14D101E000BF00BFBE
:10A9500000BF4B7800EB4004084D2D6805EB8404E4
:10A960002372002300EB4004044D2D6805EB8404A2
:10A97000A37200E000BF00BF30BD0000142F002014
:10A9800001460A46906970472DE9FE4380460C4611
:10A9900091464546AE692869B0F5007F02D0062091
:10A9A000BDE8FE831648006808B11120F8E7C6F834
:10A9B0001890B460124805600027124905F1140090
:10A9C000FEF75CFF07464FB944B907F051FC0E484B
:10A9D000007808B9002000E00D20074677B100207C
:10A9E0000749086054B1094A07CA8DE80700B069F1
:10A9F000029069464046B268904700BF3846CFE7AC
:10AA0000982E00206D150300942E00203846030078
:10AA100030B503461D4611B101290ED105E014469B
:10AA20000CB100202070002030BD0AB90720FBE7E0
:10AA30001446281D20600020F6E700BF00BF062056
:10AA4000F2E700002DE9FE4307460D46B846D8F868
:10AA5000184000261B480068404502D01120BDE880
:10AA6000FE83FEF7EFFE08B11120F8E795E8070036
:10AA7000C4E90412E060AB889AB22968A868FEF7BE
:10AA800039FE064656B9A06840B907F0F1FB0E48FA
:10AA9000007808B9002000E00D200646A06870B1DB
:10AAA0006EB10A4A07CA8DE8070004F10C00019054
:10AAB000A069029069463846A268904700BF3046B8
:10AAC000CDE70000982E0020942E00205046030071
:10AAD000FEB506463746BD6913480068B84201D046
:10AAE0001120FEBDFEF7AEFE08B11120F9E7FEF71A
:10AAF00047FF044614B900200B490860A86880B1DC
:10AB00000A4A07CA8DE807000CB1012000E00020C6
:10AB10008DF80100A869029069463046AA689047FE
:10AB200000BF2046DDE70000982E002044460300C9
:10AB30002DE9FE4307460D46B846D8F818400026D2
:10AB40001B480068404502D01120BDE8FE83FEF797
:10AB500079FE08B11120F8E795E80700C4E904126E
:10AB6000E060AB889AB22968A868FEF709FE06463D
:10AB700056B9A06840B907F07BFB0E48007808B9C9
:10AB8000002000E00D200646A06870B16EB10A4AB0
:10AB900007CA8DE8070004F10C000190A06902903B
:10ABA00069463846A268904700BF3046CDE70000AE
:10ABB000982E0020942E00205C46030030B50346FA
:10ABC0000020042B23D2012A07D1012903D103F14C
:10ABD0000E04E4B200E00024224679B1012902D03B
:10ABE000022911D104E003EB43040A4D2A550DE07C
:10ABF00003EB4304074D2C44627007E003EB43046E
:10AC0000044D2C44A27001E0072000BF00E00720A3
:10AC100030BD0000505800202DE9FC4704460D4689
:10AC20001646A71C4FF001080020019001A8FEF76E
:10AC3000CBFF3048406828602E4840682D4989681D
:10AC4000411A2D480068401CA0EB010915E00121C4
:10AC50002A4802F014FE02F0CDFA824651462748F7
:10AC600002F00DFE2348406822498968411A2248B3
:10AC70000068401CA0EB010900BF4F45E7D8B8F1C0
:10AC8000000F30D00021009176B1009921F003012E
:10AC9000491C0091009921F00401091D00910099BF
:10ACA00064F3891100910DE0009921F00301891CE2
:10ACB0000091009921F00401091D0091009964F3AD
:10ACC0009F5100910B4949680B4A12681140094A8B
:10ACD0000C3202EB81000099016006494968394451
:10ACE0000C3A516000BF9DF80400FEF773FF404628
:10ACF000BDE8FC87E0680020B02E0020FC78002032
:10AD000070B504460D460A2D03D10D212046FFF7EC
:10AD1000F7FFA168481CA06020684554D4E90110E1
:10AD2000884202D3204603F000F970BD04488068D1
:10AD300003494968884201D1012070470020FCE79F
:10AD4000E068002070B504460D46032C06D1A9200A
:10AD50000349086000BF002004F07EF870BD0000C9
:10AD60002005004010B506490648FEF7EAF90649F5
:10AD70000648FEF7E6F90449014807F0BBFA10BDA2
:10AD8000CC2C0020B82B0020D32C0020C02B00207E
:10AD90004FF0FF31054A42F82010082804DBFF235A
:10ADA000A0F108015A325354704700004059002066
:10ADB0000146024850F82100704700004059002029
:10ADC0002DE9F04F03460C464FF0FF390AB1002041
:10ADD00000E0082084460AB1082000E00C208046EC
:10ADE000614624E0154850F82100401CF0B91D468A
:10ADF0000846274616464FFA80FBDFF840A00AF1C6
:10AE0000300A0AF805B0DFF834A04AF820704EB9CD
:10AE10004FFA85FBA0F1080ADFF820E00EF15A0E88
:10AE20000EF80AB000BF4FFA81F902E0491C414513
:10AE3000D8D300BF4846BDE8F08F0000405900203D
:10AE400001460148405670477059002070B590B0D7
:10AE500006460C461546A07818B901208DF80E005C
:10AE600002E0A0788DF80E002088ADF80C000020DC
:10AE70000290607C02A907F0BDFBA07C0DF10901E6
:10AE800007F0B8FBE07B08B1012000E000209DF84E
:10AE90000A1060F3C3018DF80A10207C08B101206C
:10AEA00000E000209DF80A1060F304118DF80A10EC
:10AEB000207B08B1012000E000209DF80A1060F31B
:10AEC00000018DF80A10207D08B1022000E0012069
:10AED0009DF80A1060F342018DF80A101C2109A8A0
:10AEE000FCF7A8FA607BC0F3001018B9607BC0F3D0
:10AEF0004010F8B100200090E07C0DF1010107F056
:10AF000079FB00BF9DF8000020F00F00401C8DF879
:10AF100000009DF8000020F0F00010308DF80000D7
:10AF200000BF9DF8020020F00600801C8DF8020092
:10AF3000CDF838D0607B8DF82400A07B8DF82500FB
:10AF4000142104A8FCF776FA03A8049002A805903F
:10AF5000A088ADF81C00A06820B1E088ADF818000A
:10AF6000A0680890A069002849D000200190A0693D
:10AF70000088ADF82C00A0694088ADF82E00A069CB
:10AF800040680A9001A80D90A169087B01A907F00B
:10AF900031FBA169487B0DF1050107F02BFBA0698E
:10AFA000807A08B1012000E000209DF8061060F3CF
:10AFB000C3018DF80610A069C07A08B1012000E035
:10AFC00000209DF8061060F304118DF80610A069AA
:10AFD000007A08B1012000E000209DF8061060F31F
:10AFE00000018DF80610A069807B08B1022000E006
:10AFF00001209DF8061060F342018DF80610E0690B
:10B0000008B1E0690C902B4604AA09A93046AADFD2
:10B0100010B070BD70B504460D460020E070401EB3
:10B02000E0622946204602F095FA08B1042070BD7E
:10B0300004F22E2002F0BFF84AF65521884201D0D2
:10B040000320F4E794F83000E92807D094F83000A2
:10B05000EB2817D13220005D902813D104F166004F
:10B0600002F09DF820F07F400749884201D100207E
:10B07000DDE704F1820002F092F80449884201D130
:10B080000020D4E70220D2E7464154004641543321
:10B09000024600E0521C107810B110788842F9D1B5
:10B0A0001078704770B505460DB9094C01E0084CA1
:10B0B000083409E0204602F046F8064606B904E0E6
:10B0C00028467168884700BFF4E700BF70BD0000E4
:10B0D0003459002010B504462CB9012006494870A7
:10B0E0000020FFF7DFFF012C04D101200249887006
:10B0F000FFF7D8FF10BD00002C5900200246891E22
:10B100005069801E884201D8002070475389906A98
:10B1100001FB0300F9E72DE9F047024613468C4690
:10B12000D3E90245DCE90267B6EB040877EB0500DA
:10B1300002D30120BDE8F0870020FBE701468878B4
:10B14000012805D191F82000012801D10020704785
:10B150000120FCE733B58BB00546002000900C9829
:10B1600078B100240BE021460CA802F05CFB28B16A
:10B17000009A501C009001A820F81240641C142C66
:10B18000F1D32C2269462846FCF73BF90DB030BDBF
:10B1900001460888062808DB0888B0F5486F06DDF8
:10B1A00008884FF6FF72904201D007207047488808
:10B1B000062808DB4888B0F5486F06DD48884FF65A
:10B1C000FF72904201D00720F0E708884FF6FF7227
:10B1D000904208D04888904205D008884A8890421A
:10B1E00001DD0720E2E70020E0E72DE9F041074616
:10B1F0000D46144698462088801D404502D90C20F3
:10B20000BDE8F0813846FFF7C3FF064600BF304671
:10B2100000B1F5E700BF0520218868542088401C54
:10B2200020801220218868542088401C2080228899
:10B230005119388808F01BFB218808442080228897
:10B240005119788808F013FB2188084420800020D9
:10B25000D6E710B5044600BF2046FEF74BF900BF05
:10B2600010BD0000F8B505460C46607A88B9207A12
:10B2700010B91048476801E00E4887682A463946E9
:10B280006068FEF74FFC064616B1304607F050F8EE
:10B290000EE0002020720748406948B101208DF877
:10B2A0000000ADF80250034841696846884700BF76
:10B2B000F8BD00009458002010B501220021084676
:10B2C000FFF77CFC044600BF1CB1072C01D02046D0
:10B2D00010BD00BF072202210120FFF76FFC0446CA
:10B2E00000BF1CB1072C01D02046F1E700BF0422AB
:10B2F00002210020FFF762FC044600BF1CB1072CAE
:10B3000001D02046E4E700BF0020E1E72DE9F04747
:10B3100082468946DAF80040B9F1000F06D1E768A5
:10B3200017B16069B84215D8012713E04946504665
:10B3300001F020FC0646022E02D20120BDE8F08773
:10B34000701C08B93046F9E76069B04201D930464F
:10B35000F4E74F463D4600BF6D1C6069A84204D823
:10B360000225BD4201D90020E8E72946504601F0F8
:10B3700001FC064606B909E0012E01D0701C08B98F
:10B380003046DBE7BD42E7D10020D7E700BF00BF72
:10B390004FF0FF322946204605F0CEFC8046B8F13A
:10B3A000000F08D1B9F1000F05D02A4649462046C2
:10B3B00005F0C2FC8046B8F1000F0DD1E560D4E97C
:10B3C0000410801E814202D22069401E2061207933
:10B3D00040F00100207107E0B8F1010F02D14FF0F9
:10B3E000FF3000E0012005462846A7E72DE9F35F7E
:10B3F0008A46DAF80090009800F120050B222021FF
:10B40000284602F01DF80020804607464FF0080B42
:10B4100000BF38467F1C19F80040202C00DC55E0A6
:10B420002F2C01D05C2C0AD100E07F1C19F80700FA
:10B430002F28FAD019F807005C28F6D046E02E2C09
:10B4400001D0D8450CD3BBF10B0F01D02E2C02D06C
:10B450000620BDE8FC9F4FF008084FF00B0BD8E723
:10B46000812C01DB9F2C03DDE02C1CDBFC2C1ADC87
:10B4700038467F1C19F80060402E01DB7E2E03DD6C
:10B48000802E05DBFC2E03DCABF10100404501D82A
:10B490000620DEE7404608F101082C54404608F13A
:10B4A00001082E5411E0214614A0FFF7F1FD08B168
:10B4B0000620CEE7612C04DB7A2C02DCA4F120000C
:10B4C000C4B2404608F101082C54A2E700BF09EBC2
:10B4D0000700CAF80000B8F1000F01D10620B8E754
:10B4E0002878E52801D105202870202C01DC0420D3
:10B4F00000E00020E8720020ABE70000222A2B2C9D
:10B500003A3B3C3D3E3F5B5D7C7F00002DE9FF41C7
:10B5100005460C4629492A4A891AC908042242EAE2
:10B5200001402B46224627A103F068FA0020029032
:10B530000390ADF80840ADF80A40009001906A46CB
:10B5400002A9284690DF0646002E32D0304604F08D
:10B5500017F8074619491A4A891AC908012242EA06
:10B5600001403B462A46234903F048FABDF8000053
:10B5700010B9BDF8020068B1BDF80230BDF8002076
:10B580000E490F4FC91BC908012747EA01401AA1FC
:10B5900003F034FABDF8040058B1BDF8042007499F
:10B5A000074BC91AC908012343EA0140224903F0A5
:10B5B00019FA304604B0BDE8F08100006053030082
:10B5C000605303005570646174696E672064617430
:10B5D00061206C656E67746820746F202575206F1C
:10B5E0006E20636F6E6E656374696F6E20307825B0
:10B5F000782E0000744A03005468652072657175E6
:10B6000065737465642054582F5258207061636BC1
:10B610006574206C656E67746820697320746F6F41
:10B62000206C6F6E672062792025752F2575206F3D
:10B6300063746574732E0000C04A030020BF704716
:10B640002DE9F04104460E46D4F800800021204642
:10B6500000F000F90546EDB9002700BF4046A1699A
:10B6600001F078FF054605B113E0E0690078E528B0
:10B6700002D0E069007820B9781C0746B04201D1B9
:10B6800007E000270121204600F040F80546002D84
:10B69000E4D000BF042D00D107252846BDE8F08185
:10B6A0002DE9F041044627680021204600F0D2F839
:10B6B000054615B12846BDE8F08100BF3846A169AE
:10B6C00001F048FF054605B11DE0E06906780EB9B6
:10B6D000042518E0E069C07A00F03F00A071E0693D
:10B6E000C07A00F0080038B90B2204F12001E069AB
:10B6F00001F087FE00B906E00021204600F006F8C0
:10B700000546002DDAD000BF2846D4E72DE9F047E2
:10B71000044689462568206900F12007A06910B118
:10B72000B7F5001F02D30420BDE8F087C7F3080077
:10B73000002868D1A069401CA061606938B92889D7
:10B74000B0EB571F5FD80020A0610420ECE76889A8
:10B75000401E00EA5720002855D12046616901F0BB
:10B7600009FA0646012E01D80220DDE7701C08B94F
:10B770000120D9E76869B0423FD8B9F1000F03D181
:10B780000020A0610420CFE720466169FFF7BEFDDD
:10B7900006460EB90720C7E7012E01D10220C3E7F4
:10B7A000701C08B90120BFE7284607F0FBFB08B171
:10B7B0000120B9E74FF40072002105F1300001F0DB
:10B7C0003FFE4FF0000831462846FFF797FCE8623D
:10B7D0000CE00120E870284607F0E4FB08B10120E6
:10B7E000A2E708F10108E86A401CE8626889404560
:10B7F000EFD8E86AA0EB0800E862666131462846A7
:10B80000FFF77CFCA0612761C7F3080105F1300058
:10B810000844E061002087E770B5044626680121EE
:10B820002046FFF70DFF054695B93046A16901F0A6
:10B8300091FE054665B920220021E06901F000FE75
:10B840000B2204F12001E06901F0EDFD0120F07010
:10B85000284670BD2DE9F04104460D462668B5F531
:10B86000001F02D205F01F0010B10220BDE8F081D8
:10B870002561A7681FB93078032800DB776A47B9CC
:10B880003089B0EB551F01D80220EFE7706AA06144
:10B890001CE070894FEA402811E03946204601F04B
:10B8A00069F90746781C08B90120DFE7022F02D3A7
:10B8B0007069B84201D80220D8E7A5EB08054545D4
:10B8C000EBD239463046FFF719FCA0616761A069E9
:10B8D00008B90220CAE7A06900EB5520A061C5F3B2
:10B8E000080106F130000844E0610020BEE70000D6
:10B8F0002DE9F04104463E480078844202DB0320F3
:10B90000BDE8F08104EB44003A49096851F8200091
:10B9100008B90320F4E704EB44003649096801EB59
:10B920008000407A00F0010038B904EB440031494E
:10B93000096801EB8000407AE2E704EB44002D49FE
:10B94000096801EB8000406838B92B4804EB4401DA
:10B95000284A126802EB81014860012004EB44018F
:10B96000244A126802EB8101887204EB44002149E9
:10B97000096851F82060214F306822463946036833
:10B9800030469847054600BF4DBB07E004EB440135
:10B99000184A126802EB81014868804704EB4400B2
:10B9A0001449096801EB8000807A0028EED104EB8D
:10B9B00044001049096801EB8000007A78B904EB73
:10B9C00044000C49096801EB8000407A20F0010036
:10B9D00004EB4401074A126802EB8101487204EB50
:10B9E00044000449096801EB8000407A88E70000C0
:10B9F000182F0020142F00203DB6020035A90200A8
:10BA0000F8B504460E4615462A480078844201DB04
:10BA10000420F8BD26B1012E1BD0022E45D12EE008
:10BA20000120009000BF04EB4401234A126852F841
:10BA300021006A46002102F0A2F8074617B1112F33
:10BA400000D003E09DF800000028ECD100BF0020EA
:10BA5000DFE704EB44001849096851F8200008B9F1
:10BA60000320D6E72F4604EB4401134A126852F82C
:10BA7000210002F07DF8006838600020C9E704EB7F
:10BA800044000D49096851F8200008B90320C0E7B7
:10BA90002F4604EB4401084A126852F8210002F0D4
:10BAA00067F8808838800020B3E700BF00BF01201E
:10BAB000AFE70000182F0020142F00202DE9FE4FC3
:10BAC0000446884691461E462F480078844200DA94
:10BAD00016B90420BDE8FE8F04EB44002B49096829
:10BAE00051F8200048B104EB44002849096801EBF3
:10BAF0008000407A00F0010008B10320EAE7CDF8A9
:10BB000000900196CDF80880012004EB44011F4A03
:10BB1000126802EB8101887204EB44001B4909683A
:10BB200051F820506F4628684169284688470068C8
:10BB30003968884201D8072004E0286839468268BD
:10BB4000284690478246BAF1000F1BD107E004EB6C
:10BB500044010E4A126802EB81014868804704EBF9
:10BB600044000A49096801EB8000807A0028EED180
:10BB700004EB44000549096801EB8000007A08B92C
:10BB80000020A7E70120A5E7182F0020142F002090
:10BB9000014607480078814201DB0120704701EB34
:10BBA0004100044A126802EB8000407AF6E7000088
:10BBB000182F0020142F002070B504463648007856
:10BBC000844201DB032070BD04EB44003349096863
:10BBD00051F8200008B90320F5E704EB44002F4991
:10BBE000096801EB8000407A00F0010038B104EBF5
:10BBF00044002A49096801EB8000407AE3E704EB3E
:10BC00004401264A126852F821000022114601F030
:10BC1000B6FF00BF04EB44002049096851F82060DA
:10BC20003068416830468847054600BF112DF1D085
:10BC30008DB907E004EB4401184A126802EB810158
:10BC40004868804704EB44001449096801EB800010
:10BC5000807A0028EED104EB44001049096801EB1A
:10BC60008000007A78B904EB44000C49096801EBC4
:10BC70008000407A40F0010004EB4401074A12685A
:10BC800002EB8101487204EB44000449096801EBAE
:10BC90008000407A97E70000182F0020142F002022
:10BCA0002DE9FE4F0446884691461E4635480078E9
:10BCB000844200DA16B90420BDE8FE8F04EB44008C
:10BCC0003149096851F8200048B104EB44002E497D
:10BCD000096801EB8000407A00F0010008B1032000
:10BCE000EAE704EB44002849096801EB8000407A48
:10BCF00000F0040008B10220DEE7CDF800900196C4
:10BD0000CDF80880012104EB44001F4A126802EBC1
:10BD10008000817204EB44001B49096851F82050EF
:10BD20006F46286841692846884700683968884214
:10BD300001D8072004E028683946C26828469047A1
:10BD40008246BAF1000F1BD107E004EB44010E4A12
:10BD5000126802EB81014868804704EB44000A49FD
:10BD6000096801EB8000807A0028EED104EB4400E2
:10BD70000549096801EB8000007A08B900209BE7BB
:10BD8000012099E7182F0020142F0020024A10608C
:10BD9000024B197070470000142F0020182F00204C
:10BDA00010B50021034801F08BFD044684F3100018
:10BDB00010BD0000FC78002070B505460C464FF41D
:10BDC000803000FA04F1284600F0AAF970BD70B581
:10BDD00005460C464FF4A07000EB840086B2314655
:10BDE000284600F0B7F970BD2DE9F04704460D462E
:10BDF00016461F464FF4803000FA05F84FF4A07045
:10BE000000EB85001FFA80F926F07F464146206846
:10BE100003F091F84146206803F07EF84946206817
:10BE200003F070F832462946206803F05BF841467B
:10BE3000206803F077F81FB14146206803F081F8CD
:10BE4000BDE8F08710B50446206803F050F810BD37
:10BE50002DE9F04704460D4617466079324941F80E
:10BE600020706079314901EBC000007968B1082683
:10BE70002F49304A891AC908022242EA01402EA1FC
:10BE800002F0A6FD3046BDE8F08729882068C0F89A
:10BE9000081500BF94F90420AB7810461946002815
:10BEA00008DB4FEA417C4FEA1C68DFF8B0C00CF8B1
:10BEB00000800BE04FEA417C4FEA1C69DFF8A0C02C
:10BEC00000F00F08A8F104080CF8089000BF00BFAC
:10BED00094F90410084600280DDB00BF00BF00F0F5
:10BEE0001F0301229A4043099B0003F1E023C3F89A
:10BEF000002100BF00BF00BF00BF012061790B4AD5
:10BF000002EBC10108716079114641F8304000260A
:10BF10000749084A891AC908032242EA014011A1C7
:10BF200002F056FD3046AEE77C2E0020802E002029
:10BF3000E05303006053030052544320696E73744E
:10BF4000616E636520616C726561647920696E69F8
:10BF50007469616C697A65642E00000000E400E099
:10BF600018ED00E05254433A20696E697469616CBF
:10BF7000697A65642E00000010B5014691F904004D
:10BF8000002807DB00F01F0301229A40024B4409FE
:10BF900043F8242000BF10BD00E200E070B5054664
:10BFA0000C4622460221284600F0C6F870BD10B5A6
:10BFB00004464FF48271204600F0CCF810BD10B555
:10BFC00004460021206802F0C7FF10BD10B50446EA
:10BFD0000421206802F0C0FF10BD2DE9F84F04468F
:10BFE0008846154699464FF4803000FA08FA4FF417
:10BFF000A07000EB88001FFA80FB25F07F455146BA
:10C00000204600F08DF8206802F071FF0646414698
:10C01000206802F061FF009032464146206802F03D
:10C0200061FF5946206802F06DFF3146009806F026
:10C03000E2FF012806D1102003F022FB59462068B8
:10C0400002F060FF206802F052FF064631462846A3
:10C0500006F0D1FF07465146206802F063FF012F2A
:10C060000FD16A1C4146206802F03CFF102003F00B
:10C0700007FB206802F03BFFB04225D00D20BDE851
:10C08000F88F2A464146206802F02CFF206802F013
:10C090002EFF0646681E314606F0ADFF07466FF0DC
:10C0A0007F40A0EB0900B84201D20D20E7E75FB95D
:10C0B0006A1C4146206802F015FF206802F017FF55
:10C0C000B04201D00D20DAE701225146204600F0AF
:10C0D00033F80020D3E7000010B510480068407E18
:10C0E00060B106210120FEF7E9F9044624B10B48AE
:10C0F0000068416903208847002010BD01200749DE
:10C100000968087601210846FEF7D8F904461CB1F3
:10C1100000200249096808762046EEE7242F002017
:10C1200070B504460D462946206802F0F5FE294602
:10C13000206802F000FF70BD70B504460E4615463B
:10C140003146206802F0EEFE1DB13146206802F053
:10C15000F8FE70BD70B505460C462868015929B136
:10C160002146286802F0CEFE012070BD0020FCE7C9
:10C1700038B50546284600F047FA04463CB96946FA
:10C18000284607F0B2FC04460CB90020286020467F
:10C1900038BD2DE9FC4707468846914600243E46B7
:10C1A00013E06B46012201A9484600F040F90098CF
:10C1B000012800D00DE09DF8045000BF06F8015B97
:10C1C000641C0A2D00D104E000BFA8F10100A042C8
:10C1D000E7DC00BF0020307014B13846BDE8FC87B2
:10C1E0000020FBE7F7B582B016460398019001A83E
:10C1F00000F098FD0546002D02DA0B2005B0F0BDD9
:10C200000E4850F825400CB100202070029810B163
:10C210000020029908700949029841F82500029807
:10C2200008B1012E01D00020E8E7002202A903A8EE
:10C2300000F03AFA07463846E0E700001C2F0020DD
:10C240002DE9F74F8EB0044616461CB9092011B0EF
:10C25000BDE8F08F06F03F06324602A90FA800F0B5
:10C2600023FA0546002D70D10298039003A80F9978
:10C2700000F0EDFB05462DB99DF8370000F0800079
:10C2800000B1062506F01C00002856D045B1042D4B
:10C2900003D103A8FFF7C0FA054646F008060AE0F6
:10C2A0009DF8120000F0110008B1072503E006F028
:10C2B000040000B10825002D51D106F00800002827
:10C2C0004DD000F0C7FC01900A9901F10E000199D0
:10C2D00006F05EFD0A9901F11600019906F058FD7D
:10C2E00020200A99C8720A99029800F045FF8146F9
:10C2F00000220A99029806F039FD0A9901F11C0002
:10C30000002106F045FD01200299C870B9F1000F27
:10C3100025D00298C06A01900022494603A804F083
:10C3200085FE0546DDB9DDE9011001F013F905468A
:10C33000A9F101000299C86011E085B99DF81200C9
:10C3400000F0100010B1042509E05DE006F00200E5
:10C3500028B19DF8120000F0010000B107254DB989
:10C3600006F0080008B146F040060298C06A206254
:10C370000A986062002D55D10A99029800F0FCFEDF
:10C38000A0600A9901F11C0000F009FFE06002982A
:10C3900020600298C088A080267400206074E0614C
:10C3A00060614FF40072002104F1280001F048F8A8
:10C3B00006F0200040B3E06830B3E06860610298A6
:10C3C00040894FEA402AA768D4F80C800CE039462F
:10C3D000204600F0CFFB0746012F00D80225781C2D
:10C3E00000B90125A8EB0A080DB9D045EFD8A7611F
:10C3F00055B9C8F3080038B139460298FEF77EFEF9
:10C40000B0F1000B01D102250CE00BEB5820E061EC
:10C41000E26902994878012304F12801FFF74EFBF5
:10C4200000B101250DB10020206028460FE72DE95D
:10C43000FF4F85B0044615469A46DDF818B0002037
:10C44000CAF8000003A9204607F04FFB04900498A7
:10C4500010B9607C049018B1049809B0BDE8F08F61
:10C46000207C00F0010008B90720F6E76169E06868
:10C47000401A01900198854200D9019DA0E0A08A50
:10C48000C0F3080000287ED103984089401E6169EE
:10C4900000EA5129B9F1000F17D1606910B9A068FD
:10C4A000029004E02046A16900F064FB029002982B
:10C4B000022802D202206074CFE70298401C10B913
:10C4C00001206074C9E70298A061A1690398FEF792
:10C4D00015FE064616B902206074BEE74E444FEAC8
:10C4E0005528B8F1000F29D009EB080003994989B4
:10C4F000884203D903984089A0EB0908039948783A
:10C50000434632465946FFF7D9FA10B1012060740C
:10C51000A3E7207C00F0800068B1E069801B404503
:10C5200009D2E169891B0BEB41204FF4007204F141
:10C53000280100F078FF4FEA482737E0E069B04271
:10C5400020D0207C00F0800078B1E269039948781F
:10C55000012304F12801FFF7A3FB10B1012060744F
:10C560007BE7207C00F07F0020740399487801234A
:10C57000324604F12801FFF7A1FA18B101206074D6
:10C580006BE700E0E661A08AC0F30800C0F5007721
:10C59000AF4200D92F46A08AC0F3080204F1280058
:10C5A00011183A46584600F03EFF00BFBB44606990
:10C5B00038446061DAF800003844CAF80000ED1B26
:10C5C000002D7FF45CAF002047E733B58BB00D46FC
:10C5D000002269460BA800F067F804468CB968464B
:10C5E0000B9900F034FA04465CB99DF82B0000F07A
:10C5F000800008B1062404E01DB12946684600F019
:10C600004BFB20460DB030BDF8B5044669462046C8
:10C6100007F06BFA0646002E44D1207C00F0400063
:10C6200000283FD0207C00F0800070B1E2690099C2
:10C630004878012304F12801FFF732FB08B10120FB
:10C64000F8BD207C00F07F00207400F003FB07465B
:10C65000216A009800F07EFF06461EBB656AE87AF4
:10C6600040F02000E8722946A268206806F07EFBB0
:10C6700005F11C00E16806F08BFB394605F1160058
:10C6800006F086FB002105F1120006F08DFB01206B
:10C690000099C870009806F03DFC0646207C00F02A
:10C6A000BF0020743046CBE72DE9F74F8AB0002158
:10C6B0000B9801600A9800F035FB08900898002854
:10C6C00003DA0B200DB0BDE8F08FB149089851F89E
:10C6D00020400CB90C20F5E70B9804600C9800F092
:10C6E000FE000C90207878B16078FFF751FA81460F
:10C6F00009F0010040B90C9820B109F0040008B11C
:10C700000A20DFE70020DDE7002020700898607035
:10C710006078FFF7EDF8814609F0010008B10320C9
:10C72000D0E70C9820B109F0040008B10A20C9E74D
:10C73000002739462046FEF76DFC0546022D01D044
:10C740002EDA2DE0002614E04FF4DF7000EB061126
:10C7500004F13000084409900998007920B1099843
:10C76000083000F01CFD00E0002002A941F826007E
:10C77000761C042EE8D3002606B1761E00BF02A860
:10C7800050F8267027B139462046FEF743FC00E0FA
:10C7900003200546022D03DB701C06460428EED359
:10C7A000042D01D101208DE7022D01DB0D2089E749
:10C7B00004F13B0000F0FFFCB0F5007F01D00D203C
:10C7C00080E704F1460000F0F6FC8046B8F1000F67
:10C7D00004D104F1540000F0E2FC8046C4F8188053
:10C7E0004020005DA070A078012804D0A078022825
:10C7F00001D00D2066E7A07808FB00F83D20005D21
:10C800006081608918B16089411E084008B10D201F
:10C8100058E704F1410000F0CEFC2081207A00F0BE
:10C820000F0008B10D204DE704F1430000F0C3FCF8
:10C830008246BAF1000F04D104F1500000F0AFFCC1
:10C84000824604F13E0000F0B6FC0190019808B960
:10C850000D2037E701984044218900EB1110079023
:10C860000798824501D20D202CE70798AAEB00001B
:10C870006189B0FBF1FBBBF1000F01D10D2021E775
:10C8800003254FF6F570834500D8022540F6F57074
:10C89000834500D801250BF102006061E761019832
:10C8A0003844206207983844A062032D13D104F164
:10C8B0005A0000F080FC08B10D2003E7208908B180
:10C8C0000D20FFE604F15C0000F069FC6062606925
:10C8D0008000069014E0208908B90D20F2E6206A55
:10C8E00040446062022D02D16069400007E0207D73
:10C8F00000F00100616901EB410100EB510006907D
:10C90000A169069800F2FF10B1EB502F01D20D2063
:10C91000D8E64FF0FF302061E06080202071032DC9
:10C920002CD104F1600000F046FC012826D1791CCE
:10C93000204600F00FFE08BB0020207104F22E20DC
:10C9400000F039FC4AF65521884217D104F1300035
:10C9500000F025FC0F49884210D104F5057000F065
:10C960001EFC0D49884209D104F5067000F017FC41
:10C97000206104F5077000F012FCE06025700748A4
:10C980000088401C80B205490880E080002099E6BC
:10C990001C2F00205252614172724161202F0020F1
:10C9A00010B50446E07FFF2808D0A07F18B1E07FD3
:10C9B00001F099FC02E0E07F01F034FD0020607797
:10C9C000207204F10800D4E90021904710BD70B531
:10C9D00005460E46144624B13146284600F032FF83
:10C9E00003E03146284600F00FFF70BD30B5044625
:10C9F0001088C01C984201D90C2030BD0220158837
:10CA000048551088401C1080012015884855108812
:10CA1000401C108015884C551088401C1080002048
:10CA2000EBE770B504460D4640F21442115B01225B
:10CA3000D4F81004FDF7F0F9064606B1357004F19C
:10CA40003C0204F5826104F1540072DF70BD2DE9EF
:10CA5000F34104462646D6F8008002E00198401CC7
:10CA60000190019800782F28F8D0019800785C2870
:10CA7000F4D00020B06001980078202808D28021EE
:10CA80002B20015500212046FEF7E4FE05462CE050
:10CA900000BF01A92046FEF7A9FC054605B123E029
:10CAA0002046FEF7FDFD05462B20075D3DB1042D18
:10CAB00004D100BF07F0040000B9052514E007F019
:10CAC000040000B110E0B07900F0100008B90525AD
:10CAD0000AE0208AC0F3080208F13000111840462D
:10CAE00000F04AFBB060D4E700BF2846BDE8FC81F7
:10CAF00070B505460C4660880C490988884214D1F7
:10CB0000208840F6772188420FD1A088C01E0849AE
:10CB100008802B886A880749074E891BC9080426A4
:10CB200046EA014005A101F069FF70BD042F002015
:10CB3000062F0020F8530300605303004154542093
:10CB40004D54552065786368616E676520636F6D2D
:10CB5000706C657465642E2063656E7472616C2000
:10CB60002564207065726970686572616C20256447
:10CB7000000000002DE9F04781460C46D9F800502E
:10CB8000022C02D36869A04202D84FF001085EE08F
:10CB90004FF0FF382878012804D002282CD0032831
:10CBA00051D13CE0264606EB5606286A00EB56219A
:10CBB000284600F0CFFC00B148E03046761CC0F3B8
:10CBC000080105F13000475C286A00EB5621284631
:10CBD00000F0C0FC00B139E0C6F3080105F13000F7
:10CBE000405C47EA002704F0010008B1380901E081
:10CBF000C7F30B00804629E0286A00EB1421284681
:10CC000000F0A8FC00B121E040F2FF1101EA44026B
:10CC100005F13001501800F0CEFA804616E0286A7F
:10CC200000EBD411284600F095FC00B10EE040F274
:10CC3000FF1101EA840205F13001501800F0AFFA4B
:10CC400020F0704802E04FF0010800BF00BF4046EE
:10CC5000BDE8F0871CB51F201D2117231A46CDE91A
:10CC6000001001214FF4FD6000F001F81CBDF0B58B
:10CC70000446DDE905560020A4F2BC7740EA47608F
:10CC80004F1C40EA475040EA024040EAC32040EAD5
:10CC9000451040EA5600F0BD2DE9F04705460C4628
:10CCA00000206072A86908B9BDE8F0870026374601
:10CCB0001CE03046761CEA6912F80090B9F1200FAA
:10CCC00000D113E0B9F1050F01D14FF0E509092EAC
:10CCD00005D12E2238467F1C04F109010A5438463A
:10CCE0007F1C04F1090101F8009000BF0B2EE0D376
:10CCF000002104F10900C155E869C07A2072E96990
:10CD000001F11C0000F04BFA2060E96901F1160006
:10CD100000F045FA8046A4F806804FEA1840A0804B
:10CD200000BFC1E770B502464FF0FF301568DDB1B6
:10CD3000116800E0491C0D78212D02D30D783A2DA1
:10CD4000F8D10D783A2D0ED1146814F8015BA5F1D5
:10CD500030030A2B06D28C4204D11BB918464D1C55
:10CD60002946156070BD002000BFFBE770B50B4879
:10CD7000FFF768F80A4B0CCB841843F1000509490A
:10CD800003C9201A75EB010004D24FF08073E41838
:10CD900045F100052046294670BD0000582E0020B0
:10CDA000682E0020702E002038B51F2000906846A5
:10CDB00001F0A6FA044600BFD4F810050099C84057
:10CDC00000F0010038BD0000024600210CE001EB3C
:10CDD0008100074B33F82000904204D101EB810021
:10CDE00003EB80007047491C0029F0D00020F9E7D0
:10CDF000805800202DE9FC5F83460E4691461F4671
:10CE0000DDE90C45002E01DA704200E03046824632
:10CE10004FF0010803E09AFBF9FA08F10108CA454E
:10CE2000F9DA474500D9B84634B1002E03DB05F0E6
:10CE30000400042800D1641E05F0020000B167B1AF
:10CE400005F0010048B944B104E0641E20215846B1
:10CE5000FDF756FF0CB1A045F7D3002E05DA764258
:10CE60002D215846FDF74CFF07E005F0040004288B
:10CE700003D12B215846FDF743FF05F0020002289D
:10CE80000DD105F0010050B94FB944B104E0641E62
:10CE900030215846FDF734FF0CB1A045F7D33B468F
:10CEA0004A4631465846CDE9004506F0E7FCBDE864
:10CEB000FC9F30B5024600201378C3F38003D3B142
:10CEC000137803F00303012B02D0022B10D107E0EB
:10CED0001388C3F383139B1C0C6823440B6008E086
:10CEE0000B680225146805EB945423440B6000E0A2
:10CEF00000BF00BF012030BD70B505460C464FF4A1
:10CF00008C71284602F008FB38B14FF48C7128462A
:10CF100002F009FB2046FFF743FD70BD70B50546E2
:10CF20000C464FF48871284601F067FF68B14FF452
:10CF30008871284601F068FF607900F0040020B194
:10CF4000206810B10120216888474FF48A71284673
:10CF500001F053FF68B14FF48A71284601F054FF85
:10CF6000607900F0080020B1206810B1022021682B
:10CF700088474FF48E71284601F03FFF68B14FF4A7
:10CF80008E71284601F040FF607900F0100020B952
:10CF9000206810B10020216888474FF4827128462C
:10CFA00001F02BFF58B14FF48271284601F02CFF9D
:10CFB00001202071206810B103202168884770BDCE
:10CFC0002DE9F04781460C4616464FF480374FF462
:10CFD000A078002520E03946484601F0B5FFA8B109
:10CFE0004146484601F0A1FF80B13946484601F06C
:10CFF00090FF3946484601F09BFF4146484601F004
:10D000007AFFE8B21B4A52F8241088477F0008F1E3
:10D0100004001FFA80F86D1CB542DCD34FF4807811
:10D020000121484601F090FF68B14146484601F0B1
:10D030007CFF40B14146484601F05DFF0D4850F885
:10D040002410042088474FF482780221484601F0DA
:10D050007BFF68B14146484601F067FF40B1414659
:10D06000484601F048FF034850F82410052088473F
:10D07000BDE8F087402E00202DE9F04704460E461B
:10D080009046002722E0384602F088FA05463846E6
:10D0900002F08BFA81462046294642580AB1012205
:10D0A00000E0002282B14846D4F80413014009B1DF
:10D0B000012100E0002139B12946204602F07AFA28
:10D0C0002846D6E900219047781CC7B24745DADBED
:10D0D000BDE8F0872DE9F0410446A08800EB020C82
:10D0E000B4F80480904501DD104600E0A088A8EB6C
:10D0F0000005E088C618B4F80680984501DD18469A
:10D1000000E0E088A8EB00074888B4F800804045BC
:10D1100004DB4888B4F80280404502DD0020BDE809
:10D12000F0818888A84202D38888604501D9002010
:10D13000F5E7C888B84202D3C888B04201D90020B8
:10D14000EDE70120EBE70146086808B102680A60D4
:10D15000704710B5044622460221002001F09CF8D9
:10D16000002105E054F8210008B1012010BD491C40
:10D170000229F7D30020F9E770B505460C4604F103
:10D180001A0000F018F806462878032805D104F1A3
:10D19000140000F010F846EA0046304670BD014623
:10D1A000C8788A7842EA00204A7842EA00200A7861
:10D1B00042EA00207047014648780A7842EA002097
:10D1C0007047000010B502F021FA20B902F042FACF
:10D1D00000200149887010BD2C590020F7210180E2
:10D1E000172141800021017141711B218171C171A1
:10D1F000704770472DE9FF4100272E4800F038FBAB
:10D200002C48001F00F034FB2B48806803902B480B
:10D2100005680398284028490C3101EB800800BFBD
:10D2200003A94046FFF745FE30B103982840224944
:10D230000C3101EB800800E000E0F1E700BF0024C2
:10D240000AE00398411C284003911B490C3151F816
:10D2500020004DF82400641C022CF2D3009800F04A
:10D26000030001280DD0022814D1BDF80670042156
:10D27000009801EB9050401E039901EB9000039041
:10D2800009E0BDF806700098C0F3831003990844C4
:10D29000039000E000BF00BF0648001F00F0E1FA65
:10D2A000064616B1044903988860384604B0BDE8C4
:10D2B000F0810000F8780020E0680020B02E002007
:10D2C00000BF1A4A64213820FCF7E6F9044600BF83
:10D2D000254625B100BF2846FCF70CF900BF00BF6A
:10D2E00000BF06F0A7FF1249124A891AC908032293
:10D2F00042EA014010A213A101F074FB16490A682A
:10D300000B490C4BC91AC908032343EA014013A176
:10D3100001F068FB15A01B4908601B4848600846DF
:10D3200006F01EFCFAF788FB05F0C4F97C350020F6
:10D33000F85303006053030031323A32383A323145
:10D3400000000000636F6D70696C652074696D6525
:10D35000203A2573000000008010001043555354FC
:10D360004F4D4552203A256400000000414453319E
:10D370003239335F5445535445525F3343485F5607
:10D3800032000000FC2C00209DFE02002DE9F0413F
:10D3900005460E4614469846A888871C2088801C9F
:10D3A0003844404502D90C20BDE8F081FE2F01D958
:10D3B0000C20F9E7781C218870542088401C2080BC
:10D3C000FF20218870542088401C208022889119D9
:10D3D000288806F04CFA218808442080A888002874
:10D3E0000DDDA86808B90720DEE7AA882388981908
:10D3F000A968FAF706F82088A98808442080002048
:10D40000D2E7F0B503461D460C46002000BF15F8D4
:10D41000017B14F801CBA7EB0C00561E321E01D085
:10D420000028F4D0F0BD30B503460C463AB100BF39
:10D4300014F8015B03F8015B551E2A1EF8D130BDBC
:10D4400010B5034600BF03F8011B541E221EFAD17B
:10D4500010BD2DE9FF4F87B0044691461E46A246F7
:10D460002546BAF806009AF805104843001F0690B2
:10D47000BAF806B0301DB0FBFBF00590301DB0FBD4
:10D48000FBF10BFB11000490D9F8000081190698FC
:10D49000814202D90698801B01E0D9F800000746B6
:10D4A000C9F8007003E02D680598401E05900598A6
:10D4B0000028F8D103900498ABEB0008B84501D9D7
:10D4C000384600E04046804623E003990898084427
:10D4D0000290281D049908440190149828B14246EE
:10D4E000DDE90110F9F78DFF04E04246DDE90101B5
:10D4F000F9F787FF002004902D68A7EB0807039831
:10D5000040440390BB4501D9384600E05846804668
:10D5100000BF002FD9D10BB0BDE8F08F70B5034626
:10D520000C469CB101F026FB054600220AE00848A3
:10D5300000EB820108881E68B04202D11A60002008
:10D5400070BD521CAA42F2D30520F9E70020F7E78C
:10D550000000000070B504460D460026E06AA842AF
:10D5600010D0204605F01EFD06465EB96078012306
:10D570002A4604F13001FEF7A1FA10B14FF0FF3551
:10D580000126E562304670BD2DE9F84F05460F468D
:10D59000144698462878012804D1687810B90720E5
:10D5A000BDE8F88F2088801C404508D828780128DD
:10D5B00007D12088801C69780844404501D90C2097
:10D5C000EEE72088A8EB0000801E86B20096218836
:10D5D000891CC81969467DDF814600BF484600B1F5
:10D5E000DEE700BF2878022804D06878BDF8001074
:10D5F000884206DBBDF80000B04202DC4FF0090AA9
:10D600000BE04FF0080A2878012805D16878B0426D
:10D6100002DC6878009000E00096BDF80000FE286B
:10D6200001D90C20BCE7BDF80000401C21887854CB
:10D630002088401C2080208807F800A02088401CFB
:10D6400020802088BDF80010084420800020A7E733
:10D65000014604480088814201DA481C00E00020AD
:10D66000C0B27047542E0020FEB504460D4600207F
:10D6700001900290CDF808D00220ADF804000020FF
:10D68000ADF8060001AA29462046ADDF06462EB9B0
:10D690000298FDF746F908B10120FEBD0020FCE725
:10D6A0000B4802684FF08050D0F834110D2A0DD18C
:10D6B00021B1012904D0022906D103E001207047DD
:10D6C0000120FCE70120FAE70120F8E70020F6E757
:10D6D000300100100B4802684FF08050D0F8341130
:10D6E0000D2A0DD121B1012904D0022906D103E070
:10D6F000002070470020FCE70120FAE70120F8E74E
:10D700000020F6E7300100100B4802684FF080500F
:10D71000D0F834110D2A0DD121B1012904D00229EC
:10D7200006D103E0012070470120FCE70120FAE761
:10D730000120F8E70020F6E7300100100B480268EE
:10D740004FF08050D0F834110D2A0DD121B10129AC
:10D7500004D0022906D103E0012070470120FCE734
:10D760000120FAE70120F8E70020F6E73001001079
:10D7700010B5044609B90E2010BD92FBF3F003FB6F
:10D78000102008B10920F7E7216000206060A06048
:10D79000A281E38100BFEFE770B504460D4629463C
:10D7A0002046F9F739FD18B12A882168881870BD1C
:10D7B0000020FCE770B505460C4620886188884249
:10D7C00004D12846F9F76AFD012070BD0020FCE76E
:10D7D00070B504460D4629462046F9F742FD18B1BA
:10D7E0006A882168881870BD0020FCE770B505467E
:10D7F0000C4620886188884204D12846F9F728FD24
:10D80000012070BD0020FCE770B505460C4604F011
:10D810001F0301229A40D143620905EB820000F008
:10D8200039F8064670BD10B50246480952F8200086
:10D8300001F01F040123A340184008B1012010BDCE
:10D840000020FCE770B505460C4604F01F030122DA
:10D8500002FA03F1620905EB820000F03CF806468B
:10D8600070BD10B504460021204600F01EF810BD22
:10D8700010B504460121204600F02DF810BDF8B582
:10D8800004460D466A4629462046F9F75CFD0646E1
:10D890000098F8BDF8B504460D466A46294620466C
:10D8A000F9F737FD06460098F8BDF8B504460D4671
:10D8B0006A4629462046F9F72CFD06463046F8BD53
:10D8C000F8B504460D466A4629462046F9F708FD94
:10D8D00006463046F8BDF8B504460D466A46294668
:10D8E0002046F9F709FD06460098F8BDF8B504464C
:10D8F0000D466A4629462046F9F732FD064600984D
:10D90000F8BDF8B504460026002000906846FCF7F4
:10D910005BF9206800686168884215D92068006852
:10D92000401E226810600178204600F033F8064659
:10D93000207A21680978401AC5B220680079A84287
:10D9400001DA2068057100BF9DF80000FCF742F97C
:10D950003046F8BD0246D068081A138AB0FBF3F0CF
:10D96000C0B27047F8B504460D462E460020009020
:10D970006846FCF729F931462046FFF7EBFF21689E
:10D980000A68511C2368196010709DF80000FCF7AC
:10D9900021F9F8BD0246138AD06801FB03007047E5
:10D9A00010B5014600BF09B90E2010BD00BF087AAE
:10D9B0000B79C01AC2B2D1E90030186005E00868DE
:10D9C0000368581C0C6820601A70101EA2F1010335
:10D9D000DAB2F4D10B68187100BFE6E730B5024641
:10D9E0000B46D40802F00702012090401D5D28403C
:10D9F00030BD024600BF0AB90E20704700BF17298C
:10DA000001DBF72901DD0720F7E711800020F4E7AB
:10DA100070B504460E4600BF0CB90E2070BD00BFA5
:10DA20002661F720208060801B202071002505E002
:10DA3000A11D01EBC500FFF7D1FB6D1C002DF7D038
:10DA40000020EBE72DE9F047064688464546B488B6
:10DA5000012C01DBBDE8F0873088242820D006DCCB
:10DA6000102809D011280CD0232823D11DE03A28F2
:10DA70000CD055281ED10EE03146284602F066FB38
:10DA800019E03146284602F06EFD14E03146284682
:10DA900002F032FE0FE03146284602F06FFD0AE048
:10DAA0003146284602F02EFC05E03146284602F0B9
:10DAB000D1FC00E000BF00BFA81D00EBC40000794E
:10DAC00070B3A81D30F834102046A5DF0746C7B94B
:10DAD0000021A81D00EBC40001710121A81D00EB6D
:10DAE000C4004171A91D31F834201149114BC91AE4
:10DAF000C908042343EA014023460F4900F07EFF92
:10DB000012E0112F10D0384601F03AFD8146084945
:10DB1000084A891AC908012242EA01404A4600E03F
:10DB200003E006A100F05EFF00BF00BF92E7000027
:10DB300060530300605303002C4A030073645F6268
:10DB40006C655F67617474635F65786368616E6755
:10DB5000655F6D74755F72657175657374282920D2
:10DB600072657475726E65642025732E0000000066
:10DB700010B50446206841692046884710BD70B53D
:10DB800004460D461646206832462946036920465B
:10DB9000984770BD01464FF08040405808B10120C1
:10DBA00070470020FCE708B500224FF080410A5082
:10DBB0000958009100BF08BD014908607047000086
:10DBC00008030040012291070A5070472DE9F041F7
:10DBD00004460CB9BDE8F08100BF4FF47A7505B971
:10DBE00004E0054FAE013046B84700BF601E041E7A
:10DBF000F3D100BFEEE70000D143030070B540F65B
:10DC0000F8700068401C18B94FF01020406902E01D
:10DC100040F6F87000680546681C00281CD01449BE
:10DC2000144A891AC908032242EA01402A4612A16D
:10DC300000F0D8FE284613DF04465CB10C490D4ABB
:10DC4000891AC908012242EA014016A100F0C0FE6B
:10DC5000204670BD0020FCE70549064A891AC9081C
:10DC6000012242EA01401CA100F0B2FE0420F0E7CC
:10DC7000F85303006053030053657474696E6720A2
:10DC8000766563746F72207461626C6520746F20B6
:10DC9000626F6F746C6F616465723A203078253002
:10DCA000387800004661696C65642072756E6E6933
:10DCB0006E672073645F736F66746465766963650D
:10DCC0005F766563746F725F7461626C655F6261D9
:10DCD00073655F73657400004E6F20626F6F746CC4
:10DCE0006F616465722077617320666F756E640082
:10DCF00010B50E490E4A891AC908032242EA0140AA
:10DD00000C4A0DA100F06EFE0A4813DF04465CB118
:10DD10000649074A891AC908012242EA014011A1AD
:10DD200000F056FE204610BD0020FCE7F85303002B
:10DD3000605303000070020053657474696E6720BD
:10DD4000766563746F72207461626C6520746F20F5
:10DD50006D61696E206170703A20307825303878B6
:10DD6000000000004661696C65642072756E6E6922
:10DD70006E672073645F736F66746465766963654C
:10DD80005F766563746F725F7461626C655F626118
:10DD900073655F736574000010B500240F48007848
:10DDA00008B1852411E000200C49886048600861B2
:10DDB000C8600B4801F03EFC044601F00BFB08B9BB
:10DDC00001F02EFC01200549087001F01FFC10B184
:10DDD000012002498870204610BD00002C59002007
:10DDE000D5B0020008B5002000906846FBF7ECFEB5
:10DDF0000748C068401E0649C8600846C06808B9A0
:10DE0000FFF7E0F99DF80000FBF7E4FE08BD000015
:10DE10002C5900202DE9FF4705460C46164698462A
:10DE20002F781A4840F82760194840F827804FF0AB
:10DE30000009184B0FCB8DE80F0020788DF80000FB
:10DE400060788DF80100A0788DF80200E0788DF8F8
:10DE5000030020798DF8050060798DF80600A06830
:10DE60000290207B8DF80C00607B8DF80D000EB1C8
:10DE7000094800E0002002463B466946281D01F0A3
:10DE800077FE8146484604B0BDE8F087205A00205E
:10DE9000305A0020684403001D2C03002DE9FF4781
:10DEA00004460D4616461F46DDF830804FF0000947
:10DEB000009501960297CDF80C8000226946201D3E
:10DEC00001F0A4FF8146484604B0BDE8F0872DE983
:10DED000FF4704460D4616461F46DDF830804FF0DA
:10DEE0000009009501960297CDF80C800022694642
:10DEF000201D01F08BFF8146484604B0BDE8F08745
:10DF00000FB438B50446059810B938BC5DF814FB59
:10DF10000020009006A800906A462046059900F06F
:10DF200012F80020009000BFEFE770B50446A0682B
:10DF300000B970BDD4E90403A268216898470020A5
:10DF4000A06000BFF5E72DE9FC5F82460D46144650
:10DF50000DB9BDE8FC9F00BF2E786D1C06B9E1E04D
:10DF6000252E70D100274FF0010900BF2E782B2EEF
:10DF70000CD02D2E02D0302E0CD103E047F001073B
:10DF80006D1C0AE047F002076D1C06E047F004072D
:10DF90006D1C02E04FF0000900BF00BFB9F1000F97
:10DFA000E4D14FF0000800BF2A2E06D12168081DD9
:10DFB0002060086880446D1C0DE02E78302E01DB57
:10DFC000392E00DD07E06D1CA6F1300008EB88015A
:10DFD00000EB4108E8E700BF4FF0000B2E782E2E33
:10DFE00010D16D1C00BF2E78302E01DB392E00DDE4
:10DFF00007E06D1CA6F130000BEB8B0100EB410B31
:10E00000F1E700BF2E7800BF6C2E01D0682E02D140
:10E010006D1C2E7800E000E0F6E700BF692E21D0ED
:10E0200008DC252E6DD0582E39D0632E0CD0642EEE
:10E030006CD116E0702E4CD0732E3ED0752E1FD0B2
:10E04000782E63D12AE065E02168081D2060D1F8B0
:10E05000009009F0FF00019050460199FCF750FE36
:10E0600055E000BF2168081D2060D1F800905B4694
:10E070000A2249465046CDE90087FEF7BBFE46E03E
:10E080002168081D2060D1F800905B460A224946AD
:10E090005046CDE9008705F0F1FB38E000BF21686C
:10E0A000081D2060D1F800905B461022494650467A
:10E0B000CDE9008705F0E2FB29E02168081D20601A
:10E0C000086801903B4642465046019904F0E8FE3C
:10E0D0001DE02168081D2060D1F8009030215046D5
:10E0E000FCF70EFE78215046FCF70AFE00200821BE
:10E0F0000B461022CDE900104946504605F0BEFB04
:10E1000005E025215046FCF7FBFD00E000BF00BF05
:10E110006D1C03E031465046FCF7F2FD28780028DC
:10E120007FF41AAF00BF9AF80C0010B15046FFF709
:10E13000FCFE00BF0DE72DE9FF470C4615461E46C5
:10E14000DDE90C78684600F00BF9814644EA4500A9
:10E1500040EA860040EA072040EA084109F5E0600D
:10E16000009A40F82210BDE8FF872DE9FF470C46D2
:10E1700015461E46DDE90C78684600F001F9814637
:10E1800044EA450040EA860040EA072040EA0841A8
:10E1900009F5E060009A40F82210BDE8FF872DE9FC
:10E1A000FF470C4615461E46DDE90C78684600F030
:10E1B000F7F8814644EA450040EA860040EA072035
:10E1C00040EA084109F5E060009A40F82210BDE8F5
:10E1D000FF872DE9F84F05460C4600263746B04626
:10E1E000B1460095684600F08BF8824646EA470043
:10E1F00040EA840040EA082040EA09410AF5E0606C
:10E20000009A40F8221000BFBDE8F88F1CB5044604
:10E210000020009003460122114601902046FFF79E
:10E22000A4FF1CBD2DE9F84F06460D4614460027F5
:10E23000B846B9460096684600F082F8824647EA3A
:10E24000480040EA850040EA092040EA04410AF516
:10E25000E060009A40F8221000BFBDE8F88F73B567
:10E260000D46684600F07CF8044604F5E06000992D
:10E2700050F8210020F4403104F5E060009A40F8A5
:10E280002210009950F8210040EA054104F5E060B1
:10E29000009A40F822107CBD3CB503460A4D30CDB3
:10E2A000CDE9004518460BE05DF82040D4F8204544
:10E2B00014605DF820501468C5F82045121D401CFC
:10E2C0005C188442F0D83CBDF043030031B5684689
:10E2D00000F016F804460121009A01FA02F0C4F891
:10E2E0000C0500BF38BD31B5684600F049F804465A
:10E2F0000121009A01FA02F0C4F80C0500BF38BDF4
:10E3000001460868202802D24FF0A04070470878E4
:10E3100000F01F0008600148F8E70000000300500B
:10E3200001460868202802D24FF0A04070470878C4
:10E3300000F01F0008600148F8E7000000030050EB
:10E3400001460868202802D24FF0A04070470878A4
:10E3500000F01F0008600148F8E7000000030050CB
:10E3600001460868202802D24FF0A0407047087884
:10E3700000F01F0008600148F8E7000000030050AB
:10E3800001460868202802D24FF0A0407047087864
:10E3900000F01F0008600148F8E70000000300508B
:10E3A00001460868202802D24FF0A0407047087844
:10E3B00000F01F0008600148F8E70000000300506B
:10E3C00001464A09002312B1012A06D102E04FF0AA
:10E3D000FF3302E040F2FF3300BF00BF01F01F0136
:10E3E00001208840184008B1012070470020FCE758
:10E3F00031B56846FFF7B4FF044600BFD4F81005F6
:10E400000099C84000F0010038BD31B56846FFF7FB
:10E4100077FF04460121009A01FA02F0C4F80805CA
:10E4200000BF38BD31B56846FFF7AAFF0446012199
:10E43000009A01FA02F0C4F8080500BF38BD31B5F2
:10E440006846FFF7ADFF04460121009A01FA02F089
:10E45000C4F8080500BF38BDF8B504460D466DB9CF
:10E4600000946846FFF76CFF06460121009A01FA06
:10E4700002F0C6F80C0500BF00BF0DE0009468462E
:10E48000FFF75EFF06460121009A01FA02F0C6F886
:10E49000080500BF00BF00BFF8BD000001460148ED
:10E4A000084470470060004038B504462046FFF736
:10E4B000F5FF002101602046FFF7F0FF00680090A3
:10E4C00000BF38BD10B504462046FFF7E7FF0068DF
:10E4D000012800D110BD0020FCE7000001490860C0
:10E4E000704700000463004070B504460E46FBF719
:10E4F000BFFB0546681C08B9284670BDE8B2E16854
:10E50000087100BF0A48006928B909480461002061
:10E51000E168086009E006480069C0680068E168D1
:10E52000086003480069C06804602846E5E7000009
:10E53000E0780020704710B5FAF7B4F810BD7047C6
:10E5400038B504460D4605484FF48063044A294611
:10E550000090204600F006F838BD00006D2303004F
:10E56000C05B00202DE9F04F93B082460E4617465F
:10E570009846DDF87090304600F0F5FB18210DA8A4
:10E58000F8F758FF0D97CDF83880CDF84890002562
:10E590002B46082207A9304600F002FC08250998FE
:10E5A0000A90BDF82000ADF82C00BDF82200ADF8AF
:10E5B0002E0000208DF83100079800F0030001289C
:10E5C0001BD107984FEA902B0798C0F3C2008DF833
:10E5D00030000798C0F38314A2002B4601A93046EF
:10E5E00000F0DEFB05EB84050DA80AAB224601A96D
:10E5F0000090584600F0F6FA27E0079800F0030074
:10E60000022822D107984FEA905B0798C0F3C20016
:10E610008DF8300000BFBBF1080F01D2584600E072
:10E62000082004462B46224605A9304600F0B8FBD8
:10E630002544ABEB040B0DAB0AAA214605A800F05C
:10E6400017FABBF1000FE6D100BF304600F099FB8E
:10E6500013B0BDE8F08F000010B502460B4C04EB80
:10E66000C203012906D0022906D0032906D00429B5
:10E6700008D105E0022007E0042005E0187903E056
:10E68000587901E0002000BF00BF10BD60530300B7
:10E6900010B54FF0FF34FFF74EFF04210548FFF798
:10E6A00023FF044600BF01200249C968487100BF2A
:10E6B00010BD0000505303002DE9F04F8BB0FCF764
:10E6C00035FB18B100200BB0BDE8F08F0021B54834
:10E6D000816100BF00BF00BFBFF34F8F00BF00BF0D
:10E6E00000BFA0F5805080680A90AF4804680A987F
:10E6F0002040AE4901EB800A00250026002006904C
:10E7000000BF0AA95046FEF7D4FBB0B1A548806906
:10E7100098B9A6480C3840680A99884207D8A34897
:10E720000C384068A1490C3988600020CBE70A9872
:10E7300020409E4901EB800A00E000E0E1E700BFD5
:10E7400000270AE00A98411C20400A91974951F895
:10E75000200007A941F827007F1C022FF2D3079859
:10E7600000F0030002287AD10798800D05904FF43D
:10E7700048710798B1EB905F02DD0798800D01E0CA
:10E780004FF448708146079869F39F50079009F14C
:10E79000080004900798C0F3C200069084480499CA
:10E7A00000F084FA0546002D57D0284600F0DBFA29
:10E7B0003346082207A9284600F003FB08360A98CA
:10E7C0002040611C081A4FEA8008C14532D9B8F1CF
:10E7D000000F05D00A982040744901EB800000E04A
:10E7E00072480390B8F1000F01D0404600E048465F
:10E7F00000F0FF0BB8F1000F01D06C4800E00020E2
:10E800000290B8F1000F02D0A9EB080000E0002050
:10E81000C0B2019033465A462846039900F0D1FA17
:10E820005E44029828B133462846DDE9012100F014
:10E83000C8FA0BE00A9820405C4901EB800B334694
:10E840004A465946284600F0BCFA00BF0598C01C4D
:10E850000A9901EB90000A9000BF43E0FFE7079898
:10E8600000F0030001283DD10798C0F3831006286B
:10E8700003DA0798C0F3831000E00620079960F3DD
:10E88000891107910798C0F3831000F102080798D7
:10E89000C0F3C20006904FEA8801454800F006FA2E
:10E8A0000546F5B1284600F05EFA3346082207A96E
:10E8B000284600F086FA083600270DE00A98421C28
:10E8C00020400A92394A02EB80013346042228464E
:10E8D00000F077FA361D7F1C0798C0F38310B8420A
:10E8E000ECD800BFDDB32F48D0F81080806918B194
:10E8F000284600F046FA31E019E04FF0000900BF69
:10E90000D8F80C004079012800D18146B9F1000FF8
:10E9100008D000BFD8F8000029460268404690475A
:10E9200000BF00BFD8F80C00D0F8008000BFB8F1DD
:10E93000000FE2D1284600F024FA0020059005A837
:10E94000FBF742F91748806918B918490C390A9839
:10E9500088609DF81400FBF73DF900BF1DE0FFE75C
:10E960001048D0F810800AE0C146D9F8000081684C
:10E970004846884700BFD8F80C00D0F80080B8F1AE
:10E98000000FF1D10B490C4A891AC908022242EA48
:10E9900001400AA100F01CF800BFFCF7C7F980F0A5
:10E9A000010090E6E0780020B02E0020EC68002006
:10E9B00018540300F8530300605303004261636B73
:10E9C000656E647320666C75736865640000000092
:10E9D00070B504460D4600231A462946204604F029
:10E9E0001BFA70BDF8B505460E4614460094012387
:10E9F0006A463146284604F00FFAF8BD2DE9FC417D
:10EA000006460F4614461D460094019502236A46A9
:10EA10003946304604F000FABDE8FC812DE9FE439A
:10EA200006460F4614461D46DDF8288000940195E1
:10EA3000CDF8088003236A463946304604F0ECF9E5
:10EA4000BDE8FE832DE9FF4706460F4614461D46E6
:10EA5000DDE90C8900940195CDF80880CDF80C9083
:10EA600004236A463946304604F0D6F9BDE8FF87EC
:10EA70002DE9F05F07460E4690461D46082E01D947
:10EA8000BDE8F09F95F80C90002028732946404679
:10EA900002F04CF800240CE0B44205D23A5D1DA10E
:10EAA0002846FFF72DFA03E01CA12846FFF728FAB5
:10EAB000641C082CF0D31AA12846FFF721FA002481
:10EAC0001DE0B44216D217F804A0BAF17E0F09DC9B
:10EAD000F8F78AFC006810F80A0000F03E0008B160
:10EAE000504600E02E2083465A460EA12846FFF7E6
:10EAF00007FA03E00CA12846FFF702FA641C082C71
:10EB0000DFD301222946404601F0ECFF85F80C9046
:10EB100000BFB5E72025303278000000202020001B
:10EB20007C00000025630000200000002DE9F0417A
:10EB300006460F4600BF002009490870094800F04A
:10EB40001AF9044614B12046BDE8F081064800F0E9
:10EB5000B5F906480649401AC5080020F4E7000048
:10EB6000E068002018540300A8460300185403006E
:10EB70006053030002480349401AC0087047000070
:10EB8000185403006053030013B50C462146684631
:10EB9000FEF7C4FC28B90448009A00EBC2010868DB
:10EBA0001CBD0020FCE700006053030070B50B485B
:10EBB000046901200A4908700CE000BF0120E168E7
:10EBC000487100BF2546286841682846884700BF2D
:10EBD000E0680468002CF0D170BD0000E0780020EF
:10EBE000E06800202DE9FF4707460C461646984688
:10EBF0000C9D95F80C90002028732946404601F0A2
:10EC000095FF072E47D2DFE806F004090F161F2AEA
:10EC1000370039462846FFF773F93DE03946284664
:10EC20002268FFF76DF937E039462846D4E900231A
:10EC3000FFF766F930E0A068009039462846D4E92D
:10EC40000023FFF75DF927E0D4E90201CDE90001D7
:10EC500039462846D4E90023FFF752F91CE0D4E9ED
:10EC600002122069CDE90012029039462846D4E903
:10EC70000023FFF745F90FE0D4E90223D4E904109B
:10EC8000CDE90023CDE9021039462846D4E9002316
:10EC9000FFF736F900E000BF00BF002229464046DA
:10ECA00001F020FF85F80C90BDE8FF872DE9F84FB3
:10ECB00007468A46388AA0F104080AF10400404455
:10ECC000401EB0FBF8F0C0B200903846FEF719FEC7
:10ECD000044614B90020BDE8F88F002020710121FE
:10ECE0006171A4F8068025460098A0F1010B2C461E
:10ECF0002F604FF0000912E03846FEF702FE06468C
:10ED000036B16079401C60712E603760354604E092
:10ED1000204600F008F80020DDE709F10109D94597
:10ED2000EAD32046D7E72DE9F05F0446274697F857
:10ED300005802646A8F1010B002501E036686D1C10
:10ED40005D45FBD3D6F800A02646002507E0D6F89F
:10ED5000009031465046FEF705FE4E466D1C454577
:10ED6000F5D3BDE8F09F70B5044625460121281D66
:10ED7000FEF785FD70BD10B504462046FEF710FE77
:10ED800010BDF8B5044626460121301DFEF7AEFD44
:10ED900000906D46287810B92046FFF7C4FFF8BDF3
:10EDA0002DE9FC4105460E4614461F4601940120FC
:10EDB0003B4601AA314600902846FEF74AFBBDE8D3
:10EDC000FC812DE9FC4105460E4614461F46019480
:10EDD00000203B4601AA314600902846FEF739FB49
:10EDE000BDE8FC8100BF00BF00BFBFF35F8F00BF65
:10EDF00000BF00BF0021016070470246505808B1B3
:10EE0000012070470020FCE708B50022425042581C
:10EE1000009200BF08BD000010B500200A4908702C
:10EE200000BF0A49086000BF00BF00BF00BFBFF3BA
:10EE30005F8F00BF00BF00BF00BF0549054800F05D
:10EE4000FCFA002010BD0000902E00208C2E002027
:10EE5000C0440300585B002070B50446144D0121E6
:10EE60002846FEF72DFD064600BF00BF00BF00BFCD
:10EE7000BFF35F8F00BF00BF00BF0EB9012000E0ED
:10EE8000002000B970BD042C0BD00A48007818B1DE
:10EE90000748FFF7A7FFF5E7074804700120054979
:10EEA000087003F0E7FC0248FFF79CFF00BFE9E7AA
:10EEB0008C2E0020902E0020882E002000218268B9
:10EEC000916082681161826851618268D160826854
:10EED0005160826811607047024602F5A86050F8E0
:10EEE0002100704700F5A86343F8212070470146D0
:10EEF000D1F80405704708B50022425042580092EC
:10EF000000BF08BD08B5002242504258009200BF21
:10EF100008BDC0F848137047C0F848137047C0F8E0
:10EF200044137047C0F84413704702465058704766
:10EF3000C0F808137047C0F808137047C0F80413EE
:10EF40007047C0F8041370470246D2F80403084023
:10EF50007047012242507047012242507047000022
:10EF6000024A1060121D1160704700002C760040AC
:10EF700001460348085808B1012070470020FCE70B
:10EF80000070004008B50021034A815011464158E5
:10EF9000009100BF08BD0000007000400121014A3F
:10EFA0008150704700700040014609B90E2070473B
:10EFB0000248006808600020F9E7000038470300B5
:10EFC000FEB506460C462046FFF7EEFF05460DB19E
:10EFD0002846FEBD00200090019002908DF8006050
:10EFE00001208DF802000621ADF8041069462020AA
:10EFF000226869DF054675B1284600F0C1FA074668
:10F000004F49504A891AC908012242EA01403A464A
:10F010004D49FFF7E7FC002000900190029001208D
:10F020008DF8010000208DF802008DF8030069467C
:10F030004020226869DF054675B1284600F0A0FA35
:10F0400007463F493F4A891AC908012242EA01405E
:10F050003A463E49FFF7C6FC00200090019002901E
:10F060008DF80060F720ADF8020069462320226881
:10F0700069DF054675B1284600F082FA0746304937
:10F08000304A891AC908012242EA01403A46304909
:10F09000FFF7A8FC002000900190029002208DF85C
:10F0A000000069460120226869DF054675B12846DF
:10F0B00000F066FA07462249224A891AC908012245
:10F0C00042EA01403A462349FFF78CFC00200090B9
:10F0D000019002904FF4C86000906946A120226818
:10F0E00069DF054675B1284600F04AFA074614491B
:10F0F000144A891AC908012242EA01403A461649CF
:10F10000FFF770FC00200090019002908DF8000045
:10F110006946A020226869DF054675B1284600F0DF
:10F120002FFA07460649074A891AC908012242EA06
:10F1300001403A460949FFF755FC002049E7000025
:10F140000854030060530300B4500300FC50030054
:10F15000485103001450030060500300C04F0300E7
:10F160002DE9F04104462568204660DF0646206808
:10F17000A84225D91E491F4A891AC908022242EA13
:10F1800001401DA1FFF724FC19491A4A891AC90830
:10F19000022242EA01402A4623A12368FFF72EFCFF
:10F1A00001F066FE2168471A1149124A891AC908F6
:10F1B000022242EA01403A4628A1FFF713FC00E090
:10F1C00000BF1EB90120304908700EE0304600F043
:10F1D000D7F907460649074A891AC908012242EAAF
:10F1E00001403A4629A1FFF7FDFB3046BDE8F0811A
:10F1F0000854030060530300496E737566666963C3
:10F2000069656E742052414D20616C6C6F6361744E
:10F21000656420666F722074686520536F6674445D
:10F2200065766963652E00004368616E67652074CA
:10F2300068652052414D207374617274206C6F6355
:10F240006174696F6E2066726F6D2030782578204A
:10F25000746F20307825782E000000004D617869A9
:10F260006D756D2052414D2073697A6520666F720D
:10F27000206170706C69636174696F6E20697320BE
:10F28000307825782E000000F72E002073645F622E
:10F290006C655F656E61626C6528292072657475A6
:10F2A000726E65642025732E000000002DE9F04188
:10F2B000ADF5027D80461848007818B90DF5027D3D
:10F2C000BDE8F0811DE04FF4FA70049004A905A890
:10F2D00061DF044604B115E005AD104901A800F056
:10F2E000ACF809E000BF0398064637682846716805
:10F2F000B84701A800F0C2F800BF03980028F1D178
:10F3000000BFE0E700BF052C04D000BF2046FAF79D
:10F31000F1F800BF00BFD1E7F72E00202C47030013
:10F320001CB51B48007808B108201CBD01201949F4
:10F330000870002002F0A6FF112801D10020F4E798
:10F34000002002F0BDFF14480068019000200090EA
:10F350006846FAF739FC114901A810DF04460CB9D8
:10F36000012000E000200A4908709DF80000FAF72B
:10F3700031FC0CB12046D8E7002006490870084946
:10F38000087003F0EBFA012002F09AFF0020CCE7AE
:10F39000F42E0020F62E00200847030035940200CA
:10F3A000F52E00203EB50A49684600F046F809E00F
:10F3B000684600F03FF8044625686068A84768463C
:10F3C00000F05CF8684600F035F80028F0D13EBD4A
:10F3D000FC4603000148007870470000F42E00202E
:10F3E0002DE9FF41074618E003A84BDF044604B1AE
:10F3F00014E00F49684600F020F809E000BF0298C9
:10F4000005462E6869680398B047684600F036F8EC
:10F4100000BF02980028F1D100BFE5E700BF052C2E
:10F4200004D000BF2046FAF765F800BFBDE8FF81B1
:10F430004C47030001468868704770B504460D4686
:10F44000256028686060204600F001F870BD14E077
:10F45000D0E900215268914202D1002181607047B9
:10F460004168096842685268914203D0416809685E
:10F470008160F4E7416808314160E9E710B504466E
:10F48000A06800B910BD2168A06889680844A06020
:10F49000D4E901104968884205D16068083060608D
:10F4A0002046FFF7D4FF00BFECE770B505460E46D7
:10F4B0006C6806E020683146AA68904700B903E00E
:10F4C000246820680028F5D100BF206830602660DD
:10F4D00070BD014648680068704701464A68106878
:10F4E0004A68126822B14A68126812684B681A604A
:10F4F000704710B503460A460020596807E00C68BB
:10F50000944203D114680C60012003E009680C6880
:10F51000002CF4D100BF10BD0246505808B10120A4
:10F5200070470020FCE708B5002242504258009284
:10F5300000BF08BDC0F80813704701224250704751
:10F5400070B502460D4B03F5947413E0E61AF01003
:10F5500000EBD076761003EBC6010D68954201D919
:10F560000C4606E0954202D201F1080301E048682A
:10F5700070BD00BFA342E9D30020F9E7E0440300D7
:10F5800030B504462046FFF7DBFF05460DB90248BB
:10F5900030BD2846FCE70000CC44030001464FF490
:10F5A000A07000EB810080B2704701464FF48030BC
:10F5B0008840704708B5002242504258009200BF70
:10F5C00008BD0021C0F8001570470521C0F80015DE
:10F5D00070470146D1F8C404C1F8C404704702461C
:10F5E000505808B1012070470020FCE708B5002200
:10F5F00042504258009200BF08BDC0F80413704743
:10F60000C0F800127047012242507047034800685A
:10F6100008B1012070470020FCE700000004014011
:10F6200010B500F08DF901200149086000BF10BD40
:10F630001805004001460020054A12790AB18520CC
:10F6400004E0034A11600122014B1A717047000067
:10F65000202E002010B50220FEF7AEFA4FF4827083
:10F66000FEF7A1FA0C20FEF7ADFA00BF00BF034879
:10F670000068C0F300400028F8D110BD1804004015
:10F6800070B5044604B970BD024EA5012846B047C6
:10F6900000BFF8E7914403000146080B40B27047F1
:10F6A0000146080B40B270470146080B40B2704754
:10F6B0002DE9F04706460D46304601F07FF9F0B1DE
:10F6C0003046FBF7BDFBA0F10808404601F002FA06
:10F6D0000446032C08D13046FEF78AFE08B1032009
:10F6E00000E00220074605E0012C01D1022000E0E5
:10F6F0000320074639463046FEF7B1FD2AE0304682
:10F7000001F068F930B33046FBF79AFB0446A000DD
:10F7100000F5807087B220460F4951F8201041F063
:10F7200001020D4941F8202000BF3846FEF7BCFE1B
:10F730007DB13046FBF784FB8146FBF739FB804601
:10F74000B8F1000F04D0012101FA04F0FEF7C6FE63
:10F7500000BF00BFBDE8F087106500402DE9FC4701
:10F7600006460D4617464FF00008304601F018F9DE
:10F7700010B14FF0080864E0A878C0F340023946A1
:10F780003046FBF71DFB0446601C002856D0A878C5
:10F79000C0F3800030BBA87800F0010090B1019662
:10F7A00001A8FEF7DDFD814609F5E060019950F8FA
:10F7B000210020F0020A09F5E060019940F821A03B
:10F7C00000BF0CE095F80190002000904B460246E7
:10F7D000014601903046FEF7AEFC00BF00BF304648
:10F7E00001F0CEF8A878C0F34000D0B128781649CF
:10F7F00051F82410154A1140134A42F824101146BA
:10F8000051F824104FF47C5202EA06224FF44033A0
:10F8100003EA00431A4311430B4A42F8241000BF85
:10F820000EE0A4F108000A49085C297840EA81103A
:10F8300042B2A4F1080006490A5401E04FF004085E
:10F8400000BF4046BDE8FC8710650040FFC0FCFFDC
:10F850009A5900202DE9F041304890F8640018B121
:10F8600008263046BDE8F081002408E02046FEF777
:10F87000A7FD10B1204601F0BDF8601CC4B22A2CCF
:10F88000F4DB002404E02046FBF782FA601CC4B2DB
:10F890000C2CF8DB21485E3000210160818020487B
:10F8A000FFF7FEFE0546062728463946002804DBFA
:10F8B0004A07130E1B4A135408E04A074FEA126C1A
:10F8C000194A00F00F031B1F02F803C000BF00BF5E
:10F8D0001348FFF7E5FE0546284600280DDB00BF6C
:10F8E00000BF00F01F02012191404209920002F185
:10F8F000E022C2F8001100BF00BF00BF00BF4FF4FC
:10F90000BE70FEF7D1FD4FF00040FEF7E7FD01208D
:10F91000024981F8640000263046A3E740590020E0
:10F920000060004000E400E018ED00E0014601F056
:10F930006040B0F1005F01D1012070470020FCE77A
:10F940002DE9F04106254FF08040FFF7A5FE044663
:10F950002046E21704EBD2625211920002F1E0223B
:10F96000D2F800212146E31704EBD3635B11A4EB2B
:10F9700043160123B3401A400AB1012200E00022DD
:10F9800082BB4FF08040FFF787FE04462E4620469C
:10F990003146002804DB4A07130E134A135406E0CD
:10F9A0004A07170E114A00F00F031B1FD75400BF60
:10F9B00000BF4FF08040FFF76FFE0446204600284E
:10F9C0000DDB00BF00BF00F01F0201219140420982
:10F9D000920002F1E022C2F8001100BF00BF00BF98
:10F9E00000BF00BFBDE8F08100E400E018ED00E0DA
:10F9F0002DE9F84307460E46384601F0E9F804467B
:10FA0000D4B14FF00008002000906846FAF7DCF807
:10FA1000207910B14FF0010802E02660012020712A
:10FA20009DF80000FAF7D6F8B8F1000F03D01125C1
:10FA30002846BDE8F88300BF00252846F9E770B5E1
:10FA40000546284601F0C4F8044614B100202060A1
:10FA5000207170BD10B5044600212068FFF779FAC7
:10FA60000220617901EB4101014A505410BD0000B0
:10FA7000442E00202DE9F0430346164658792D4ABE
:10FA800042F82060587900EB40002B4A105C18B116
:10FA900008242046BDE8F08393F904508F78284667
:10FAA0003A46002808DB4FEA427C4FEA1C68DFF840
:10FAB0008CC00CF800800BE04FEA427C4FEA1C69D6
:10FAC000DFF87CC000F00F08A8F104080CF80890DB
:10FAD00000BF00BF93F90420104600280DDB00BFD3
:10FAE00000BF00F01F070125BD404709BF0007F117
:10FAF000E027C7F8005100BF00BF00BF00BF0A8861
:10FB00001868C0F8082500BF08795A7902EB42024C
:10FB1000094D2A445070C8785A7902EB42022A44AF
:10FB2000907001205A7902EB4202A854002420462A
:10FB3000B0E70000402E0020442E002000E400E04A
:10FB400018ED00E02DE9F04104460D464FF48076B3
:10FB5000012731462068FFF7CEF939462068FFF7C4
:10FB6000DEF91DB139462068FFF7E8F9BDE8F081FC
:10FB70002DE9FF4F83B007460C46387900EBC000F3
:10FB80006A4901EB8006307F28B14FF0080A5046E1
:10FB900007B0BDE8F08F3D683A79654B53F8221005
:10FBA0003868FFF725FF18B14FF0110A5046EFE70C
:10FBB0000598306006987060207B012803DC20786F
:10FBC000FEF791FB02E02078FEF72CFC002000906D
:10FBD0000190207800231A460121FEF7C6FA6078CA
:10FBE000FF2808D094F801904846FEF77CFB484671
:10FBF000FEF70CFB01E04FF0FF39A078FF280ED094
:10FC000094F802804FF0010B002000905B46024602
:10FC1000014601904046FEF7A8FA00BF01E04FF010
:10FC2000FF38A07886F82000E078F077E078FF28A9
:10FC30000DD0207918B1E078FEF755FB02E0E078AE
:10FC4000FEF7F0FBE078FEF7E1FA2079B077207854
:10FC5000C5F80805C5F80C95C5F8108500BFA06863
:10FC6000C5F8240500BF217B627B0AB1012300E0B7
:10FC70000023184631B1012906D0022907D00329F3
:10FC800008D000BF00BF08E040F0020005E040F0EF
:10FC9000040002E040F0060000BF00BFC5F85405B4
:10FCA00000BFA079C5F8C00500BF00BF0720C5F898
:10FCB000000500BF306888B33868FFF7F5FC83465D
:10FCC0006179029158460299002804DB4A07130E15
:10FCD000184A135408E04A074FEA126C164A00F01B
:10FCE0000F031B1F02F803C000BF00BF3868FFF7F7
:10FCF000DBFC8346584600280DDB00BF00BF00F048
:10FD00001F02012191404209920002F1E022C2F853
:10FD1000001100BF00BF00BF00BF00BF0020707710
:10FD2000012030774FF0000A504631E7D8590020C3
:10FD30004444030000E400E018ED00E02DE9FC413C
:10FD40000546287900EBC0002D4901EB80042068AE
:10FD500008B32868FFF7A8FC06463046002817DBE2
:10FD600000F01F0201219140264A430942F8231066
:10FD700000BF00BF00BFBFF34F8F00BF00BF00BF79
:10FD800000BF00BF00BFBFF36F8F00BF00BF00BF49
:10FD900000BF00BF00BF2F68206898B11A493846DD
:10FDA000FFF7C8FB607F68B114213846FFF7C5FB39
:10FDB00000BF4FF482713846FFF7AEFB0028F8D041
:10FDC0000020607794F82000FF280CD094F8206081
:10FDD0000020009003460122014601903046FEF7C4
:10FDE000C4F900BF00BF00BF0020C7F8000500BF76
:10FDF0002868FFF724FE00202077BDE8FC81000082
:10FE0000D859002080E100E0520108002DE9F041BE
:10FE100005460E461746287900EBC000154901EB50
:10FE200080044FF00008607F20B14FF01108404679
:10FE3000BDE8F081206820B107F0140008B9012066
:10FE4000607796E80E10C4E9053CC4E90312E07F30
:10FE5000FF2808D0A07F18B1E07FFEF7E3FA02E0A8
:10FE6000E07FFEF740FA3B4632462146286802F022
:10FE7000F5FEDDE7D859002000B5014602480160D3
:10FE800000F004F800BD000004E5014000BF024896
:10FE900000680028FBD0704700E401402CB51949E8
:10FEA000194A891AC908032242EA014017A1FEF73C
:10FEB0008FFD1D48002101601C481B49086000BFE0
:10FEC0001B4804F071F80546002D19D019A00D4902
:10FED0000D4A891AC9080322CDE9000542EA01400A
:10FEE000CA2320A226A1FEF7ADFDFEF7E5FB00BF69
:10FEF00000BF24B100BF2046F9F7FCFA00BF00BFE5
:10FF000000BF2CBDF853030060530300696E697491
:10FF1000207A646174616368616E6E656C207365DC
:10FF20007276696365000000F82C0020393F0300F9
:10FF30002C3100207A646174616368616E6E656C57
:10FF40005F696E697428266D5F7A6872732C20264B
:10FF50007A646174616368616E6E6C655F696E6915
:10FF6000742900007372635C616473313239335FEA
:10FF700073696D706C655F7465737465722E630070
:10FF800025733A2564205A4552524F525F434845E3
:10FF9000434B28257329206661696C3A256400006B
:10FFA00010B1032801D101E000E000BF00BF70479D
:10FFB00010B50446FCF7DAFE014A03C210BD00008A
:10FFC000702E002010B504460548006830B1044882
:10FFD000006803F015F800200149086010BD00001A
:10FFE000602E0020DCB506463078002823D13B2166
:10FFF0001148008876DF044600BF2746002F19D03D
:020000040003F7
:100000000EA01149114A891AC9080322CDE9000737
:1000100042EA014073230EA215A1FEF713FDFEF77D
:100020004BFB00BF00BF25B100BF2846F9F762FABD
:1000300000BF00BF00BFDCBD042F00206572725FEF
:10004000636F646500000000F85303006053030011
:100050002E2E5C6C69627A6E6F726469635C737277
:10006000635C7A626C655F6D6F64756C652E6300AE
:1000700025733A2564205A4552524F525F434845F2
:10008000434B28257329206661696C3A256400007A
:1000900070B50546AE883046FCF796FE044674B14E
:1000A0004FF6FF7340F2F31205F1080104F10A0064
:1000B000FDF710F8607221463046FBF7D3F870BDAB
:1000C0002DE9F0410546EF7BAE88012F01D0BDE858
:1000D000F0814FF6FF70FCF777FE04461CB9042050
:1000E00002F026F9F3E700BF2680002020720E48B8
:1000F0000168C4F80A104068C4F80E0000BF4FF64B
:10010000FF7340F2F31205F1100104F10A00FCF74D
:10011000E1FF60720548C08918B921463046FBF7F7
:10012000A1F800BFD3E70000182E0020945800204B
:100130008188014A91807047D07F0020CA7B012AC4
:1001400002D18A88A0F82424704700002DE9F047E6
:1001500005460F46BE88A81D00EBC6042879A0718D
:10016000F87B012802D0022806D102E028882080EE
:1001700003E06888208000E000BF00BF208861881D
:10018000884236DD22882049204BC91AC908042339
:1001900043EA014033461EA1FEF730FC2188304679
:1001A000A5DF8046B8F1000F02D1012060711FE089
:1001B000B8F1110F0DD1012020711349134A891A8A
:1001C000C908042242EA014032462149FEF70AFCEE
:1001D0000EE04046FFF7D4F981460B490B4A891AD5
:1001E000C908012242EA01404A461AA1FEF7FAFB79
:1001F00000BFA079E179884203DDA1793046FBF7A1
:1002000085F9BDE8F08700006053030060530300E8
:1002100052657175657374696E6720746F207570AF
:100220006461746520415454204D545520746F20EE
:100230002575206279746573206F6E20636F6E6E12
:10024000656374696F6E20307825782E0000000099
:10025000184B030073645F626C655F67617474635D
:100260005F65786368616E67655F6D74755F726501
:10027000717565737428292072657475726E656472
:100280002025732E0000000030B587B00546002001
:10029000039004900590069002208DF80C001749F9
:1002A00003C9CDE9000102A80190154A518990883F
:1002B0006A46ADDF044654B902A8FAF729FB30B10B
:1002C00001218DF812100020ADF8100003E040F27B
:1002D000FD10ADF8100000BF0949888803A9B0DF00
:1002E0000446112CF8D0BDF8100008B107B030BD9D
:1002F0002846FAF757F800BFF8E7000078470300F0
:10030000D07F002070B58EB004460E462C22311DE1
:1003100003A8F7F776F8BDF80C50BDF81000C1B28D
:10032000A01D00EBC500C171A11D01EBC501CA797B
:100330002749284BC91AC908042343EA01402B4620
:1003400025A1FEF75BFBBDF812202149214BC91AFC
:10035000C908042343EA01402BA1FEF743FBBDF883
:1003600010201B491B4BC91AC908042343EA01404A
:100370002AA1FEF737FBBDF816201549154BC91AFF
:10038000C908042343EA014029A1FEF72BFBBDF86D
:1003900014200F490F4BC91AC908042343EA01402E
:1003A00027A1FEF71FFB206980B1294903C9CDE9C8
:1003B0000101ADF80650A01D00EBC500C0798DF815
:1003C000080001A920462269904700BF0EB070BD09
:1003D000605303006053030044617461206C656ED8
:1003E000677468207570646174656420746F20257B
:1003F00075206F6E20636F6E6E656374696F6E201B
:1004000030782530782E00006D61785F72785F6FEC
:1004100063746574733A2025750000006D61785F20
:1004200074785F6F63746574733A202575000000FB
:100430006D61785F72785F74696D653A202575002B
:100440006D61785F74785F74696D653A2025750019
:10045000E84303002DE9F04705460E46341D218888
:10046000A81D00EBC10794F8048022880B490C4BAF
:10047000C91AC908042343EA0140434609A1FEF70B
:10048000BDFAB879404501DAB87900E040468146C6
:1004900020884946FBF73AF8BDE8F087605303002F
:1004A0006053030050656572206F6E20636F6E6E3F
:1004B000656374696F6E2030782578207265717578
:1004C000657374656420612064617461206C656E7D
:1004D000677468206F662025752062797465732EB5
:1004E000000000002DE9F0410646B7883846FCF7C9
:1004F0006BFC05466DB16868F9F743FB044614B11F
:10050000204601F015FF00BF4FF6FF70288000BFA6
:1005100000BFBDE8F08100000549898882889142CA
:1005200000D070474FF6FF71014A918000BFF8E795
:10053000D07F002070B504460E46002084F82E04BB
:10054000B088B4F8241488420CD1207950B9012124
:100550002046F9F748FD054625B1A06B10B12846A5
:10056000A16B884770BD70B504460D46AA88A11DD1
:1005700001EBC200FCF732FE70BD00002DE9FC4724
:1005800006460F46BD88B7F80690B01D00EBC504BF
:100590002B492C4A891AC908042242EA01404B46D9
:1005A0002A4629A1FEF72AFAB9F1170F01DA172016
:1005B00000E0484681462088484501DD484600E085
:1005C00020886080002020710095238862881C4963
:1005D000DFF870C0A1EB0C01C9084FF0040C4CEA25
:1005E000014028A1FEF71AFA21882846B5DF804687
:1005F000B8F1000F0ED04046FEF7C2FF8246104908
:10060000104A891AC908012242EA014052462DA126
:10061000FEF7E8F9607908B1BDE8FC87306968B198
:10062000344903C9CDE90001ADF802506088ADF846
:100630000400694630463269904700BF00BFEBE7CF
:10064000605303006053030050656572206F6E2095
:10065000636F6E6E656374696F6E203078257820E5
:1006600072657175657374656420616E20415454C0
:10067000204D5455206F662025752062797465736E
:100680002E0000005570646174696E6720415454F7
:10069000204D545520746F20257520627974657340
:1006A0002028646573697265643A20257529206F76
:1006B0006E20636F6E6E656374696F6E203078258F
:1006C000782E000073645F626C655F676174747399
:1006D0005F65786368616E67655F6D74755F72658D
:1006E000706C7928292072657475726E6564202596
:1006F000732E0000E04303002DE9FC4105460E4641
:10070000B788B6F80A80A81D00EBC70420884045CA
:1007100001DD404600E0208860806088172801DA0B
:10072000172000E06088608062881149114BC91A67
:10073000C908042343EA01403B460FA1FEF75EF9D6
:10074000286978B1607968B11A4903C9CDE9000117
:10075000ADF802706088ADF80400694628462A6941
:10076000904700BF002060712071BDE8FC8100004F
:100770006053030060530300415454204D545520EE
:100780007570646174656420746F202575206279CA
:10079000746573206F6E20636F6E6E656374696F2E
:1007A0006E20307825782028726573706F6E7365BF
:1007B000292E0000D843030070B50546AE1D3088D1
:1007C0000749C98888420AD10548007E38B1F9F73F
:1007D000B5FD04461CB1024841690220884770BD3E
:1007E000D07F00200548D0E900304FF080729A1881
:1007F00040F100000149C1E900207047682E002047
:1008000070B50546A8880E498988884200D070BD19
:10081000AC1D2078022810D160880949C988884217
:100820000BD1207A042808D0207A062805D0207A17
:10083000052802D0A01CFFF727FD00BFE7E7000056
:10084000D07F00202DE9F04104460D462888262857
:1008500001D0BDE8F081287A012802D0287A022848
:100860000ED1A078F8F7AAFD074639462046F9F7D9
:10087000BAFB064626B1A06B10B13046A16B884783
:1008800000BFE6E72DE9F0410446A51D288812497E
:10089000C98988421DD1688902281AD1B4F8048018
:1008A0004046FCF791FA064696B105F10C00FAF7BE
:1008B00038F820B131464046FAF7D4FC08E07068B9
:1008C000F9F75FF9074617B1384601F031FD00BF6F
:1008D00000BFBDE8F081000094580020FEB504463A
:1008E0000E46B51D002000900190029029882089B5
:1008F00081420FD1688902280CD105F10C00FAF76A
:1009000010F818B1012084F8220029E0002084F8B2
:10091000220025E02988208B81420FD16889022896
:100920000CD105F10C00F9F7FCFF18B1012084F897
:10093000230015E0002084F8230011E02888A18915
:1009400088420DD1E06958B100208DF8000005F112
:100950000C0001906989ADF808106846E169884784
:10096000FEBD01460868012805D00868022802D0AB
:100970000868042801D1012070470020FCE700002E
:1009800070B5024605490B46D40802F007021D5D0A
:100990000126964035431D5500BF70BD9E5900206D
:1009A000014605484056012202EBE07008B10120E3
:1009B00070470020FCE70000705900200146044801
:1009C0004056082801DB012070470020FCE70000AA
:1009D00070590020014606484056002805DB0448AF
:1009E0004056082801DA012070470020FCE700008B
:1009F00070590020FF2201490A54704770590020A5
:100A00002DE9F84F814600BF00244FE02C480057E5
:100A1000401C00B949E0204600F054F8054649461C
:100A20002846FCF7DBFF00283ED0204600F052F8B5
:100A3000064600956846FDF793FC83460BF5E0609B
:100A4000009950F82100C0F301408046B8F1020F30
:100A500001D1032000E00220824651462846FDF7DE
:100A6000FEFB00956846FDF77BFC8346012000995C
:100A70008840CBF8200500BF2846FAF7E1F9834605
:100A8000FAF796F9074677B1032E09D0B8F1020FAD
:100A900001D1012E04D0B8F1030F04D1022E02D1EE
:100AA00031462846B84700BF00BF641C042CADD3B4
:100AB0004846FCF74EFB0028A6D1BDE8F88F0000A1
:100AC0009A59002001460248425C22F0C00070475B
:100AD0009A59002001460248425C90097047000084
:100AE0009A59002070B504460D461646207A05280E
:100AF0000CD0607A28B10A480AA102682846FDF79E
:100B0000FFF909A12846FDF7FBF904E01EB106A193
:100B10002846FDF7F5F92846FDF707FA70BD0000F5
:100B2000C82E0020257300000D0A0000F8B5044609
:100B30000D46E08838B116A00090E38816A218A1EF
:100B40002846FDF7DDF9207A05281FD0607A58B1D4
:100B5000217AA088FDF780FD174951F820603246C0
:100B600016A12846FDF7CCF92846216802F026FB9D
:100B7000A0880021FEF708F80646207A104951F8AF
:100B8000202033460FA12846FDF7BAF9F8BD000032
:100B90001B5B306D000000001B5B313B33316D008F
:100BA00025734C6F67732064726F707065642028C2
:100BB00025642925730D0A00C82E00202573000026
:100BC000B42E00203C25733E2025733A20000000FF
:100BD00001460348814201D1024870470020FCE7EA
:100BE00000200040282E00202DE9F04107460D4648
:100BF00016463C48007808B9BDE8F0813A4C6520BB
:100C0000A0700020607003202070C4F803700020E2
:100C10005AE000EB400115F8213000EBC001E21D65
:100C2000535400EB400135F82110C1F3072300EBCA
:100C3000C001491C535400EB400155F82110C1F389
:100C4000074300EBC001891C535400EB400105EB46
:100C500081010B7900EBC001C91C535400EB40012A
:100C600005EB81018988C1F3072300EBC001091D51
:100C7000535400EB400105EB81014968C1F3074380
:100C800000EBC001491D535400EB400105EB81010D
:100C90000B7A00EBC001891D535400EB400105EBBA
:100CA00081010989C1F3072300EBC001C91D535419
:100CB00000EB400105EB81018968C1F3074300EBBC
:100CC000C00108315354401CB042A2DB06EBC60001
:100CD000C01D1FFA80F84146034803F05EF900BFCB
:100CE0008AE70000112D0020D450002070B5064C7A
:100CF0006820A07000206070032020700325294622
:100D0000204603F04AF970BDD45000202DE9F0418F
:100D100005460E46074C6920A07000206070032035
:100D20002070E570267105273946204603F035F915
:100D3000BDE8F081D45000202DE9F04704460D466F
:100D400016464FF00209022D74D36069A84271D98A
:100D50002078012804D0022849D003280DD15EE074
:100D60002F4607EB5707206A00EB57212046FCF778
:100D7000F1FB8146B9F1000F00D075E038467F1CC9
:100D8000C0F3080104F1300001EB000805F0010098
:100D900028B1F1B298F8000061F31F1000E030466E
:100DA00088F800000120E070206A00EB57212046FF
:100DB000FCF7D0FB8146B9F1000F00D054E0C7F337
:100DC000080104F1300001EB000805F0010010B14A
:100DD000C6F3071006E098F8000000F0F000C6F334
:100DE0000321084388F800000120E0703CE0206AFD
:100DF00000EB15212046FCF7ADFB8146B9F1000F51
:100E000000D031E0B1B240F2FF1202EA450304F132
:100E10003002981801F0C8FF0120E07024E0206A39
:100E200000EBD5112046FCF795FB8146B9F1000F88
:100E300001D019E019E040F2FF1101EA850204F146
:100E400030015018FCF7ABF966F31B00064640F280
:100E5000FF1101EA850204F130015018314601F01A
:100E600097FF0120E07000BF00BF4846BDE8F08753
:100E700002480068810201F1005070470C01001027
:100E800010B586B0694630A0FBF79FFB044630489A
:100E900030490860002C4ED1BDF80400BC2101EBA4
:100EA0006020A0F5FA602C490870BDF80400C0F37A
:100EB00043104870BDF8040000F01F008870BDF8B2
:100EC0000600C012C870BDF80600C0F345100871D6
:100ED000BDF80600C006800E48711E4800680A680A
:100EE0000260496841601B4900980968C860012098
:100EF0001849486019491A4A891AC908032242EA5E
:100F0000014018A1FDF764FD1449154A891AC90862
:100F1000032242EA01400CA215A1FDF763FD0F492F
:100F20000F4BC91AC908032343EA014013A1009AD1
:100F3000FDF758FD05E0002006490968C86005492D
:100F4000486006B010BD0000302E62696E000000DF
:100F5000CC550020802D0020892D0020F85303005F
:100F60006053030066696C656C6973743A00000035
:100F7000206E616D653A2573000000002073697A68
:100F8000653A25640000000010B50446142C01DB0E
:100F9000002010BD21460548FCF754FC21460348BB
:100FA000001FFCF74FFC0120F3E70000B8580020B9
:100FB00070B50546002406E0044901EB840029468B
:100FC000FCF722FC641C1E2CF6D370BDB458002024
:100FD00010B598B00F488068C04317900D4841681D
:100FE00017A8FCF757FC179901A8FAF7B3F82C22B9
:100FF00001A90CA8F6F705FA002405E00DA931F8BF
:101000001400FFF7D5FF641C0C98A042F6D818B066
:1010100010BD0000B058002010B50446214602481B
:10102000FCF7F2FB10BD0000B85800202DE9F04796
:1010300081460E4617464FF00008D9F80040022EB0
:1010400002D36069B04202D80220BDE8F08767B1E0
:1010500000BF4FF0FF3239462046FFF76DFE804655
:10106000B8F1000F01D04046EFE700BF31464846D7
:10107000FBF780FD054605B922E0012D01D10220D4
:10108000E3E7681C08B90120DFE70022314620466B
:10109000FFF752FE8046B8F1000F01D04046D4E77A
:1010A000D4E90410801E814206D22069401C2061D0
:1010B000207940F0010020712E466069B042D5D8F9
:1010C00000BF0020C1E70000042804D102490968DC
:1010D000491C014A11607047F82E002010B50446E3
:1010E0002046FAF764FF08B1FFF77CFB0021204699
:1010F000FAF76DFE10B12046FEF764FF012120468D
:10110000FAF765FE10B12046FEF752FF204601F0C7
:10111000E9FF204600F044F810BD00002DE9F05F23
:10112000834688464FF00D09002088F80000DBE96F
:101130000267FBF71BFE341A67EB01050021084626
:10114000091BA8411ADAB4F5350F05D3F8F798FC56
:1011500011490844002101E03046394682464FF4E7
:101160009603524600210D48FAF737FF8146B9F140
:10117000000F02D10120BDE8F09F03E000210748E5
:10118000FAF71AFEB9F10D0F04D1584601F038FFF5
:1011900088F800000020EEE7FFFFB400582E002082
:1011A000F8B5074655E000BF2B48FEF792F9064612
:1011B0000EB1304600E0002004460025002C40D04F
:1011C0006B1ED4E9021059405840014302D101F08E
:1011D000E1FB3EE02148006808B9012517E01F49FE
:1011E000D4E902300A68D2E90212591A90410ED2AB
:1011F00001251A480068D0E90210AA1E514050404B
:10120000014304D0154801681348FEF74EF9BDB1FB
:1012100001F0C0FB044669462046FFF77FFF58B146
:101220000E48006810B93846FAF7C9FE0B4804604A
:101230009DF8000018B90DE000200849086007E09B
:1012400008E00648006810B93846FAF7BFFE01E02A
:1012500000BFA8E700BFF8BD7C440300602E00205B
:1012600070B504460E462546D5E90010884770BD86
:1012700010B504462046F7F721FD10B942F20100EF
:1012800010BD2046002803DB1F4A125C520905E00E
:101290001E4A00F00F031B1FD25C52091146082999
:1012A00004D20120884000F0EC0008B9002000E0E2
:1012B000012010B942F20200E2E71548806868B1E7
:1012C0006009134951F8200004F01F0201219140E8
:1012D000084361090E4A42F8210012E02046002826
:1012E0000DDB00BF00BF00F01F0201219140420949
:1012F000920002F1E022C2F8001100BF00BF00BF5F
:1013000000BF0020BCE7000000E400E018ED00E0B2
:101310004C5B002070B50446F7F7ECFC054614481A
:101320008068D8B9012012498860124800681249C3
:1013300008400F49086010484FF0E021C1F88001D3
:101340000C488038D0F88400094948604FF0FF31DC
:101350000848001D01600020207001E0012020707D
:101360001DB900BF62B600BF00BF002070BD000005
:101370004C5B002080E100E0FC06FFBD38B5044670
:101380000D4624B1012C1FD0032C38D132E00020AF
:10139000002817DB00F01F0201219140194A430980
:1013A00042F8231000BF00BF00BFBFF34F8F00BF44
:1013B00000BF00BF00BF00BF00BFBFF36F8F00BF03
:1013C00000BF00BF00BF1BE0002000906846F8F798
:1013D000FBFB0D48007808B9FCF7DEFC0A48C06842
:1013E000401C0949C860012088709DF80000F8F78A
:1013F000F1FB05E0FEF714F9FCF7F4FC00E000BF98
:1014000000BF38BD80E100E02C59002070B50146D6
:101410000878821122B1012A1CD0022A26D100E0CC
:1014200000BF087A8009CE7900EB86008E7906F03D
:10143000030600EB8623487900F00F04887AC00980
:101440004E7A06F0030600EB46056019C61F581CCD
:10145000B04070BD487A0C7A00EB0420CC7904F0DF
:101460003F0400EB0443581C8002F2E700BF00BFBA
:101470000020EEE72DE9F04705460E4690463A4833
:1014800090F8230010B11120BDE8F087002401215D
:10149000354880F8231005F08000A8B10624022109
:1014A000314880F8231077202F4981F82800002147
:1014B0002D4880F8291080F82A1080F82B1080F829
:1014C0002C10FF2180F82D1005F07F0126482830D0
:1014D0000155320E601C244928310A54C6F30742D4
:1014E000A01C0A54C6F30722E01C0A54201D0E5407
:1014F000402D02D0482D04D101E0952703E0872735
:1015000001E0FF2700BF00BF601D174928310F54BD
:10151000B8F1020F03D0B8F1030F0AD104E005219E
:10152000114880F8241009E005210F4880F82410A4
:1015300004E001210C4880F8241000BF00BF05F032
:10154000800008B1012002E0074890F8240081469D
:1015500009F10E00C3B2044A38320621A2F110008C
:1015600000F054FE00208FE7645B00202DE9FE436D
:10157000054668784249087042480668B469287888
:1015800020B1012834D002286CD14CE0687880B1B9
:10159000B1464846F9F79CFA074600BFB846B8F18D
:1015A000000F04D000BF4046F7F7A4FF00BF00BF04
:1015B00000BFF8F757F9006820604FF400706060D2
:1015C000304800688069806888B1002000900190F0
:1015D0000290687808B1012000E000208DF8010039
:1015E000A069029069463046A268904700BF43E078
:1015F0002448006880698068A0B1234A07CA8DE842
:101600000700687808B1012000E000208DF8010093
:1016100004F10C000190A069029069463046A2686E
:10162000904700BF28E01748006880698068C0B113
:10163000154A0C32D2E900109268CDE901020091FE
:10164000687808B1012000E000208DF8010004F165
:101650000C000190A069029069463046A26890474C
:1016600000BF09E000BF032700BF0320F7F742FFD8
:1016700000BF00BFBDE8FE8300BF00BFFAE7000067
:10168000942E0020982E0020204603002DE9FC5FB8
:1016900080468946154698F8006098F801000006D3
:1016A00098F8021040EA014098F8031040EA01203F
:1016B00098F8041040EA010B0127FE48808BB0F532
:1016C0000E7F7DD010DC40F21322A0EB020190428D
:1016D00052D004DCD0B1B0F5047F72D12FE00629DE
:1016E0007AD01329F9D1BAE040F26122811A9042EE
:1016F00069D006DCA0F24D20002870D00628ECD17D
:1017000074E10A296CD00F29E7D1FEE12BE2012216
:1017100000214020FFF7AEFE044600BFA246BAF10A
:10172000000F04D000BF5046F7F7E4FE00BF00BF33
:1017300000BF00274FF40471DE48818300BF17B952
:101740000120BDE8FC9F00BF012200214020FFF7DF
:1017500091FE044600BFA246BAF1000F04D000BFBC
:101760005046F7F7C7FE00BF00BF00BF002740F29A
:101770001321D048818300BF0FB90120E1E700BFEA
:1017800000BF26F0030040B100BF0420287000BF56
:101790000021C84881830220D3E700BF03224FF411
:1017A000D5714820FFF766FE044600BFA246BAF195
:1017B000000F04D000BF5046F7F79CFE00BF03E0C7
:1017C00089E0D1E108E04BE100BF00BF002740F213
:1017D0001921B848818300BF1FB90120B1E7D7E0C4
:1017E00072E100BF06F00400A0B9B248807A20F090
:1017F0000700C01CAF49887200BF26F0030040B14B
:1018000000BF0420287000BF0021AA488183022065
:1018100097E700BF0021A7480184807A00F0070005
:10182000032802D14FF0804000E000200190022206
:10183000E9200199FFF71EFE044600BFA246BAF157
:10184000000F04D000BF5046F7F754FE00BF00BFA2
:1018500000BF002740F226219648818300BF0FB9C0
:1018600001206EE700BF06F00400B8B39148807A0B
:1018700020F00700401C8F49887226F0040600BF44
:101880008C48008C401C81B28A480184008CB0F5E1
:10189000FA6F08DD00BF0220287000BF00218548D4
:1018A000818302204DE7022200214120FFF7E2FD63
:1018B000044600BFA246BAF1000F04D000BF504654
:1018C000F7F718FE00BF00BF00BF00274FF40E71EE
:1018D0007848818300BF17B9012032E713E000BFC9
:1018E00000BF26F0030040B100BF0420287000BFF5
:1018F000002170488183022023E700BF06F0010029
:101900000028BDD18EE000BF26F0030040B100BF2B
:101910000420287000BF002166488183022010E760
:1019200000BF47E06348008C401C81B261480184DD
:10193000008CB0F5FA6F08DD00BF0220287000BFF0
:1019400000215C4881830220FBE65A48807A00F03F
:101950000700032802D14FF0804000E000200190F2
:101960000222E9200199FFF785FD044600BFA24647
:10197000BAF1000F04D000BF5046F7F7BBFD00BF1F
:1019800000BF00BF002740F24D214A48818300BFBD
:101990000FB90120D5E600BF00BF26F0030040B11B
:1019A00000BF0420287000BF00214248818302202C
:1019B000C7E600BF06F001000028B3D102220021D3
:1019C0007A20FFF757FD044600BFA246BAF1000F88
:1019D00004D000BF5046F7F78DFD00BF00BF00BF29
:1019E000002740F253213348818300BF0FB9012003
:1019F000A7E600BF00BF26F0030040B100BF0420EF
:101A0000287000BF00212B488183022099E600BF87
:101A10000BF0804030B12748807A20F00800083071
:101A2000244988722348807A00F00700032829D0CF
:101A3000012251025020FFF71DFD044600BFA246BF
:101A4000BAF1000F04D000BF5046F7F753FD00BFB6
:101A500000BF00BF002740F261211648818300BF0C
:101A60000FB901206DE600BF00BF26F0030040B1B2
:101A700000BF0420287000BF00210E48818302208F
:101A80005FE600BF0B4848300A49C860012148386A
:101A90008182012200214920FFF7ECFC044600BFAF
:101AA000A246BAF1000F04D000BF5046F7F722FD5E
:101AB00000BF01E0645B002000BF00BF002740F2D0
:101AC0006B212C48818300BF0FB9012039E600BF8C
:101AD00000BF26F0030040B100BF0420287000BF03
:101AE00000212448818302202BE600BF08F1010871
:101AF000A9F1010000F0FF0900BF00211D48C183CA
:101B000000BF4FF41C71818300BF6B461022494611
:101B1000404600F0B3F8022801DA002011E600BFC9
:101B200000BF00BF9DF8000048B100BF9DF8000055
:101B3000287000BF00210F488183022001E600BF0A
:101B40000C484830FFF762FC0A4948604FF40071C6
:101B50000848018100BF0020287000BF002105480F
:101B600081830220EDE5D2E5002700210148818331
:101B70000320E6E5645B00202DE9F84F06460F469A
:101B800014464FF0010A3C48808B38B1B0F5267FEF
:101B900022D0A0F2A220002867D156E064E096F897
:101BA000008000BF28F0030048B100BF042020706F
:101BB00000BF0021304881830220BDE8F88F00BFBC
:101BC000761C781EC7B200BF00212B48C18300BF1E
:101BD0004FF42671818300BF6B464FF40072394683
:101BE000304600F04BF8022801DA0020E5E700BF9C
:101BF00000BF00BF9DF8000048B100BF9DF8000085
:101C0000207000BF00211C4881830220D5E700BF5F
:101C10001948808A01281EDD012200214C20FFF78F
:101C200029FC054600BFA946B9F1000F04D000BF4A
:101C30004846F7F75FFC00BF00BF00BF4FF0000A47
:101C400040F2A2210C48818300BFBAF1000F01D1FC
:101C50000120B2E700BF00BF0020207000BF0021BC
:101C6000054881830220A8E799E74FF0000A002188
:101C7000014881830320A0E7645B00202DE9F04741
:101C800004460D4616461F464FF001088448C08B97
:101C900040F2D912811A90427AD005DC48B1A0F204
:101CA000C710002875D16EE0072973D01329F9D128
:101CB000DBE0ECE07A48818AC182BDE0002178480F
:101CC0000184FF20764981F82800002174480183AF
:101CD000032180F823105FE07148008C401C81B222
:101CE0006F480184008C44F62061884209DD00BF02
:101CF0000220387000BF00216948C1830220BDE87E
:101D0000F08702E0641C681EC5B215B12078FF2878
:101D1000F8D045B32078FE281CD1641C681EC5B2DB
:101D200004225F4880F82320B54201DD304600E000
:101D300028460146002004E0225C594BDB681A5417
:101D4000401C8842F8D356480183C0680844544A6E
:101D5000D06021E000BF0520387000BF002150484E
:101D6000C1830220CBE710234D4A38320121A2F172
:101D7000100000F04BFA00BF4FF0000840F2C7110E
:101D80004748C18300BFB8F1000F04D10120B6E776
:101D90002CE07DE049E000BF414890F82300032893
:101DA0009AD029E03E48008B301A1FFA80F9B9F129
:101DB000F00F01DD4FF0F00909F0FF033848012171
:101DC000C268283000F022FA3548C06848443449D7
:101DD000C8600846008B484481B23148018300BF87
:101DE0004FF0000840F2D911C18300BFB8F1000FD5
:101DF00001D1012083E700BF2948008BB042D1DB2D
:101E00002748C08A401E81B22548C182022300F1C2
:101E100038020121283000F0F9F900BF4FF0000826
:101E20004FF4F0711E48C18300BFB8F1000F01D11B
:101E3000012064E700BF00251948C08A00287FF40C
:101E40003DAFFF20164981F82800022301F1380236
:101E50000121A2F1100000F0D9F900BF4FF00008F5
:101E60004FF4F6710E48C18300BFB8F1000F01D1E5
:101E7000012044E700BF0021094880F8231000BF7B
:101E80000020387000BF0648C183022037E711E701
:101E90004FF0000800210248C18303202FE7000013
:101EA000645B00202DE9F04706468846144601256C
:101EB000D548808BB0F53B7F70D009DC88B1A0F2AB
:101EC000C320002842D010287DD0212868D1A3E06B
:101ED000A0F20A30002879D0162878D02628F5D12B
:101EE0006CE18AE196F800A000BF2AF0030048B137
:101EF00000BF0420207000BF0021C348818302205E
:101F0000BDE8F08700BFC048807A00F007000128D4
:101F100030D0BD48808A01282CDDBB4801220169F0
:101F20005920FFF7A7FA074600BFB946B9F1000FDD
:101F300004D000BF4846F7F7DDFA00BF00BF00BF7E
:101F4000002540F2C321B048818300BF0DB90120B4
:101F5000D6E700BF96F800A000BF2AF0030040B10A
:101F600000BF0420207000BF0021A7488183022009
:101F7000C6E700BFA448818AC182D2E00021A248FE
:101F80000183042180F82310FF209F4981F8280055
:101F90000846808A012804DDFC2103E05DE012E0B0
:101FA0002CE1FE21984880F82910022300F1380224
:101FB0001946283000F02AF900BF002540F2D3214D
:101FC0009148818300BF1DB9012099E78DE0C7E0EA
:101FD00000BF25E08C48008BC0F500701FFA80F927
:101FE000B9F1F00F01DD4FF0F009874AD368128B89
:101FF000981809F0FF010123834A383200F006F9EE
:102000008148008B484481B27F48018300BF00258E
:102010004FF43971818300BF0DB9012070E700BF13
:102020007948008BB0F5007FD4DB7748C06800F5B5
:1020300000707549C8600321734880F8231003239A
:1020400000F138020121283000F0E0F800BF00253F
:102050004FF43B716C48818300BF0DB901204FE7FD
:1020600000BF694890F83A0000F01F01052915D01B
:102070000B2901D00D2908D100BF0520207000BF19
:1020800000226148828302203AE700BF04202070CA
:1020900000BF00225C488283022031E700215A48B9
:1020A000018433E05848008C401C81B256480184BA
:1020B000008C44F62061884208DD00BF02202070B9
:1020C00000BF002150488183022019E710234E4AA7
:1020D00038320121A2F1100000F098F800BF00256D
:1020E00040F20A314848818300BF0DB9012007E75B
:1020F00000BF002007E0315C21B10022424981F895
:10210000232002E0401C4045F5D300BF3E4890F834
:1021100023000328C6D03C48C08A401E81B23A48FA
:10212000C1823948C08A00287FF428AF3648808AA7
:10213000012859DDFF20344981F82800FD2132486B
:1021400080F82910032300F138020221283000F022
:102150005DF800BF00254FF448712B48818300BF14
:102160000DB90120CCE600BF0021274801840321DE
:1021700080F8231033E02448008C401C81B22248B0
:102180000184008C44F62061884208DD00BF0220F3
:10219000207000BF00211C4881830220B0E610237C
:1021A000194A38320121A2F1100000F02FF800BFC7
:1021B00000254FF44C711448818300BF0DB90120F4
:1021C0009EE600BF002007E0315C21B100220E49ED
:1021D00081F8232002E0401C4045F5D300BF0A48A7
:1021E00090F823000328C6D000BF0020207000BF55
:1021F000002105488183022082E673E60025002144
:102200000148818303207BE6645B00202DE9F843CD
:1022100005460E461746984600BF134890F85800EA
:1022200000906846FCF7BCF881460121009A01FA4B
:1022300002F0C9F80C0500BF00BF00BF3B463246A4
:1022400029460A48CDF80080FBF741FE044600BF4E
:10225000A146B9F1000F04D000BF4846F7F74AF98C
:1022600000BF00BFBDE8F883645B00206846030040
:1022700010B501E001F057FCF7F7E4FA0028F9D1B6
:1022800010BD0000FEB505460C496846FDF7D5F8BF
:102290000DE06846FDF7CEF80446266828466168DA
:1022A000B04708B91120FEBD6846FDF7E7F868465B
:1022B000FDF7C0F80028ECD100BFF4E7C4460300E6
:1022C000FEB505460A496846FDF7B7F80AE06846D4
:1022D000FDF7B0F80446266828466168B0476846AE
:1022E000FDF7CCF86846FDF7A5F80028EFD1FEBD54
:1022F000E046030070B504460D46A1200B49087066
:102300000120487008462168C0F80210A188C180E9
:10231000A1790172093029680160A9888180A979B1
:1023200081711021093801F031FE70BD5432002056
:1023300010B504460348806918B1024881692046F7
:10234000884710BD9458002070B505460E463146AA
:10235000284675DF044624B1112C02D02046FFF731
:10236000E7FF0CB9012070BD0020FCE72DE9F84F14
:1023700088461546002D35D04FF000090A20009000
:1023800000BF08EB09012A460020F6F78FF9044642
:10239000A1442D1BFCB91448007800B920E00126A7
:1023A00006B90FE000BF4FF47A7707B906E0DFF80F
:1023B0003CA04FEA871B5846D04700BF701E061E40
:1023C000F1D100BF0098401E0090009818B900207D
:1023D0000549087004E0012003490870002DD0D1A0
:1023E00000BF00BFBDE8F88F9C2E0020A14603006F
:1023F0002DE9F04707460E4614469A46B86A10B9CA
:102400000720BDE8F0874FF0000836E008EB4801F0
:10241000B86A00EB8105A88800F10209B9F1FE0F46
:1024200001D90C20EDE709F10100218870542088C2
:10243000401C20801620218870542088401C208059
:1024400022889119288801F012FA218808442080F6
:10245000A88800280DDDA86808B90720D1E7AA8858
:1024600023889819A968F4F7CCFF2088A988084424
:10247000208008F1010000F0FF0897F82C0040458B
:10248000C4DC0020BDE70246022082F8310092F849
:10249000240010B10720087001E003200870108AA2
:1024A00088810020C2F8200402F226404860D068EB
:1024B0008860002070470246012082F83100002029
:1024C000C2F8200402F22640486000208860022002
:1024D0000870802088810020704770B504460D4642
:1024E0006069A860208BA88194F8240018B10620A8
:1024F00084F83C0002E0012084F83C00204601F012
:1025000053FA78B10220287504212046FAF789FA97
:10251000064600BF304600B170BD00BF052084F8FC
:10252000310002E0032084F8310004F58260C4F831
:1025300020040020F0E770B504460D46E069A8606D
:10254000208CA88194F8240018B1062084F83C005F
:1025500002E0012084F83C00204601F025FA78B121
:102560000220287504212046FAF75BFA064600BFD0
:10257000304600B170BD00BF062084F8310002E093
:10258000042084F8310004F58260C4F8200400209F
:10259000F0E7000070B5054611480068407E08B1BC
:1025A000062070BD00BF0F4800F1080102682846F0
:1025B0009047044600BF24B90120094909684876BC
:1025C0000BE00F2C09D10849084A891AC9080122D1
:1025D00042EA01400649FCF7FBF92046E1E700002A
:1025E000242F0020EC7F0020F853030060530300E9
:1025F0009051030000BF0A7822F00F020A700A7897
:1026000022F0F0020A7000BF062850D2DFE800F086
:10261000030E1B28354200BF0A7822F00F020A7011
:102620000A7822F0F0020A7000BF40E000BF0A788A
:1026300022F00F02521C0A700A7822F0F0021032C7
:102640000A7000BF33E000BF0A7822F00F02521C6C
:102650000A700A7822F0F00220320A7000BF26E0E9
:1026600000BF0A7822F00F02521C0A700A7822F08A
:10267000F00230320A7000BF19E000BF0A7822F081
:102680000F02921C0A700A7822F0F00210320A70CF
:1026900000BF0CE000BF0A7822F00F02921C0A7003
:1026A0000A7822F0F00220320A7000BF00BF00BF9B
:1026B000704700000EB501F0C5FBF6F79DF8F6F780
:1026C0007BF8F6F729FBF6F755F8F5F747FAF5F733
:1026D00049FAF5F744FA0220F5F7EEFA0220F5F789
:1026E0003FFA03211F20FBF774FD03211F20FBF796
:1026F00070FD00BFFDF7AEF80546002D1AD03DA0D5
:102700004149424A891AC9080322CDE9000542EA33
:1027100001404FF4BA733EA244A1FCF793F9FBF7D2
:10272000CBFF00BF00BF24B100BF2046F6F7E2FE9A
:1027300000BF00BF00BF45480068029003208DF82D
:10274000090002208DF8080000BF414A02A91F209D
:10275000FDF704F80546D5B13E482B492B4A891AA6
:10276000C9080322CDE9000542EA01404FF4BC73D9
:1027700027A22EA1FCF766F9FBF79EFF00BF00BF62
:1027800024B100BF2046F6F7B5FE00BF00BF00BF72
:1027900001211F20FCF78CFFF6F7C6FD29E0F6F7B4
:1027A00041FFFBF789FFFAF7FFFA08B1012000E0CB
:1027B0000020054601F032FD044627480068A0428B
:1027C00016D02548046001F01DFD06460E490F4A4B
:1027D000891AC908032242EA0140204932460B689F
:1027E0001FA1FCF70BF9F8F7BDFA00201B490860A0
:1027F00000BFD4E76E7266785F6770696F74655F5B
:10280000696E697428290000F853030060530300BF
:102810007372635C616473313239335F73696D70F5
:102820006C655F7465737465722E630025733A2559
:1028300064205A4552524F525F434845434B282526
:102840007329206661696C3A25640000984303008F
:102850006991020018480300082D0020E02C002098
:102860002564206368616E6765636F756E743A25D1
:10287000640A000010B50CE000BF2C4880680446D4
:102880002B4800782168884700B910BD2748FCF71D
:10289000F5FD00BF254880680028EDD100BFFCF79A
:1028A00085F900BF00BFFBF707FF0028FBD100BF81
:1028B00000BF1F480078032803D01D480078022875
:1028C0001DD100BF00BF00BF00BF00BFBFF34F8FCF
:1028D00000BF00BF00BF1748006800F4E060164961
:1028E0000843001D1349086000BF00BF00BFBFF3CD
:1028F0004F8F00BF00BF00BF00BF00BFFDE7FCF768
:1029000069FD10B133DF044600BF00BF01200B4951
:10291000086000BF00BF00BF00BFBFF34F8F00BF04
:1029200000BF00BF00E020BFFDE70000585B0020B3
:10293000882E00200CED00E00000FA0500050040A4
:1029400070B504460D462CB901200349487000209B
:10295000F8F7A8FB70BD00002C59002070B51620B8
:10296000FEF786FC044600BF254625B100BF284679
:10297000F6F7C0FD00BF00BF70BD10B500BF00F08E
:1029800009F818B14FF0FF328260C2600028F6D11A
:1029900010BD000010B50448FCF79FFD04460CB1C3
:1029A000204610BD0020FCE77C4403002DE9FE43D7
:1029B00006468846F468357C9648C08A30B900BF20
:1029C000944991F85800FBF73AFD00BF914890F800
:1029D0002300022804D08F4890F8230001287DD1DD
:1029E000A81FC5B2A41D706800784C2803D115B18A
:1029F000681EC5B2641C02E0681EC5B2641C15B135
:102A00002078FF28F8D045B9706800784C2803D1A9
:102A1000681CC5B2641E00E00024002C49D17D482A
:102A200090F82200012844D001208DF80100794857
:102A300090F82200012806D0022805D0042816D0DC
:102A400005281CD117E000BF00208DF800000321ED
:102A5000704880F8221000BFF6F792FF074627B1B2
:102A600000BF3846F6F746FD00BF00BF10E001206A
:102A70008DF800000CE002208DF8000008E000BF97
:102A8000032700BF0320F6F735FD00BF00BF00BFDE
:102A900000BF00BF5F4991F85800FBF7D0FC00BFB2
:102AA00003215C4880F82210016868468847BDE829
:102AB000FE83584890F82300022817D10121554879
:102AC00080F82310277827F0010070B9514890F85A
:102AD00024000E30C3B24F4A383200E00AE006212B
:102AE000A2F10A00FFF792FBE1E700BF002149488D
:102AF00080F8231006200290464890F82200012812
:102B000006D002280BD0042830D0052875D150E01B
:102B10000221404880F822100021818300BF02AAD0
:102B200029462046FEF7B2FD02281EDB00208DF864
:102B300004009DF808008DF805000321354880F851
:102B4000221000BF014691F85800FBF778FC00BF47
:102B500000BF314A4FF080415068C0F8241500BFD3
:102B600000BF2C48016801A888474FE002AA294607
:102B70002046FFF701F802281ADB01208DF8040037
:102B80009DF808008DF805000321224880F82210E6
:102B900000218182C18280F8231000BF014691F894
:102BA0005800FBF74CFC00BF1A48016801A8884791
:102BB0002CE002AA29462046FFF774F902281ADB06
:102BC00002208DF804009DF808008DF8050003210F
:102BD000104880F82210002180F823108182C182E1
:102BE00000BF014691F85800FBF729FC00BF0948D7
:102BF000016801A8884709E0FFE700BF032700BF7D
:102C00000320F6F777FC00BF00BF00BF00BF00BF86
:102C10004DE70000645B00206846030070B586B095
:102C200004460D462E4620788DF804006068029018
:102C3000217A8DF80C10E1680491217C8DF8141034
:102C4000044850F82610044850F8262001A8904760
:102C500006B070BD305A0020205A00202DE9F04700
:102C600004460E4615461F46286818B12868FCF72A
:102C70005DFE28B1A86850B1A868FCF757FE30B9CE
:102C8000002070774FF010084046BDE8F087D5E986
:102C90000001C4F844054FF4A962115100BFD5E901
:102CA0000201C4F834054FF4A762115100BF4FF47C
:102CB0008C712046FCF737FC2046394601F00102B2
:102CC00032B100BF01234FF4AA62135000BF06E0E7
:102CD00000BF00234FF4AA62135000BF00BF01F0F1
:102CE000020232B100BF01234FF4A862135000BFAB
:102CF00006E000BF00234FF4A862135000BF00BFDE
:102D000000BF07F0080018B910212046FCF715FC99
:102D10003068A0B900BF4FF48C712046FCF7FCFB73
:102D20000028F8D0F07FFF281CD0B07F18B1F07FCA
:102D3000FBF7D9FA16E0F07FFBF774FB12E0A1462F
:102D4000012020EA970ABAF1000F04D14021484639
:102D5000FCF7F0FB04E04020C9F8040300BF00BF0B
:102D600000BF00BF4FF0000840468EE770B5064632
:102D70000C461546A9B204F11A0000F015F8307897
:102D8000032804D1290C04F1140000F00DF870BDE3
:102D900000F8011B090A00F8011B090A00F8011BD1
:102DA000090A00F8011B704700F8011B091200F81E
:102DB000011B70472DE9F05F05460E4690461F4601
:102DC000DDF828904FEA154AF8F7EAFF83464AEA09
:102DD0000B42781C00EA09000E4941F8202007EA5E
:102DE000090001EB8004206865F3C50020602068BD
:102DF00068F389102060206866F39F2020602068B7
:102E000020F00300401C2060206820F004002060B7
:102E1000BDE8F09FEC6800202DE9FC47804689461C
:102E200016461C461C480768012201A92046F7F7F0
:102E3000F3FEC0B1019800F1020A002509E056F83E
:102E4000252050460AF1010A3840144941F8202053
:102E50006D1CA542F3D30097224649464046019B8C
:102E6000FFF7A8FF00BF0D480C38007880B10020A4
:102E700000906846F6F7A8FE00BF00BFFBF71CFCF9
:102E80000028FBD100BF9DF80000F6F7A3FE00BFAD
:102E9000FAF7AFF9BDE8FC87B02E0020EC680020FF
:102EA0002DE9F04781460C4615469846002608F065
:102EB0000100A0B105E0641C761C39464846F7F7CE
:102EC0001FFF2778002FF6D104E06D1E2021484611
:102ED000F7F716FFB5421BD9002DF6D118E01CB14B
:102EE0002046F4F7B2FA064604E06D1E202148465B
:102EF000F7F706FFB54201D9002DF6D105E0641CB5
:102F0000761C39464846F7F7FBFE2778002FF6D1A6
:102F1000BDE8F08770B50446204600F043F805464A
:102F2000002D38D1207803282ED1207901282BD1EB
:102F30004202002104F13000FAF782FA4AF65521E4
:102F400004F22E20FFF730FF144904F13000FFF7A0
:102F50001FFF134904F50570FFF71AFF04F506700B
:102F60002169FFF715FF04F50770E168FFF710FF0F
:102F7000E069401CE0626078012304F13001E26AFC
:102F8000F8F78EFE00202071607800221146F8F7D5
:102F900037FD00B10125284670BD00005252614145
:102FA000727241612DE9F04104460027E078F8B1E2
:102FB000E56A607801232A4604F13001F8F770FED3
:102FC00008B1012714E00020E070206A281AA169E6
:102FD00088420DD2A67809E0A069054460780123F3
:102FE0002A4604F13001F8F75BFE761E022EF3D27A
:102FF0003846BDE8F0810246501A20F07F40704705
:103000002DE9FE4304464FF00008334800780128BC
:103010005ED1002C5CD0F9F7A9FED4E90232C01AC7
:10302000914147D3002000906846F6F7CDFD206916
:1030300018B94FF0FF31A160E1609DF80000F6F78C
:10304000C9FD60690190A0690290244A082101A885
:10305000F6F78CFA054600BF2F4627B100BF384669
:10306000F6F748FA00BF00BF002000906846F6F768
:10307000ABFD206988B14FF0FF33D4E9021059400D
:103080005840014309D0D4E902302169591840F170
:103090000000C4E90210012600E000269DF80000AF
:1030A000F6F798FD2EB121460D48FCF7FEF94FF0DA
:1030B00001080DE04FF0FF33D4E9021059405840A9
:1030C000014305D021460648FCF7EFF94FF001080F
:1030D0004046BDE8FE830000642E0020611203001C
:1030E0007C440300F8B50646694620480068FAF7B4
:1030F0006FFB044637E0207820B1012810D0022869
:1031000024D11DE06068D0E902104FF0FF33594030
:103110005840014303D016486168FCF7C6F916E031
:10312000144960680968884203D100201149086089
:1031300005E00F486168FCF7DCF9054600BF06E0D2
:10314000FFF71BFC01200C49087000E000BF00BF26
:10315000694606480068FAF72DFB6946034800688F
:10316000FAF736FB0446002CC5D1F8BD78440300BD
:103170007C440300602E0020642E0020F8B5054634
:103180000E4669460B480068FAF706FB04467CB118
:1031900025706660694607480068FAF727FB28B182
:1031A00000BF0548F8F7E8FE00BF00BF0020F8BDEB
:1031B0000420FCE778440300582E002070470000EC
:1031C00010B531493148F5F78BFF2F490C313048A4
:1031D000F5F786FF00F0ACFF38B1F4F767FD012882
:1031E0000AD00120F4F768FD06E0F4F75FFD02283D
:1031F00002D00220F4F760FDA2202649264A126878
:1032000001EB0211087002202249234A126801EBE7
:10321000021148701C4800681E491F4A126801EBE1
:103220000211C1F802001848C1681A481A4A126807
:1032300000EB0210C0F80610134801691548164A41
:10324000126800EB0210C0F80A1002211148124A5D
:10325000126800EB02108173A2200E490E4A126818
:1032600001EB0211C8730C480068401C0A49086051
:1032700008460068082806D18021064800F086FE2E
:1032800000200549086010BDBC4E0020B82B00206E
:10329000C02B0020D4320020DC2C00202DE9F0438C
:1032A000A3B005460E4690461F46002038800122F6
:1032B00029462448F8F7C4FF8146B9F1000F0DD024
:1032C0002149224A891AC908012242EA01402A46B4
:1032D0001FA1FBF787FB23B0BDE8F0830024194A48
:1032E000802103A8F8F755FF11E001AB02AA1CA149
:1032F00003A8F4F7C7F8029806F8140006EB440197
:1033000001984870641C444500DB07E000BF0D4A8B
:10331000802103A8F8F73DFF0028E6D100BF3C80DC
:1033200009490A4A891AC908032242EA0140234688
:103330002A460DA1FBF762FB0248F8F719FF00BF10
:10334000C9E7000054330020F85303006053030022
:103350006F70656E202573206661696C65640A0074
:1033600025782C25780000006C6F6164202573207F
:103370006366672073697A653A25640A0000000075
:1033800070B586B006460C462146304600F051F92D
:1033900008B106B070BD94F82F0018BB207B02283E
:1033A00002D0207B03281DD1616AA069814219D116
:1033B000E06960626069A06294F82000C0F3401088
:1033C00084F82C00002084F82D00207B032804D1F1
:1033D0002146304600F0C4F93DE02146304600F079
:1033E0008DF838E0142204F10C0101A8F4F709F873
:1033F00094F82F00E0B13046FCF7EBF8054605F0F5
:10340000020018B101208DF8000010E005F0040062
:1034100018B102208DF8000009E005F0010018B194
:1034200003208DF8000002E004208DF8000002E087
:1034300000208DF80000002084F8300094F820006F
:1034400000F0040010B194F82F0018B16846D4E9D8
:103450000021904700BF00BF9BE70146032001F019
:1034600001020AB14FF4024001F002020AB148F22F
:10347000012001F004020AB148F20220704770B541
:1034800005460C46A16A606B884235D200BFD5F86C
:103490001805C0B2626B616A8854606B401C60633F
:1034A000A06A401E616B814209D194F8200000F0AF
:1034B000400020B902212846FCF7A2F818E0A16AD2
:1034C000606B884206D194F8200000F0400008B9F3
:1034D000012070BDA16A606B884209D194F8200078
:1034E00000F0400020B1022084F82D000020F0E719
:1034F00020212846FCF787F80120EAE7F8B50646C0
:103500000C460027344800904FF482713046FCF797
:103510006DF84FF492713046FCF768F84FF48E71F5
:103520003046FCF763F84FF484713046FCF75EF8E0
:103530000020606384F82F00A06A012809D194F864
:10354000200000F0400020B902213046FCF758F876
:1035500003E001213046FCF753F820213046FCF708
:1035600052F894F82D00022803D000213046FCF7D1
:103570004AF8206838B140F28620A060A168304641
:10358000FCF73BF825E002E00098401E0090009810
:10359000002805DD2146304600F04BF80028F3D125
:1035A00094F82F0058B13046FCF713F8054625B1C2
:1035B0002846FFF752FF074600E0032700BF0098A8
:1035C000002806DC3046FBF7FCFF3046FBF7FDFF2A
:1035D00003273846F8BD0000A086010070B50546F7
:1035E0000C46A16A606B884206D2626B616A885C95
:1035F000C5F81C0500BF1AE094F82C0028B11C2166
:103600002846FCF700F8002070BD94F8200000F078
:10361000400040B11C212846FBF7F5FF012084F84B
:103620002D000020F0E714212846FBF7ECFF0120D5
:10363000EAE770B505460C4600264FF4827128462D
:10364000FBF7CDFF28B14FF482712846FBF7CEFF80
:10365000012694F82F0078B14FF492712846FBF7B9
:10366000C5FF4FF48E712846FBF7C0FF4FF48471FD
:103670002846FBF7BBFF5FE04FF492712846FBF74B
:10368000AEFF60B14FF492712846FBF7AFFF1421F3
:103690002846FBF7B8FF012084F82F004CE04FF4D8
:1036A0008E712846FBF79BFF08B34FF48E712846B6
:1036B000FBF79CFF606B401C60634FF492712846DF
:1036C000FBF78DFF60B14FF492712846FBF78EFF38
:1036D00014212846FBF797FF012084F82F002BE0E8
:1036E00021462846FFF77AFF30BB002070BD4FF41B
:1036F00084712846FBF773FFF0B14FF484712846BC
:10370000FBF774FF4FF492712846FBF768FF60B136
:103710004FF492712846FBF769FF14212846FBF706
:1037200072FF012084F82F0006E021462846FFF7AB
:10373000A6FE08B90020D9E77EB1002084F82D004C
:1037400094F82F0038B92146284600F0F1F980F0AE
:10375000010084F82F000020C8E70120C6E7000020
:10376000F8B506460C4600272F4800904FF48271AA
:103770003046FBF73BFF4FF492713046FBF736FFC4
:103780004FF48E713046FBF731FF4FF484713046B1
:10379000FBF72CFF00213046FBF732FF002060636F
:1037A00084F82F0020213046FBF72DFF94F82D00E0
:1037B000012803D008213046FBF725FF214630467B
:1037C000FFF70CFF206838B140F28620A060A168A6
:1037D0003046FBF712FF25E002E00098401E009003
:1037E0000098002805DD21463046FFF722FF00281B
:1037F000F3D194F82F0058B13046FBF7EAFE0546A6
:1038000025B12846FFF729FE074600E0032700BF41
:103810000098002806DC3046FBF7D3FE3046FBF765
:10382000D4FE03273846F8BDA086010030B5044613
:103830001088C01C984201D90C2030BD0220158888
:1038400048551088401C10800A201588485510885B
:10385000401C108015884C551088401C108000209A
:10386000EBE7014608784A7840EA022070470246B2
:103870000A70100A48700220704700002DE9FF4FBF
:1038800081B0884616461F46DDE90E4B45464FF08F
:10389000010A03E0B5FBF6F50AF1010AB542F9D2D7
:1038A000574500D9BA460BF0010098B994B10BF016
:1038B0000200022803D117B93020009001E0202037
:1038C000009004E0641EDDE90010F7F719FA0CB16E
:1038D000A245F7D3012509E0012F01D97F1E04E09D
:1038E000B8FBF5F9B14500D201E07543F4E700BF3C
:1038F00000BFB8FBF5F909FB15880D4810F8091051
:103900000198F7F7FDF9B5FBF6F5002DF1D10BF0B5
:10391000010048B144B104E0641E20210198F7F78A
:10392000EFF90CB1A245F7D305B0BDE8F08F000068
:1039300096440300F8B506463546A8B2F9F744FAAE
:1039400004466CB3207A1749097B88420ADAA8B288
:1039500004F10A01FEF7F8FC074617B1207A401C73
:1039600020721DE0002020720E48007C50B1A8B2E9
:103970003B2176DF074627B1082F02D03846FEF7F5
:10398000D7FC00BF0748406950B100208DF8000007
:10399000A8B2ADF80200034841696846884700BFF5
:1039A000F8BD00009458002010B50446607940B17D
:1039B00094F82E0428B9204600F0B6F808B101208A
:1039C00010BD0020FCE72DE9FC47804689461546DE
:1039D0009A46DDE90A675346022249464046CDE948
:1039E000006700F017F8044600BF204608B1BDE8A4
:1039F000FC8700BF5346102229464046CDE90067A8
:103A000000F008F8044600BF204600B1EFE700BF11
:103A10000020ECE72DE9FF5F07468B4696461D46E2
:103A20000E9C4FF0000920880390C84647E0786854
:103A300000EB880000680190002202A901A864DF61
:103A4000064600BF304610B104B0BDE8F09F00BF8D
:103A50009DF80800704530D1B9F1000F01D0002069
:103A600000E00220009020889DF808100144009892
:103A700001440F98814201DD0C20E5E7B9F1000F08
:103A80000AD12088401C2080208805F800B02088BA
:103A9000401C20804FF001092088421902A901A88A
:103AA00064DF064600BF304600B1CDE700BF218885
:103AB0009DF808000844208000BF08F101083888FC
:103AC0004045B4DCB9F1000F0DD021880398401CAB
:103AD000081A1FFA80FABAF1FF0F01DD0C20B3E7D4
:103AE000039805F800A00020AEE770B504460D4627
:103AF00084B1206870B12068007858B12068C0880F
:103B0000A188884206D121684878F8F741F800F08A
:103B1000010018B100202860092602E02068286012
:103B20000026304670BD7047014691F8300470475A
:103B300070B505460C46A16A606B884207D02846DE
:103B4000FBF73FFD2846FBF740FD002070BD01203C
:103B5000FCE700000148008870470000062F0020A5
:103B6000F0B5ADB0054600BF9DF8A80020F00F00ED
:103B7000401C2A909DF8A80020F0F00010302A90F8
:103B800000BF2868F3F761FC86B232462AA829688C
:103B90007CDF044600BF2746002F1AD08DA0904935
:103BA000904A891AC9080322CDE9000742EA014078
:103BB00040F231138CA294A1FAF744FFFAF77CFD8E
:103BC00000BF00BF26B100BF3046F5F793FC00BF31
:103BD00000BF00BF00202B902C901020ADF8AC004F
:103BE0003C20ADF8AE000020ADF8B0004FF4C87036
:103BF000ADF8B2002BA87ADF044600BF2746002F9D
:103C00001AD074A07649774A891AC9080322CDE9E7
:103C1000000742EA014040F23B1373A27AA1FAF78F
:103C200011FFFAF749FD00BF00BF26B100BF3046C3
:103C3000F5F760FC00BF00BF00BF7B497B48F9F788
:103C4000E7FE044600BF2746002F1AD061A0644952
:103C5000644A891AC9080322CDE9000742EA0140F3
:103C600040F2451360A268A1FAF7ECFEFAF724FDD2
:103C700000BF00BF26B100BF3046F5F73BFC00BFD8
:103C800000BF00BFF7216948F9F7B3FE044600BF43
:103C90002746D7B14FA05249524A891AC908032270
:103CA000CDE9000742EA01404FF4A4734EA256A1A9
:103CB000FAF7C8FEFAF700FD00BF00BF26B100BF4B
:103CC0003046F5F717FC00BF00BF00BF686808B1B9
:103CD00068688047AC2102A8F3F7ACFB02208DF89E
:103CE000080000208DF80A0006208DF80B00012145
:103CF000ADF854104E49169101218DF884104021E1
:103D00002491002125914B482B9002A94A48F6F7AF
:103D1000C8F8064600BF3746D7B12EA03049314A11
:103D2000891AC9080322CDE9000742EA01404FF48D
:103D3000B8732DA234A1FAF785FEFAF7BDFC00BFD7
:103D400000BF24B100BF2046F5F7D4FB00BF00BF81
:103D500000BF01213848F6F7A1F81C2126A8F3F787
:103D600069FB002026904FF4A03027904FF4F020FC
:103D7000289003208DF8A4000020ADF8A6008DF84F
:103D8000A8002E482B902E482C9026A8F6F7E6F98E
:103D9000064600BF3746D7B10EA01149114A891A0D
:103DA000C9080322CDE9000742EA014040F2871327
:103DB0000DA215A1FAF746FEFAF77EFC00BF00BF80
:103DC00024B100BF2046F5F795FB00BF00BF00BF40
:103DD0002DB0F0BD6572725F636F64650000000016
:103DE000F8530300605303002E2E5C6C69627A6EF8
:103DF0006F726469635C7372635C7A626C655F6D39
:103E00006F64756C652E630025733A2564205A45EE
:103E100052524F525F434845434B28257329206631
:103E200061696C3A25640000F1CA0200BC7F002081
:103E3000002F0020A1FF0200887B0020E5FF020088
:103E400053B202007CB503211148F6F7CCF80546C1
:103E500000BF2E46002E19D00EA01149114A891A12
:103E6000C9080322CDE9000642EA014087230EA2D9
:103E700015A1FAF7E7FDFAF71FFC00BF00BF24B158
:103E800000BF2046F5F736FB00BF00BF00BF7CBD7A
:103E9000887B00206572725F636F646500000000BC
:103EA000F8530300605303002E2E5C6C69627A6E37
:103EB0006F726469635C7372635C7A626C655F6D78
:103EC0006F64756C652E630025733A2564205A452E
:103ED00052524F525F434845434B28257329206671
:103EE00061696C3A256400007FB505460C461148AF
:103EF000006890F8230010B9082004B070BD208835
:103F0000F42801DD0720F8E70020009001900290DE
:103F1000039008480068808AADF800000395029479
:103F200001208DF8020003490968098C88B26946AE
:103F3000AEDFE2E7102F0020704700007FB5054696
:103F40000C461148006890F8220010B9082004B00F
:103F500070BD2088F42801DD0720F8E700200090DC
:103F6000019002900390084800688088ADF8000036
:103F70000395029401208DF8020003490968098C19
:103F800088B26946AEDFE2E7102F002013B5044681
:103F900001A92046FFF7D2FF1CBD13B5044601A9B5
:103FA0002046FFF7CBFF1CBDF0B58DB004460E4692
:103FB0005D4804604FF0FF305B49096808845B4B43
:103FC0000FCB08AD0FC500BF14B90E200DB0F0BD6A
:103FD00000BF00BF0EB90E20F8E700BF3068E061F7
:103FE000214608A862DF054600BF284600B1EDE77C
:103FF00000BF20788DF832000120ADF83000A21CFF
:104000000CA9A8DF054600BF284600B1DEE700BFC7
:1040100020216846F3F70EFA0220ADF80000207860
:104020008DF80200F420ADF804000120ADF8060080
:104030008DF80C009DF80D0020F0080008308DF878
:104040000D009DF80D0020F00400001D8DF80D00FE
:1040500000208DF8110001208DF8120000BF60884B
:1040600004F10C026946F6F7F1FE07460FB1384637
:10407000ACE700BF20216846F3F7DCF90320ADF878
:10408000000020788DF80200F420ADF80400012033
:10409000ADF806008DF80C009DF80D0020F0100022
:1040A00010308DF80D0001208DF811008DF81200F0
:1040B0008DF8130000BF6088221D6946F6F7C6FE22
:1040C00007460FB1384681E700BF20216846F3F765
:1040D000B1F90420ADF8000020788DF80200F4203A
:1040E000ADF804000120ADF806008DF80C009DF835
:1040F0000D0020F0100010308DF80D0001208DF81B
:1041000011008DF812008DF8130000BF608804F1D3
:1041100014026946F6F79AFE07460FB1384655E78E
:1041200000BF002052E70000102F00206847030066
:1041300004480068B0F92000401C08B10120704715
:104140000020FCE7102F002070B505460E4606B192
:1041500005B970BD34462888102804D011281CD019
:1041600050282DD127E01849184A891AC908032276
:1041700042EA014016A1FAF72BFCA88800B220847D
:104180002189A888F9F770FA84F822002189A88883
:10419000F9F76AFA84F8230013E00B490B4A891AED
:1041A000C908032242EA01400FA1FAF711FC4FF0BF
:1041B000FF30208405E029462046FCF78FFB00E015
:1041C00000BF00BF00BFC4E7F85303006053030003
:1041D000424C455F4741505F4556545F434F4E4EFA
:1041E0004543544544000000424C455F4741505F01
:1041F0004556545F444953434F4E4E4543544544FE
:104200000000000072B60449096801EB4102C2EBEC
:10421000C11062B670470000F82E002000B572B6DB
:10422000FFF7F0FF4FF47A71B0FBF1F362B6184676
:1042300000BD00007CB54FF480410020FAF776FC09
:10424000044600BF254625B100BF2846F5F752F9C0
:1042500000BF00BFFAF71CFAF6F70AF8044600BFE1
:10426000254625B100BF2846F5F744F900BF00BF39
:10427000F5F722FC044600BF254625B100BF2846BD
:10428000F5F738F900BF00BFFAF7C6FD044600BFD6
:10429000254625B100BF2846F5F72CF900BF00BF21
:1042A000FBF73EF8044600BF254625B100BF28466F
:1042B000F5F720F900BF00BF0020019001A90120FF
:1042C000FAF77EFE044600BF254625B100BF28460A
:1042D000F5F710F900BF00BF01A8FAF741FF044647
:1042E00000BF254625B100BF2846F5F703F900BFFA
:1042F00000BF0F4903C9CDE9000140F6FF70ADF8DA
:1043000000000C4A69460C48FBF7B4FB044600BFAA
:10431000254625B100BF2846F5F7ECF800BF00BFE1
:1043200001210548FBF70EFC0348FBF793FB7CBD1E
:1043300060470300C9100300584703002DE9F0430C
:104340000246104601231C460D460026374600BF94
:10435000202802D24FF0A04803E000F01F00DFF851
:104360002480C44643EA440848EA850848EA062807
:1043700048EA07490CF5E06848F8209000BFBDE81E
:10438000F0830000000300500200000000300240F3
:10439000010000000100000003000000182D0020B3
:1043A000382D0020E02D002000000000000000005B
:1043B00008460300244A0300204A0300184A030069
:1043C00000020000110B040534580020000000001A
:1043D0000338FDD870470000770A00000000000095
:1043E000770A0000000000007ADA000000000000F8
:1043F00000000050000300506E7266785F677069BD
:104400006F74655F696E6974006E7266785F67705D
:10441000696F74655F6F75745F696E6974006E7241
:1044200066785F6770696F74655F696E5F696E69F2
:10443000740000006E7266785F7370696D5F696EFC
:104440006974000031870200598702007370696D3A
:104450005F78666572006E7266785F7370696D5F13
:104460007866657200000000FFFFFFFF0006FF0096
:1044700000000040000000003C5B00200000000045
:10448000782E002017B10200010006000000000095
:104490000338FDD870473031323334353637383948
:1044A00041424344454600002C540300305403006D
:1044B00000000000000000000000000000000000FC
:1044C000A8440300C044030004000000556E6B6E56
:1044D0006F776E206572726F7220636F6465000083
:1044E00000000000E44E030001000000904D0300B6
:1044F00002000000844B030003000000044E030090
:1045000004000000584E030005000000384D030071
:1045100006000000D44C030007000000404E0300DA
:10452000080000004C4D030009000000B04D0300DE
:104530000A000000CC4E03000B0000006C4B03008F
:104540000C000000644D03000D000000344F030018
:104550000E000000304E03000F0000006C4E030000
:1045600010000000A04E030011000000484F03009F
:10457000120000001C4F030013000000B84E03009F
:1045800080000000EC4C030081000000284C030078
:1045900082000000E84B030083000000C84B0300CA
:1045A00084000000044C030085000000104D03004F
:1045B00086000000184E030090000000B44C030079
:1045C00091000000A84B030092000000784D03000A
:1045D00000820000804E030001820000CC4D0300E9
:1045E00002820000E84D030000840000444C0300F8
:1045F00001840000F04E0300028400008C4C030094
:1046000003840000684C030089A90200D1AA0200BB
:1046100045AA020031AB020011AA020081A90200E2
:104620000200000000000000000000000300000085
:104630000000000000000000000100000000000079
:104640000000000001000000000000000000000069
:104650000201000000000000000000000201000054
:1046600000000000000000000000000000300040DA
:104670000000000001000000000000FF06FF000035
:104680000000000400000000000000000000000026
:1046900041E502003FE5020035E5020000000000B0
:1046A0000338FDD870470000C8660020FF010000F5
:1046B000C8680020000000000000000000000000AA
:1046C00000000000B4460300C446030008000000D8
:1046D00098540300A85403000000000000000000EC
:1046E000D0460300E04603000800000088540300A1
:1046F000985403000000000000000000EC46030096
:10470000FC460300080000000010020130540300C2
:10471000385403003854030058540300585403001D
:104720007054030070540300785403000C470300D6
:104730002C47030008000000B82B00207854030029
:104740008054030080540300885403003C47030056
:104750004C47030008000000004002402400040011
:1047600000000641000000009ECADC240EE5A9E01E
:1047700093F3A3B50000406E0200000000000000AB
:1047800050EADA308883B89F604F15F30000C98E75
:104790000040404040404040404041414141414054
:1047A0004040404040404040404040404040404009
:1047B0004005020202020202020202020202020298
:1047C000022020202020202020202002020202029D
:1047D00002029090909090901010101010101010F5
:1047E0001010101010101010101010100202020201
:1047F0000202888888888888080808080808080845
:104800000808080808080808080808080202020240
:1048100040000000914703006E7266785F67706920
:104820006F74655F696E5F696E69742841445331C6
:104830003239335F52454144595F50494E2C20264E
:10484000696E436F6E6669672C206164733132391B
:10485000335F72656164795F70696E5F6972712937
:10486000000000006170705F74696D65725F637253
:104870006561746528266D5F7265636F72645F752C
:10488000706C6F61645F746D722C204150505F5486
:10489000494D45525F4D4F44455F52455045415447
:1048A00045442C205265636F726455706C6F61646F
:1048B0005F746D725F636229000000006170705F59
:1048C00074696D65725F63726561746528266D5FDA
:1048D0007265636F72645F75706C6F61645F666947
:1048E0006E6973685F7061636B65745F7265706F2A
:1048F00072745F746D722C204150505F54494D4565
:10490000525F4D4F44455F53494E474C455F5348B6
:104910004F542C205265636F726455706C6F6164E4
:104920005F66696E6973685F7061636B65745F72FF
:1049300065706F72745F746D725F6362290000004E
:104940006170705F74696D65725F737461727428F1
:104950006D5F7265636F72645F75706C6F61645FC9
:1049600066696E6973685F7061636B65745F7265B9
:10497000706F72745F746D722C204150505F544997
:104980004D45525F5449434B53283330292C20283E
:10499000766F69642A296D5F7265706F72745F64E7
:1049A0006174615F73756D636865636B636F646584
:1049B000290000006170705F74696D65725F6372D9
:1049C0006561746528266D5F677265656E5F6C69E9
:1049D0006768745F6566666563745F746D722C20CA
:1049E0004150505F54494D45525F4D4F44455F52D1
:1049F000455045415445442C20426F6172644C69D6
:104A00006768745F6566666563745F746D725F681E
:104A1000616E646C65722900312E30300000000038
:104A20005344430049464C59544F500052657175E8
:104A3000657374696E6720746F2075706461746546
:104A400020415454204D545520746F202575206208
:104A500079746573206F6E20636F6E6E6563746921
:104A60006F6E203078257820287265747279292E2F
:104A70000000000073645F626C655F6761705F6473
:104A80006174615F6C656E6774685F757064617492
:104A900065282920287265717565737429206F6EE9
:104AA00020636F6E6E656374696F6E203078257851
:104AB0002072657475726E65642025732E00000087
:104AC0005468652072657175657374656420636FE1
:104AD0006D62696E6174696F6E206F662054582034
:104AE000616E64205258207061636B6574206C6540
:104AF0006E6774687320697320746F6F206C6F6EBB
:104B000067206279202575206D6963726F73656314
:104B10006F6E64732E00000073645F626C655F6784
:104B2000617474635F65786368616E67655F6D74F7
:104B3000755F726571756573742829206F6E2063C7
:104B40006F6E6E656374696F6E20307825782072A1
:104B5000657475726E656420627573792C2077694F
:104B60006C6C2072657472792E0000004E52465FA4
:104B70004552524F525F494E56414C49445F444161
:104B8000544100004E52465F4552524F525F534FC0
:104B900046544445564943455F4E4F545F454E4148
:104BA000424C4544000000004E52465F4552524F71
:104BB000525F464541545552455F4E4F545F454EF6
:104BC00041424C45440000004E52465F4552524F10
:104BD000525F4D555445585F554E4C4F434B5F46C1
:104BE00041494C45440000004E52465F4552524FE9
:104BF000525F4D555445585F4C4F434B5F464149BA
:104C00004C4544004E52465F4552524F525F4D55FF
:104C10005445585F434F4E445F494E49545F4641A7
:104C2000494C4544000000004E52465F4552524FE9
:104C3000525F4D555445585F494E49545F4641496E
:104C40004C4544004E52465F4552524F525F424CD3
:104C5000455F495053505F52585F504B545F545218
:104C6000554E4341544544004E52465F4552524FC3
:104C7000525F424C455F495053505F504545525F2B
:104C800052454A4543544544000000004E52465F99
:104C90004552524F525F424C455F495053505F4C12
:104CA000494E4B5F444953434F4E4E454354454450
:104CB000000000004E52465F4552524F525F415035
:104CC000495F4E4F545F494D504C454D454E5445FC
:104CD000440000004E52465F4552524F525F4E4FC5
:104CE000545F535550504F52544544004E52465F06
:104CF0004552524F525F4D4F44554C455F4E4F54B5
:104D00005F494E495449414C495A4544000000000E
:104D10004E52465F4552524F525F4D4F44554C459F
:104D20005F414C52454144595F494E495449414CB9
:104D3000495A4544000000004E52465F4552524FCA
:104D4000525F4E4F545F464F554E44004E52465FA1
:104D50004552524F525F494E56414C49445F53545D
:104D6000415445004E52465F4552524F525F4441B6
:104D700054415F53495A45004E52465F4552524F87
:104D8000525F494F5F50454E44494E470000000076
:104D90004E52465F4552524F525F5356435F484111
:104DA0004E444C45525F4D495353494E4700000015
:104DB0004E52465F4552524F525F494E56414C4902
:104DC000445F4C454E475448000000004E52465F39
:104DD0004552524F525F4452565F5457495F4552B5
:104DE000525F414E41434B004E52465F4552524F37
:104DF000525F4452565F5457495F4552525F444E8A
:104E000041434B004E52465F4552524F525F494E0E
:104E10005445524E414C00004E52465F4552524F4F
:104E2000525F53544F524147455F46554C4C00002A
:104E30004E52465F4552524F525F4E554C4C000009
:104E40004E52465F4552524F525F494E56414C4971
:104E5000445F504152414D004E52465F4552524FC1
:104E6000525F4E4F5F4D454D000000004E52465F71
:104E70004552524F525F464F5242494444454E00BC
:104E80004E52465F4552524F525F4452565F5457FE
:104E9000495F4552525F4F56455252554E000000F1
:104EA0004E52465F4552524F525F494E56414C4911
:104EB000445F4144445200004E52465F4552524FB7
:104EC000525F5245534F5552434553004E52465F31
:104ED0004552524F525F494E56414C49445F464CF1
:104EE000414753004E52465F535543434553530089
:104EF0004E52465F4552524F525F424C455F4950B9
:104F000053505F4348414E4E454C5F414C524541E2
:104F100044595F4558495354530000004E52465F70
:104F20004552524F525F434F4E4E5F434F554E5482
:104F3000000000004E52465F4552524F525F5449A6
:104F40004D454F55540000004E52465F4552524F5A
:104F5000525F4255535900007761726E696E670067
:104F600064656275670000001B5B313B33306D0088
:104F70001B5B306D000000001B5B313B33316D006B
:104F80001B5B313B33326D001B5B313B33336D00B8
:104F90001B5B313B33346D001B5B313B33356D00A4
:104FA0001B5B313B33366D001B5B313B33376D0090
:104FB000696E666F000000006572726F720000001B
:104FC00073645F626C655F6366675F7365742829ED
:104FD0002072657475726E6564202573207768652C
:104FE0006E20617474656D7074696E6720746F20D3
:104FF00073657420424C455F47415454535F4346A8
:10500000475F534552564943455F4348414E4745E4
:10501000442E000073645F626C655F6366675F7354
:10502000657428292072657475726E656420257315
:10503000207768656E20617474656D7074696E6741
:1050400020746F2073657420424C455F434F4D4D73
:105050004F4E5F4346475F56535F555549442E00B8
:1050600073645F626C655F6366675F73657428294C
:105070002072657475726E6564202573207768658B
:105080006E20617474656D7074696E6720746F2032
:1050900073657420424C455F47415454535F434607
:1050A000475F415454525F5441425F53495A452E21
:1050B0000000000073645F626C655F6366675F7326
:1050C000657428292072657475726E656420257375
:1050D000207768656E20617474656D7074696E67A1
:1050E00020746F2073657420424C455F434F4E4ED1
:1050F0005F4346475F4741502E00000073645F6284
:105100006C655F6366675F736574282920726574D8
:1051100075726E6564202573207768656E206174F2
:1051200074656D7074696E6720746F207365742088
:10513000424C455F4741505F4346475F524F4C45A5
:105140005F434F554E542E0073645F626C655F631E
:1051500066675F73657428292072657475726E6561
:1051600064202573207768656E20617474656D70A6
:1051700074696E6720746F2073657420424C455FBC
:10518000434F4E4E5F4346475F474154542E000005
:1051900054686520626F6F746C6F6164657220681B
:1051A00061732077726974652070726F74656374BF
:1051B0006564206974732073657474696E67732005
:1051C000706167652E20546869732070726F68691A
:1051D000626974732073657474696E67207468659E
:1051E000206164766572746973696E67206E616DA3
:1051F000652E2054686520626F6F746C6F61646502
:1052000072206D75737420626520636F6D70696CB8
:1052100065642077697468204E52465F424C5F5344
:10522000455454494E47535F504147455F50524F94
:10523000544543543D3020746F20616C6C6F77206F
:1052400073657474696E672074686520616476653F
:1052500072746973696E67206E616D652E0000005F
:105260006E72665F626C655F676174740000000057
:10527000626C655F6E757300636C6F636B0000003A
:10528000434C4F434B0000004750494F54450000EA
:1052900050525300554152540000000055415254A1
:1052A0004500000053414144430000005350494D24
:1052B000000000005457490050574D005744540017
:1052C0005254430054494D45520000006170705FD4
:1052D000627574746F6E00006170705F74696D65E3
:1052E000720000007077725F6D676D7400000000DF
:1052F000736F72746C697374000000007274745F71
:105300006C6F675F6261636B656E640061707000F3
:105310006E72665F736468006E72665F7364685F66
:10532000626C65006E72665F7364685F736F6300C2
:10533000A8540300B82B002074030000E079020099
:10534000C05503002C2F0020EC600000AE8C020042
:105350009046030000000000FC520300A02E002035
:1053600060520300000004047052030000000000BB
:10537000785203000000000080520300000000008B
:10538000885203000000000090520300000000005B
:1053900094520300000000009C5203000000000033
:1053A000A452030000000000AC5203000000000003
:1053B000B452030000000000B852030000000000D7
:1053C000BC52030000000000C052030000000000B7
:1053D000C452030000000000CC5203000000000093
:1053E000D852030000000000E45203000000000057
:1053F000F0520300000000000C53030000000404FE
:1054000010530300000003031853030000000303BC
:105410002453030000000303A82E0020C05F0020D7
:10542000E85F0020E85F00202C000000DD9902000A
:10543000D9A502000000000021A502000000000024
:1054400099A5020000000000AB9F0200887B0020AD
:1054500045DA0200BC7F0020494103002C310020C6
:1054600049410300D451002059A30200D07F0020FD
:1054700091A6020000000000412903000000000086
:1054800031A4020000000000ADF2020000000000A4
:10549000E1F30200000000007D13030000000000A3
:1054A00045AD0200000000000112160119021103AF
:1054B00012041205120616070F08FF0910100A073A
:1054C0000B070C740D010E020F03100411100A12C9
:1054D0000513391436150616141705181219121A61
:1054E000121B121C121D100A21012220232024024B
:1054F000251226162708280829122A122B122C12E8
:105500002D162E332F303012311232123312341244
:10551000351236123712381239123A123B123C1237
:105520003D123E123F1440FF5012602A62827C0CF2
:105530000214823A0B8211198213780D120E120F87
:10554000398208081B06133B1424150482110B36FC
:10555000284082011A1AFF015306FF022C40293805
:1055600029010936200140092280093E4864B043E0
:1055700003024B011510014011024504A9B55AFF61
:10558000AB14B84F031A58041AB0041A60041A7006
:10559000041A68041A78041A80041A88041A9004F9
:1055A0001A98041AA0041AA8040110128014926513
:1055B0000112020422FFFF14040090D00300000037
:040000050002720182
:00000001FF
